:020000040000FA
:10A000003DB8F39600000000000200005874020002
:10A01000000000000000010000000000000000003F
:10A02000971CDF000000000000000000000000009E
:10A030000000000000000000000000000000000020
:10A040000000000000000000000000000000000010
:10A050000000000000000000000000000000000000
:10A0600000000000000000000000000000000000F0
:10A0700000000000000000000000000000000000E0
:10A0800000000000000000000000000000000000D0
:10A0900000000000000000000000000000000000C0
:10A0A00000000000000000000000000000000000B0
:10A0B00000000000000000000000000000000000A0
:10A0C0000000000000000000000000000000000090
:10A0D0000000000000000000000000000000000080
:10A0E0000000000000000000000000000000000070
:10A0F0000000000000000000000000000000000060
:10A10000000000000000000000000000000000004F
:10A11000000000000000000000000000000000003F
:10A12000000000000000000000000000000000002F
:10A13000000000000000000000000000000000001F
:10A14000000000000000000000000000000000000F
:10A1500000000000000000000000000000000000FF
:10A1600000000000000000000000000000000000EF
:10A1700000000000000000000000000000000000DF
:10A1800000000000000000000000000000000000CF
:10A1900000000000000000000000000000000000BF
:10A1A00000000000000000000000000000000000AF
:10A1B000000000000000000000000000000000009F
:10A1C000000000000000000000000000000000008F
:10A1D000000000000000000000000000000000007F
:10A1E000000000000000000000000000000000006F
:10A1F000000000000000000000000000000000005F
:10A20000B0A1002029A3000031A30000D5A20000C6
:10A21000000000000000000000000000000000003E
:10A22000000000000000000000000000DF630100EB
:10A230000000000000000000E903002045040020A9
:10A2400015CA00004D6201000000000059690100BC
:10A250003BA300009B0400202B6C0100556C010007
:10A26000F568010000000000656201009304002011
:10A27000716901000D690100256901003DC70000F9
:10A2800059C7000075C7000091C70000000000001A
:10A29000000000003BA300003BA300003BA3000024
:10A2A00000000000000000000000000051BB0000A2
:10A2B0003BA30000630000203BA30000000000005F
:10A2C0000348854600F080FB004800470DAC0000C5
:10A2D000B0A1002004207146084202D0EFF30980AB
:10A2E00001E0EFF308807146004A104711C90000F1
:10A2F000084B19680868203080F30988022080F331
:10A300001488BFF36F8F3FBCAE4608BC04BC62B676
:10A3100018470000AC260020EFF3108072B670479B
:10A3200080F31088704700000448804704480047C5
:10A33000FEE7FEE7FEE7FEE7FEE7FEE7F567010062
:10A34000C1A2000030B50B460146002020220124A6
:10A3500009E00D46D5409D4205D31D469540491B59
:10A360002546954040191546521E002DF1DC30BDA2
:10A3700070B500242546002801DA01244042002956
:10A3800001DA01254942FFF7DDFFAC4200D040422F
:10A39000002C00D0494270BDF0B51FB40646002025
:10A3A00082B005464024019100901BE001992246AD
:10A3B0000F46304600F050FA049A059B801A9941E6
:10A3C00010D310461946224600F053F8361A8F4132
:10A3D0000197224601200021009F00F04AF838181A
:10A3E0004D4100902046641E0028DFDC019B009850
:10A3F0002946324607B0F0BDF0B51FB486B0002044
:10A400000090019002900698069980B204900798F7
:10A41000090C02040014114307900027089D0998B5
:10A4200006913E463C4603900398A9B20204000CF4
:10A43000039004982D0C154348430021224600F058
:10A4400018F8C719714110340E46402CECDB384621
:10A45000029A00F00EF8009A019B80180090594172
:10A4600002980191103002904028CCDB00980BB08C
:10A47000F0BD10B5202A04DB0146203A91400020AF
:10A4800010BD914020239C1A0346E340194390409D
:10A4900010BD10B5441A0346944209D28318891896
:10A4A00003E0491E0C785B1E1C70521EF9D210BDD1
:10A4B0000C460443A40703D009E010C9121F10C3BF
:10A4C000042AFAD203E00C781C70491C5B1C521E53
:10A4D000F9D210BDD2B201E00270401C491EFBD27D
:10A4E00070470022F6E710B513460A46044619469F
:10A4F000FFF7F0FF204610BDCAB2401E4178401C55
:10A500008A4202D00029F9D100207047421C01780C
:10A51000401C0029FBD1801A704730B5044600204A
:10A52000034600E05B1C934203D2E05CCD5C401B21
:10A53000F8D030BDF0B507460846584087B0C00F88
:10A54000049048000E46590040084908BC1A88414A
:10A5500005D2384631461E4617460B46024658007D
:10A56000400810434CD0300D039040055900400D79
:10A57000490D0590401A0290402872DA1803012113
:10A58000000B09050843019004980092002805D0AB
:10A590000199524200208841009201900298402186
:10A5A0000A1A01990098FFF764FF05460C466B46AE
:10A5B00007CB00F062F9C0197141039A0E0D002318
:10A5C000D71756401A467A40164344D0049A002AB8
:10A5D0002DD0029A012A039A15DC1205C01A914166
:10A5E00001263605001C7141D20F059ED20700934B
:10A5F000019202962A46234600F05FF907B0F0BDAB
:10A6000038463146FAE71605224A0F46B218C01AF4
:10A61000B74101210905001C4F4100187F41114637
:10A6200018187941E20F10436D19644113E0E207F5
:10A630006D0815436408C2071443039A01261205E6
:10A64000C01A91413605001C7141CE0740083043C5
:10A650004908C01851412A46234600F021F9CDE7A8
:10A66000FFE7049801224000C117121A00238B4112
:10A6700004983146C417381AA141EEE730B40124DA
:10A68000E407634030BC55E730B40124E40761407F
:10A6900030BC4FE70000E0FFF0B51FB488B00B9965
:10A6A0000998002448400999C00F490049080991B8
:10A6B000C0070B990090490049080B910999089827
:10A6C000A64608431CD00B990A98084318D009984D
:10A6D00001244000420D4800410D09982405000363
:10A6E000000B204309900B980003000B20430B90B4
:10A6F00050181C494018002201901446104605E0ED
:10A70000002001460DB0F0BD032801DA034600E049
:10A7100003239C46C11A0AAE0AE05F0008ADED5B58
:10A720004F00F75B7D430027AA187C41491C5B1E44
:10A730006145F2DD410004AB5A522104120C0A4378
:10A74000240C401C0828DFDB019802900099704619
:10A7500001910090059B049A0799069800F0ADF8C6
:10A76000D0E700000DFCFFFFF0B50C465C4085B063
:10A77000E40FE40703944C00002664085900944653
:10A78000490802460296224321D062460A431ED05F
:10A790006200570D4A000E032303550D01240246A3
:10A7A0002C492405781B1B0B360B401823432643EA
:10A7B000614600901C46501AB44103D30098401CD7
:10A7C000009002E0921800985B41002803DA002014
:10A7D000014605B0F0BD0020012109050746864667
:10A7E00011E064461D46141BB54106D36546521B55
:10A7F000B341744607430C43A646CD0740084908B9
:10A80000284392185B4105460D43EAD11046184390
:10A8100013D06046194650407140084306D0604648
:10A82000101AB34106D20122002306E000220123C0
:10A83000DB0702E00122D243531000987446010561
:10A84000381C6141029C039D0019694100F028F801
:10A85000BFE70000FD03000010B5202A04DB084616
:10A86000203AD040002110BD0B46D340D0402024D8
:10A87000A21A91400843194610BD10B5202A06DBE4
:10A88000CB170846203A1041C1170B4306E00B4690
:10A890001341D0402024A21A91400843194610BD0C
:10A8A00010B5002B08DA0024401C614192185B416E
:10A8B0001A4301D14008400010BDF0B51FB482B06A
:10A8C00005460C0003D008460CF004FA02E00CF038
:10A8D00001FA20300246009021462846FFF7C9FDC4
:10A8E000049B059A04460F4618431143084314D0AD
:10A8F000184610431BD0009840210A1A18460599A3
:10A90000FFF7AAFF05460E46009A05990498FFF73F
:10A91000B0FD084305D0012004E02046394607B0C9
:10A92000F0BD0020C11705430E432C433743009967
:10A930000E986305401A7905E40A00220C43FD0ACB
:10A940000A3002D500200146E9E7010510196941E6
:10A950000C9C0D9D00196941FFF7A2FFDFE7000085
:10A960004A0009030123090B1B0519430A4B10B5C3
:10A97000520D9A4202DA0020014610BD064B3433D4
:10A980009A4203DC9A1AFFF767FF10BD034BD218F7
:10A99000FFF76FFD10BD0000FF030000CDFBFFFFC0
:10A9A00010B5002904DB0124E40740428C41214614
:10A9B000002B04DB1C460123DB075242A3419942D2
:10A9C00000D1904210BD0000064C0125064E05E066
:10A9D000E36807CC2B430C3C98471034B442F7D3C0
:10A9E000FFF772FC2CEF02005CEF020070B58C18D0
:10A9F0000578401C6B075B0F01D10378401C2A11BE
:10AA000006D10278401C03E006780E70401C491CF9
:10AA10005B1EF9D12B0705D40023521E0DD40B70F9
:10AA2000491CFAE70378401CCB1A921C03E01D78FE
:10AA30000D70491C5B1C521EF9D5A142D8D30020D1
:10AA400070BD000003B40148019001BDF10F00206A
:10AA500003B40148019001BD7B05002003B4014807
:10AA6000019001BD1705002003B40148019001BD0C
:10AA7000C506002003B40148019001BD9F0C0020D1
:10AA800003B40148019001BDCF07002003B4014881
:10AA9000019001BD910B002003B40148019001BD5C
:10AAA0004910002003B40148019001BD150B00209E
:10AAB00003B40148019001BD7B07002003B40148A5
:10AAC000019001BDCD0C002003B40148019001BDEF
:10AAD000C106002003B40148019001BD952000206B
:10AAE00003B40148019001BD8907002003B4014867
:10AAF000019001BD530B002003B40148019001BD3A
:10AB0000D520002003B40148019001BDED150020BF
:10AB100003B40148019001BDE508002003B40148D9
:10AB2000019001BD7510002003B40148019001BDE2
:10AB30002310002003B40148019001BD1308002038
:10AB400003B40148019001BDC109002003B40148CC
:10AB5000019001BDB520002003B40148019001BD62
:10AB60004F07002003B40148019001BDC10C002033
:10AB700003B40148019001BDC70C002003B4014893
:10AB8000019001BDD121002003B40148019001BD15
:10AB9000FB06002003B40148019001BD65070020B9
:10ABA00003B40148019001BDF31B002003B4014828
:10ABB000019001BDA507002003B40148019001BD2B
:10ABC000590E002003B40148019001BD0922002064
:10ABD00003B40148019001BD7520002003B4014871
:10ABE000019001BD2D04002003B40148019001BD76
:10ABF0001901002003B40148019001BDBD040020EB
:10AC000003B40148019001BD6902002082B020F028
:10AC1000EDFF1CF0C9F80D481FF08AF91EF0C0FDC9
:10AC200001F0FAFD7D20C0001BF036FF0520400337
:10AC3000074A0168914207D181690091C38A427D28
:10AC4000017D04A00CF018F81EF042FDC16C01005B
:10AC50003DB8F39641505020696D61676520686585
:10AC60006164657220636865636B207061737365EE
:10AC7000642C20696D6167652076657273696F6EFB
:10AC80003A2025642E25642E25642E25640A0000B2
:10AC900070B5014660313F4C4A7D2270CA7D6270BA
:10ACA0004A780B781102194361813022A17B125C32
:10ACB000890992068901920E1143A173014642311E
:10ACC0004B7F0A7F19060914114321810146403147
:10ACD0004A7F0B7F12021A43E280C97EA1700146AF
:10ACE00041314A7E0B7E11021943A1800146623137
:10ACF0004B780A78190609141143A1810146A03145
:10AD00004A7F0B7F12021A43A2858A1C557F137F4C
:10AD10002A0612141A43E2850246C03256781546B6
:10AD20001378320612141A432286C230427803780E
:10AD300010060014184360861C221748FFF7A9FB71
:10AD40002A79E97910466A79090612021043AA792C
:10AD50001204104308436063082029180A7810463B
:10AD60004A78120210438A78C978120410430906FF
:10AD70000843A0630C2029180A7810464A7812026A
:10AD800010438A78C9781204104309060843E06327
:10AD900070BD0000542C0020632C002030B5044608
:10ADA00089B000200090019002900390481C034657
:10ADB0001D7828465D782D0228439D78DB782D0488
:10ADC00028431B0618430B78000218430090481DC7
:10ADD00003461D7828465D782D0228439D78DB7850
:10ADE0002D0428431B0618430B79000218430190D9
:10ADF0000846093003461D7828465D782D02284311
:10AE00009D78DB782D0428431B0618430B7A00023B
:10AE10001843029008460D3003461D7828465D7899
:10AE20002D0228439D78DB782D0428431B06184308
:10AE30000002097B08430390501C01460B7818461A
:10AE40004B781B0218438B78C9781B0418430906FA
:10AE500008431178000208430490501D01460B7806
:10AE600018464B781B0218438B78C9781B0418438B
:10AE7000090608431179000208430590104609307D
:10AE800001460B7818464B781B0218438B78C9781B
:10AE90001B04184309060843117A00020843069070
:10AEA00010460D3001460B7818464B781B021843AC
:10AEB0008B78C9781B04184309060843117B0002EC
:10AEC0000843079004A80DF02FFA68460DF04EF9DC
:10AED000102269462046FFF7B5FD012009B030BDBC
:10AEE00010B5102000F040FB05490028086000D094
:10AEF0000120292303A209490EF0B4FD10BD000072
:10AF0000C02B00202E2E5C2E2E5C737461636B5C54
:10AF100063727970745C6165732E63000000830254
:10AF200070B5254D254E287B254C002801D00128E1
:10AF300017D16068002800D001204523DB0021A242
:10AF400027490EF08FFDA068002800D00120254B76
:10AF50001CA225490EF086FD287B00280AD0012876
:10AF60001BD0C0B2022804D17D20C0012061400066
:10AF7000E06070BD616810208847A068804720614C
:10AF80006061A061E0612062606202460023A0620D
:10AF900030461946FFF700FAEAE761681020884753
:10AFA000A068804702460023206130461946FFF71B
:10AFB000F3F9E06070BD0000789500200080841EE9
:10AFC000589500202E2E5C2E2E5C737461636B5C92
:10AFD000636F6E74726F6C6C65725C62622E63007C
:10AFE0000000EEEE290200000100EEEE10B5142183
:10AFF000092000F015FB0C4C20680C490843206028
:10B0000016210A2000F00CFB206809490843206043
:10B0100015210B2000F004FB6068064908436060BE
:10B0200006490548086010BD0000034010001000EC
:10B03000800080000100010041B000005895002010
:10B0400010B51421092000F0EBFA0B4C20680B49D5
:10B050000843206016210A2000F0E2FA206808491F
:10B060000843206015210B2000F0DAFA60680549DA
:10B070000843606010BD0000000003401000100095
:10B080008000800001000100F8B5214E0746307CA9
:10B09000204C002806D0012800D1E0680020307440
:10B0A000FFF7D6FC1C498A68022002438A608A683E
:10B0B00082438A60194A53695B1D1361D368012575
:10B0C0005B085B002B43D36000220A622946FFF72E
:10B0D000C5FC09F029FC012100220846FFF7C4FC49
:10B0E0000F48A0630F486063A16A38468A09791E39
:10B0F00089069201890E1143A162FFF7BBFCE0684B
:10B10000010909010A200843E0603574F8BD000018
:10B1100078950020000802504004025000000250C0
:10B120005555550029417671F7B5294E294F307C88
:10B130000C46002806D0012800D1F86800203074A1
:10B14000FFF786FC244881680222114381608168F0
:10B150009143816021494B695B1D0B61CB680125DF
:10B160005B085B002B43CB6000210162294610463F
:10B17000FFF774FC09F0D8FB012C06D0022C04D098
:10B18000032C06D0042C06D00AE0214600220846F3
:10B1900004E0022200E0012203210846FFF764FCDC
:10B1A0000F48B8630F4878630098B96A8A09411E4E
:10B1B00089069201890E1143B962FFF75BFCF868BA
:10B1C000010909010A200843F860357403B0F0BD95
:10B1D0007895002000080250400402500000025000
:10B1E0005555550029417671F7B52F4E2F4C307CBF
:10B1F0000D46002806D0012800D1E06800203074F8
:10B20000FFF726FC2A48816802273943816081685C
:10B21000B9438160274A5169491D1161D1684B08C2
:10B220005B0001211943D1600021016201213846F0
:10B23000FFF714FC09F078FB012100220846FFF714
:10B2400013FCE8001D4A10301B498018FFF77AF8FC
:10B2500019494843963080B20299A061206BFF22C1
:10B26000120190432A0102432263206B020912015A
:10B270000807000F104320631148A0631148606362
:10B280000098A16A8A09411E89069201890E11431C
:10B29000A162FFF7EFFBE0680109090109200843FB
:10B2A000E060377403B0F0BD7895002000080250CC
:10B2B0004004025000000250710200003102000000
:10B2C0005555550029417671FFB5414E81B0307C0E
:10B2D0001C460D46002807D0012801D13D48C06812
:10B2E00000203074FFF7B4FB3B498A680220024318
:10B2F0008A608A6882438A60384A53695B1D136199
:10B30000D3685F087F0001233B43D36000220A62B9
:10B310000121FFF7A3FB09F007FB012C06D0022C4B
:10B3200004D0032C08D0042C04D00AE021460022CB
:10B33000084604E0012200E0022203210846FFF74C
:10B3400093FBE8002F011030022C04D0032C05D011
:10B35000042C08D00AE0A800083007E08D21A801DD
:10B36000C900401802E08520800038181D4A1C4999
:10B370008018FEF7E7FF1A49164C4843963080B212
:10B380000399A061206BFF221201904307432763BA
:10B39000206B020912010807000F104320631248B6
:10B3A000A063124860630198A16A8A09411E890658
:10B3B0009201890E1143A162FFF75CFBE06801096D
:10B3C000090109200843E0600220307405B0F0BD97
:10B3D00078950020000802504004025000000250FE
:10B3E0007102000031020000555555002941767167
:10B3F00010B507480024017C012903D10549C9681B
:10B40000C9004C0C00210174FFF722FB204610BD3F
:10B410007895002000080250F8B53949FF224A7398
:10B42000087300248C730A20C8733648364A0460B7
:10B430000C74D0680125800700280FDBD06802213A
:10B4400088430143D1603C22002100940098401CB5
:10B4500000900728FADB491C9142F6D3FFF760FD04
:10B4600001200146FFF7FAFA09F056FB274E306932
:10B4700010218843084330610021C943F16024480A
:10B48000816142690C210A43426142698A434261F7
:10B4900082698A4382611F4988690122D2039043ED
:10B4A000104388611C49086BD20190431043086324
:10B4B000886A9043886219488463C463184CE069C1
:10B4C0002843E061174908257068284001D1491ECA
:10B4D000FAD2FF238233144A14490EF0C3FAB0683B
:10B4E0002843B060B068A843B060206A0090684606
:10B4F0000AF08EFFE06940084000E061F8BD0000FE
:10B500007895002058950020000002504004025019
:10B51000800802504008025000080250C0810250CA
:10B5200080040250FFFF0000F4B50000000082021A
:10B5300030B4C01C0B49830808689B004C68024665
:10B54000850702D080088000001DC3189B1AA34203
:10B5500002D930BC002070479A180A60E21A4A608B
:10B5600030BC70470C2B002030B4C01C0B4A830841
:10B5700090689B00D4680146850702D0800880004F
:10B58000001DC3185B1AA34202D930BC00207047CB
:10B5900059189160E11AD16030BC70470C2B002023
:10B5A000F8B5114CE06901210843E0610F49104DE5
:10B5B00008266868304001D1491EFAD2FF23823341
:10B5C0000CA213490EF04EFAA8683043A860A86890
:10B5D000B043A860206A009068460AF019FFE0694D
:10B5E00040084000E061F8BD80040250FFFF000009
:10B5F000400402502E2E5C2E2E5C737461636B5CD3
:10B60000636F6E74726F6C6C65725C62622E630045
:10B6100000008202014A91605060704758950020F6
:10B620008208800710B4800F002A0FD0084B9200C8
:10B63000D2181368062460433F2484408906890E8B
:10B64000A34381401943116010BC7047014AF0E7E1
:10B65000A804025098040250094A8018C208202AFF
:10B6600001D2084801E00848203A01230029016876
:10B6700002D09340194301E0934099430160704721
:10B680000080FDAFF8810250FC81025010B540B23D
:10B6900009F0D0FB10BD0000F8B546480269402112
:10B6A0000A43026102698A430261434DEC68434EDA
:10B6B000200717D5E86888430027E860E96810206C
:10B6C0000143E960E9688143E960B068002802D07D
:10B6D000B1680120086009F08BFFB068002801D034
:10B6E000B0680760A00506D5E96880200143E960DD
:10B6F000E9688143E960324C206987B2380735D563
:10B70000F068002802D0F168012008601020FFF7DF
:10B71000B7F92C48C069002800D0804709F0A6FD81
:10B720006169082001436161616981436161214868
:10B73000826802210A43826082688A4382602248CA
:10B74000C068002808D0007D012805D0052803D056
:10B75000062801D0042803D1E86840084000E860CA
:10B76000F068002802D0F16800200860780708D54A
:10B77000FFF78CF9616904200143616161698143CC
:10B780006161F80707D06169012001436161606967
:10B79000400840006061B80706D561690220014396
:10B7A00061616169814361610648C069002800D018
:10B7B0008047F8BD4004025000000250A4960020CB
:10B7C00080080250109900203C2B002010B5062262
:10B7D000FEF7A3FE002801D0002010BD012010BDFF
:10B7E00010B50BF0B4FA10BD81024118064A4900A9
:10B7F000114082028018054A40011040014304486C
:10B8000041430802000E70471021020040840800E6
:10B810000101010010B443780278190E1B028478EC
:10B820001A43230C24042243C4781943230A1943DE
:10B83000037924061943437922431B021943837970
:10B84000C0791B0419430006014310BC1046704721
:10B85000044A0029D16A01D0014300E08143D1624A
:10B860007047000000000440044A0029116B01D019
:10B87000014300E081431163704700000000044071
:10B8800010B504460AF022FE154801210268890716
:10B8900014488C4208D014498C4205D013498C427C
:10B8A00002D013498C4202D14069000C0DE01149CD
:10B8B0008C4208D010498C4205D010498C4202D0ED
:10B8C0000F498C4209D14069000D0007000F04D0D8
:10B8D00041001046FEF736FD10BD104610BD0000B9
:10B8E00020250020000004400030004000100040EF
:10B8F0000080004000100140003001400040014045
:10B900000050014070B52C4B5A69032109028A434B
:10B9100001242A49002806D0C51FF93D0ED0FF3D5D
:10B92000012D45D129E0D8692043D861D869C001EB
:10B930003ED40846491E0028F8DC39E05D6A062638
:10B9400035435D625D6A25435D620024002806D0B0
:10B95000C51FF93D05D0FF3D012D05D103E0DC6990
:10B9600002E05C6A00E09C6AE50103D40D46491ED2
:10B97000002DEBDCFF20013019E09D6A25439D621C
:10B980000024002806D0C51FF93D05D0FF3D012D3C
:10B9900005D103E0DC6902E05C6A00E09C6AE50135
:10B9A00003D40D46491E002DEBDC0120400202436A
:10B9B0005A610AF08BFD70BD0000044080F5200044
:10B9C00010B40822174B002802D0082803D005E045
:10B9D000986A904301E0986A10439862986A04223A
:10B9E00090439862986A08439862986A01210843D4
:10B9F00098624A020C480CE0002A06D0D41FF93C99
:10BA000005D0FF3C012C05D103E0D96902E0596A59
:10BA100000E0996ACC0103D40446401E002CEBDC04
:10BA200010BC70470000044080F520000248016807
:10BA300001221143016070470000074010B40E4A14
:10BA40000E4B0021002806D0C41FF93C05D0FF3C56
:10BA5000012C05D103E0D96902E0596A00E0996A36
:10BA6000CC0106D41446521E002CEBDC10BC002086
:10BA7000704710BC0120704780F520000000044092
:10BA80000D484168CA024A4081684160C1688160CE
:10BA90000368C360D90C5940130A534059400160F0
:10BAA0008801064AC90E515C800909060843044909
:10BAB0000843044908407047402C002000EB020076
:10BAC00031080402FBFD7EFF0C484168CA024A406F
:10BAD00081684160C16881600368C360D90C5940C6
:10BAE000130A53405940016048078A05400F920FDE
:10BAF000C9038018C90F4018401D7047402C002012
:10BB000010B4002A07D058234B431B18DC69240BC0
:10BB100024031443DC610722D2018018026AFF2348
:10BB200002338B401A43026210BC704758225143C3
:10BB30000818C0698005800D704700000122034885
:10BB40008A4001789143017070470000242500204D
:10BB500010B500F001F810BDF8B55448006A544E15
:10BB6000C007012700285DD00025B16A3846A840EB
:10BB7000014254D04F4988633820294641434E48FA
:10BB80000C182C20005D012804D0022831D0032895
:10BB900045D139E029464948FFF7C8FFE18E4018F2
:10BBA000E086A18E081A02B2002A09DD0120800277
:10BBB000824200DB421E29464048FFF7A1FF2EE0EB
:10BBC000E06900282BD0A0688002800F022802D0F4
:10BBD000012805D008E0616800202031487203E0A8
:10BBE0006168002020310872E28E1320E369216B26
:10BBF00014E029463148FFF7A1FF236A002B03D048
:10BC0000A28E2320216B984729462C48FFF796FFE8
:10BC1000636A002B03D0A28E2320216B98476D1CF2
:10BC2000022DA2DB214A106A022381070420002989
:10BC30000BDA316BC90700D01760316B890700D56B
:10BC40001360316B490700D51060116A49070BD5A5
:10BC5000B16BC90700D09760B16B890700D59360BD
:10BC6000B16B490700D59060116A09070CD51149DD
:10BC70000C68E40700D017610C68A40700D51361B5
:10BC80000968490700D51061116AC9060CD5094930
:10BC90008C68E40700D097618C68A40700D5936195
:10BCA0008968490700D59061F8BD0000400306404F
:10BCB000C002064000030640A82C002000000640F9
:10BCC000054900200A68002A02D1EFF3108072B6FD
:10BCD0000A68521C0A607047F82A002006490A6860
:10BCE000002A02D00A68521E0A600968002902D19F
:10BCF000002800D162B67047F82A002010B400294D
:10BD000009D0002A0AD0002B02D05C1E1C4208D0A9
:10BD100010BC0320704710BC0120704710BC0220EB
:10BD2000704701600021017241724260847210BC50
:10BD30000846704770B5002401250560062383710D
:10BD400005710379002BFCD1C72A01D0042300E040
:10BD50000123036003199A710A0C641C03199A7178
:10BD60000A0A641C03199A71641C02199171C16852
:10BD7000012252041143C160057101790029FCD1EF
:10BD800000F0CEFB002070BDF0B58FB000260D4650
:10BD90006B461E83090B1E82491C0391110B34460E
:10BDA000120500D00122891889B2099100F092F998
:10BDB000000B401C81B2C4482A057DD1099B039A1F
:10BDC000D2180A928A4277D80825039804AF2946E8
:10BDD0000090FEF7B7FA0A000A99009801D0801A7D
:10BDE0000830081A0830C008009B002A01D09B1AAE
:10BDF00008338B420ED8009B00219B1A5B199C468E
:10BE00006DE0002C6BD03B885B193B80401E491CC9
:10BE10000028F6D16846008A002873D003980027CE
:10BE2000201A08901DD00399A848C9190A03A849E7
:10BE300005465118059100F04DF9059988420CD935
:10BE40006879FD21084068716879042108436871A8
:10BE5000202228460599FFF76DFF08987F1CB842FD
:10BE6000E1D80A986946001B0390098A0027884296
:10BE700024D0964D6946098A28466118C9190A03D3
:10BE800093495118029100F025F9029988420CD982
:10BE90006879FD2108406871687904210843687158
:10BEA000202228460299FFF745FF6946098A039830
:10BEB0007F1C401AB84200E0C9E0DBD86846008A1F
:10BEC0001025059006AF29462046FEF73BFA059857
:10BED0000B462218002936D0E01A103034E0002A30
:10BEE00001D0634600E0009B2C464C43E34201D165
:10BEF0002C468BE7002A02D0634601E002E0009B5B
:10BF00001C1983E70998002500287DD96F4CFD276F
:10BF10000399204649190A036D49561800F0DAF8CA
:10BF2000B0420BD9607938406071607904210843D0
:10BF30006071202231462046FFF7FCFE09986D1CF7
:10BF40008542E5D382E02046101A10300109002B0B
:10BF500002D0E01A103000E0204690420DD80022B6
:10BF6000E01A4019844676E0002E74D038884019D3
:10BF70003880491E521C0029F6D16846008B0028E3
:10BF80007BD0200719D05148514922030546571844
:10BF900000F0A0F8B84210D90720000387420CD364
:10BFA0006879FD2108406871687904210843687147
:10BFB000522239462846FFF7BDFE6846008A2018FF
:10BFC00000071CD06946098B404871180A03404994
:10BFD0000446551800F07EF8A84210D90720000347
:10BFE00085420CD36179FD200140617161790420A3
:10BFF00001436171522229462046FFF79BFE6846A5
:10C00000008B0025002800E020E01FD92F4C71197B
:10C010000A032F492046571800F05CF8B84210D99F
:10C020000F20000387420CD36179FD20014061712C
:10C030006079042108436071D82239462046FFF711
:10C0400079FE6846008B10358542E0D300200FB0A2
:10C05000F0BD00E011E0002B01D0604600E020467A
:10C060002E465643F04201D12E4682E7002B01D0E6
:10C07000604600E0204686197BE76846008A002675
:10C080000028E3D9114DA1190A0311492846571870
:10C0900000F020F8B84210D90720000387420CD3E3
:10C0A0006879FD2108406871687904210843687146
:10C0B000522239462846FFF73DFE6846008A083678
:10C0C0008642E0D3C2E70000FFFFFFFF000005400B
:10C0D00000F0FFFF124A01239178002919D111497C
:10C0E00001609F218171037101790029FCD10E4803
:10C0F0000178117041785170807890700B48007809
:10C10000C006C00E022804D11078C42801D1122024
:10C1100090709078834001200003181A7047000047
:10C12000942C002001030000000405402525002078
:10C130000E4901609F21817101210171017900295E
:10C14000FCD10B490A780B4802704A784270897812
:10C15000817009490978C906C90E022904D10178FC
:10C16000C42901D112218170704700000103000031
:10C1700000040540942C00202525002010B50A4914
:10C1800001604B2181710021C17101724172817284
:10C190000121017101790029FCD1102203490448D1
:10C1A000FEF777F910BD00000510000000040540FF
:10C1B000972C002060300249407D087070470000D5
:10C1C00025250020F8B5044601252D030698A9422F
:10C1D00002D20E18AE4202D90020C043F8BD6579E4
:10C1E000022635436571667904252E4366710090F9
:10C1F000204600F017F86079FD21084060716079F1
:10C20000284360710020F8BDF8B54579069CFD26ED
:10C21000354045714579042635434571009400F059
:10C2200001F8F8BDFFB581B015460F460C460A9ED1
:10C230000198FFF74FFF874202D2B919814203D913
:10C240000020C04305B0F0BDFF2E2AD901980B2D68
:10C2500050D06B2D4ED0BB2D4CD03B2D4AD0EB2D6A
:10C260004AD0042101221204891801608571210C31
:10C27000C171210A01724472FF218172C1720121D0
:10C28000017101790029FCD104981E49E21B1018A4
:10C290008A15FEF7FEF8FF34FF3E0134013EFF2E03
:10C2A000D4D8002E23D001980B2D27D06B2D25D06C
:10C2B000BB2D23D03B2D21D0EB2D21D004213202E8
:10C2C0000A4302608571210CC171210A0172447216
:10C2D000FF218172C1720121017101790029FCD114
:10C2E0000498E21B101807493246FEF7D2F80020E6
:10C2F00005B0F0BD0521B5E70721B3E70521DEE76D
:10C300000721DCE700040540224A917800291AD170
:10C31000214901609F218171012101710179002969
:10C32000FCD11E480178117041785170807890706E
:10C330001B480078C006C00E022804D11078C4281B
:10C3400001D11220907092781648C721113A052A1F
:10C350001CD213007B441B79DB189F4402060B0F91
:10C36000130042790A40283202E042790A40203222
:10C370004271704742790A401832F9E742790A401F
:10C380001032F5E742790A400832F1E742790A4073
:10C39000EEE70000942C002001030000000405409B
:10C3A0002525002000000540F7B50446FF20A071B8
:10C3B000E0712072607204222260E36810048343FB
:10C3C000E3600123237120790028FCD1002904D0E7
:10C3D000012907D002291ED099E0E068800880007A
:10C3E000E06094E0E06880088000401CE060029813
:10C3F00000287DD0BB20A071FF2006302060AF2038
:10C40000A072E068012189040843E060237120796B
:10C410000028FCD17BE03520FF2102312160A07192
:10C420000120207120790028FCD13C4F3B789807EF
:10C4300043D40520FF2102312160A0710122227125
:10C4400020790028FCD139781802014301204002EC
:10C450000143002022600623A37122712379002B5F
:10C46000FCD1012265790323FB26354065712360E9
:10C4700023189A71401C23189971090A401C20182E
:10C480008171E06851040843E0602271207900283E
:10C49000FCD1204600F044F8607904210843607123
:10C4A0003520FF2102312160A07101202071207907
:10C4B0000028FCD13B789807BBD5E0688008800055
:10C4C000801CE060E068012109040843E060052069
:10C4D00020607720A0714020A07201212171207975
:10C4E0000028FCD10298002811D0EB20A07100E0B8
:10C4F0000DE0FF2008302060AF20A072E06801222C
:10C5000092041043E060217120790028FCD1A069D9
:10C5100040084000A06103B0F0BD000000040540E9
:10C520004179C90703D04179490849004171C06880
:10C5300080031BD50E483B21FF2206320260817129
:10C540000021C171102202724172FF218172C172F9
:10C550000122027101790029FCD1064909780260A3
:10C5600004218171027101790029FCD1704700001A
:10C570000000054000040540F8B50446C8B2091A99
:10C580000091FF21851801318D4202D90020C0435E
:10C59000F8BD3B49FF27097885290AD0002181424F
:10C5A00043D38D4241D9374A1E788A1816705B1CD6
:10C5B0003EE0FF2A2DD8344E00993B252660A57118
:10C5C0000D0CE5710D0A25726172A772E7720121E7
:10C5D000217121790029FCD1002A14D0D107C90F7B
:10C5E00004D0284D1E7845192E705B1C91420AD24A
:10C5F000244F45181E78ED192E705E786E70891CD8
:10C600009B1C9142F5D3812220480099FFF792FBB1
:10C6100011E01C4A00201D7881180D705D784D7066
:10C62000801C9B1CFF28F6D905E0164A8A18177053
:10C63000491CFF29B3D9012121600620A071217175
:10C6400020790028FCD104202060607908436071C3
:10C650000220A0710098000CE0710098000A20727E
:10C6600000986072E068012252041043E06021717A
:10C6700020790028FCD12046FFF752FF0020F8BDAA
:10C68000942C002000040540050001000000054036
:10C69000F0B5447985B0FD252C40447144790425DA
:10C6A0002C43447100900C46C8B2A9010E1A0392A3
:10C6B0009E4200D91E46201AE5180290E8B2B34205
:10C6C00001D9014600E000212F1A01910098FFF7DF
:10C6D00001FD844201D2854203D90020C04305B048
:10C6E000F0BD0298874203D9381A050A6D1E00E092
:10C6F0000025039F32463B4621460098FFF73CFF4A
:10C70000A419BE196D1E0DD3FF27013733463A46D3
:10C7100021460098FFF730FFFF34FF360134013621
:10C720006D1EF3D20198002805D0024633462146FB
:10C730000098FFF721FF002005B0F0BD10B500F014
:10C7400001F810BD10B508220021024800F02EF8B3
:10C7500010BD00000000024010B500F001F810BD4F
:10C7600010B508220121024800F020F810BD000099
:10C770004000024010B500F001F810BD10B50822CD
:10C780000221024800F012F810BD000080000240B3
:10C7900010B500F001F810BD10B5022203210248C7
:10C7A00000F004F810BD0000C0000240F8B50024FD
:10C7B00016460546002A28D9CF000120296AA04044
:10C7C00001421FD0114B1968C90608D51A681021FB
:10C7D0008A431A6028621A680A431A6000E02862D5
:10C7E000E9690B4AA2401140AA69E1400240E240D7
:10C7F000100601433819820006488258002A01D0E9
:10C8000008469047641CB442D7D3F8BD800102406B
:10C8100001000100182D0020024841680822114340
:10C82000416070470000074010B50E49496949054D
:10C8300002D50124E40301E07D2424020246E1172D
:10C8400000232046FDF7D8FD7D22D2000023FDF70E
:10C85000A3FD0023DB4300221B1A8A4101D20020E2
:10C86000C04310BD0000044010B5024807F09CFA18
:10C8700010BD000000000740FFB507460446203702
:10C88000387A81B0002802D0022005B0F0BD002C1B
:10C8900027D00298002824D00398002821D01846D9
:10C8A000FFF7C2FF0546FFF7DFFF0646012038729B
:10C8B0000298A0610398A0830021E183E18B81426B
:10C8C00022D220684069400612D4681C0CD0FFF7C1
:10C8D000CBFF801BA84207D300203872032005B08D
:10C8E000F0BD012005B0F0BD206840694006ECD5E0
:10C8F000E08B2168A2691218401CE0831078086060
:10C90000E08BA18B8842DCD30020387205B0F0BDEB
:10C91000044612A00AF0B0F9164821680AF0ACF9F2
:10C92000154861680AF0A8F91448A1680AF0A4F94A
:10C930001348E1680AF0A0F9124821690AF09CF94D
:10C94000114861690AF098F91048A1690AF094F950
:10C950000F48E1690AF090F9FEE70000496E2048AF
:10C96000617264204661756C742048616E646C6508
:10C97000720D0A001CBB02002CBB02003CBB020073
:10C980004CBB02005CBB02006CBB02007CBB020023
:10C990008CBB0200C01C8108044889000268521840
:10C9A00002604268511A416070470000742B0020F9
:10C9B00030B40E4AC01C830811689B0054680846B6
:10C9C0008D0702D080088000001DC3185B1AA342A7
:10C9D00002D930BC00207047DB1C9B089B00C918A3
:10C9E0001160E11A516030BC70470000742B0020C8
:10C9F0000148406870470000742B0020014800681F
:10CA000070470000742B0020014A5160106070478D
:10CA1000742B002010B500F001F810BDF8B5012608
:10CA2000B607F06A5B4CC00629D50221304600F0FB
:10CA3000DFF80028F9D02068017A21291FD1C18BA5
:10CA4000828B491C9142C28B8169895C026802D148
:10CA5000FF31FF3102311161C18B491CC183C18B90
:10CA6000828B91420BD301680A6B4B4B1A400A63CD
:10CA7000036B002B03D0C28B81691020984720687C
:10CA80000068C16A490503D50121890200F086F8D2
:10CA900020680068C16A490602D5402100F07EF88E
:10CAA00020680068C16A49073AD5082100F0A0F85B
:10CAB000002830D003273F02226810680369D18C18
:10CAC000156A6D18491CD1842B702068017A2129C0
:10CAD0000FD1C28C818C8A420BD2C28C521C8A42EA
:10CAE00001680A6901D13A4302E0FF2301331A4386
:10CAF0000A61C18C828C914206D1C36A002B03D09B
:10CB0000C28C016A1020984720680821006800F054
:10CB10006FF80028D0D120680421006800F03EF8AA
:10CB200020680068C06A80050CD52068082100686C
:10CB300000F05EF80028F8D1206801210068490261
:10CB400000F02CF820680068C06A800620D52021FB
:10CB5000304600F023F820680221006800F048F811
:10CB60000028F8D02168087A002811D1CA8B88697A
:10CB7000805C3061C88B401CC883C88B8A8B904214
:10CB800006D30B6B002B03D0CA8B89691020984702
:10CB9000F8BD00002C250020EFFF0000134A1140D3
:10CBA000CA0700D0426C8A0700D5826C0A0700D5FC
:10CBB000C26C8A0600D5026D4A0600D5426D0A068F
:10CBC00000D5826DCA0500D5C26D8A0500D5026EFA
:10CBD0004A0500D5426E0A0500D5826E8A0401D549
:10CBE000A8221258C90500D5C06D7047FF2F00005C
:10CBF00081B002460092064A00201140009A70322D
:10CC0000009212680A4200D0012001B07047000073
:10CC1000FF0F7F0000220120800502600222002910
:10CC200004D0012902D0022903D005E08168114314
:10CC300001E0816891438160816801221143816034
:10CC40008168C907FCD102607047000030B54278A6
:10CC50000178120289188BB28278C11C980A83B0BD
:10CC60003F280BD0092852D204007C44247924198F
:10CC7000A7444D094D22272C4D4D5300184601F075
:10CC800097F903B030BD27481C46181802D0172862
:10CC90003DD108E04A7808781202801880B289787D
:10CCA00002F0E8FA06E0087849780902401880B2F4
:10CCB00004F02CFE21462CE0184600F037F803B0B3
:10CCC00030BD184600F0B0F803B030BD16481C4621
:10CCD000C3421CD17F226846027108784978090254
:10CCE000401885B20020009001A9284604F038FEC3
:10CCF0000146684601704570290A81700179C1704A
:10CD000004226946204600F0F7FE03B030BD194604
:10CD1000012000F01EFF03B030BD184600F0AAFA53
:10CD200003B030BDFAFBFFFFFBEBFFFF70B5374AE6
:10CD300005460026801A364C84B0954224D005DC86
:10CD4000344828180DD0022805D115E000241828F1
:10CD500025D0192841D02946012000F0FAFE04B060
:10CD600070BD0846FEF756FD6160206031462846DA
:10CD700000F0DFFE04B070BD00F02AFE3146284608
:10CD800000F0D7FE04B070BD0846FEF743FDE16039
:10CD9000A0603146284600F0CCFE04B070BD684665
:10CDA0000480087849780902401886B269463046FE
:10CDB00002F00AFC01460194684602940171467132
:10CDC000310A81710188C171090A0172052201A924
:10CDD000284600F091FE04B070BD4A78087812022F
:10CDE000801886B28878C9780902401881B2304626
:10CDF00006F05CF96946009408704E70300A88703D
:10CE00000322284600F078FE04B070BD630C0000D9
:10CE1000D8950020FFF3FFFF004870479C95002045
:10CE20000048704790950020F0B507463C48002523
:10CE30003818092683B00C4600280BD0012832D0C0
:10CE4000022845D0082850D03946012000F081FE44
:10CE500003B0F0BD6A4602A901A802F067FC257084
:10CE600069460979617069460988A170694609882F
:10CE7000601C090AE17069460979217169460989CE
:10CE80006171694609893246090A41716946098812
:10CE9000817169460988090AC1712146384600F046
:10CEA0002BFE03B0F0BD412200212046FDF7F4FD2A
:10CEB0002570651C06F0F0FE014640222846FDF76D
:10CEC000C1FD41222146384600F016FE03B0F0BDF8
:10CED0002570601C0022602309F090FE3246214636
:10CEE000384600F009FE03B0F0BD2570661C02F064
:10CEF00083FB0B06020A1A4330707270020C0D0499
:10CF00002A43B2700A02000E1043F0700B0A31710E
:10CF1000737107222146384600F0EEFD03B0F0BDE4
:10CF2000FFEFFFFF38B5184D6860184806F044FF62
:10CF3000174C3022207100211648FDF7ADFD154831
:10CF4000154A00214260C943016000218160C1602F
:10CF500000221F214261016169681346C97901837A
:10CF60000092217901220D4807F05AF800F05CF890
:10CF700000F01CF80A4802F0A1FA0A4801F040F853
:10CF8000094804F0FFFC38BD1C2B0020D5D8000058
:10CF9000D0950020D8950020FF1F0020F495002098
:10CFA00001DC00009DDB00008DD80000F8B5184CB6
:10CFB0006068002800D001206B23164A16490CF047
:10CFC00051FD6168154A0888CD79C01D104004469E
:10CFD0006843FFF7EDFC060001D0012000E00020CF
:10CFE0000F4F71230B4A39460CF03CFD2B4622466D
:10CFF00031460C48FEF782FE002807D00024C119F4
:10D000007423044A20460CF02DFDF8BD0124F6E7F8
:10D010001C2B002090D0000000000408FCFF000042
:10D02000000002089C950020F8B5184C60680028A4
:10D0300000D00120582316A21E490CF013FD616890
:10D040001D4A48888D79C01D104004466843FFF78B
:10D05000AFFC060001D0012000E00020174F5E2346
:10D060000BA239460CF0FEFC2B46224631461448F2
:10D07000FEF744FE002807D00024C119612304A252
:10D0800020460CF0EFFCF8BD0124F6E71C2B002035
:10D090002E2E5C2E2E5C737461636B5C636F6E74FA
:10D0A000726F6C6C65725C6C6863695F6D61696EF0
:10D0B0002E63000000000408FCFF000000000108CF
:10D0C0009095002070B50F4940280CD30246CD68DA
:10D0D0008C68403A01200021FDF7CBF904400D4057
:10D0E0002C430BD10CE0421E4D680C68012000213E
:10D0F000FDF7BFF904400D402C4301D0012070BD65
:10D10000002070BDD895002070B50B4B01225968E6
:10D11000520711400A000CD0421E012000215D6917
:10D120001C69FDF7A6F904400D402C4301D00120F5
:10D1300070BD002070BD0000D895002070B586B08D
:10D14000002100910191029103910491694601220D
:10D150000A7002794A7082798A70C288120ACA708B
:10D16000027A0A71427A4A71838A02691C06150A98
:10D1700025438A716C46E571150C1C0425436C46E9
:10D1800025721C02120E22436C4662721E0AA372A2
:10D19000E672027E2273028B120A6273827EA2738F
:10D1A000428B120ACA73027F0A74828B120A4A7473
:10D1B000807F8874132221463E2000F0E1FB06B0F8
:10D1C00070BD70B588B004460020009001900290B8
:10D1D00003900490059006906D460A2107902970EF
:10D1E00021796970A179A970E088010A6846C17047
:10D1F000217A0171617A4171A28A216981711006D7
:10D200000E0A06436846C6710E0C100406436846B3
:10D2100006721002090E014368464172130A8272B7
:10D22000C372284621460C3006221F31AD1DFDF782
:10D2300009FC21460C35062225312846FDF702FC63
:10D24000217E68460176208B1F22010A68464176BE
:10D25000A07E2872608B6946000A6872207FA872DF
:10D26000A08B000AE872A07F28733E2000F088FBA4
:10D2700008B070BD70B50646F9480025301888B072
:10D280000C4634287ED201007944097949188F442C
:10D29000192538794751858F99A3ACC2CCFDFCFB89
:10D2A000FAF9F8F7F6F5F4F3F2F1F0EFEEEDEC79C8
:10D2B00079EBEAE979797979797979797979E8E7AE
:10D2C000E6E5E4E32046FEF7A5FAE64A516110617F
:10D2D0002946304600F02DFC08B070BDE2482570AC
:10D2E000026821461278627002681288120AA270DF
:10D2F00000680422C079E070304600F0FDFB08B001
:10D3000070BD06F0C3FC02462570601C0B4609F098
:10D3100075FC09222146304600F0EEFB08B070BDD6
:10D320000621204603F0DAF80146304600F001FC01
:10D3300008B070BD61782078090241186846018202
:10D34000E178A07809024118684641822179017587
:10D3500061794175A179817504ABE41D06222146EE
:10D36000D81DFDF76FFBA17968464177E279827796
:10D37000807D05AB033300900193039202916846D0
:10D38000437D00E07FE2027D418A008A02F0FAFEDE
:10D390000146304600F0CDFB08B070BD257000217D
:10D3A000617002222146304600F0A6FB08B070BD35
:10D3B0002178601C02F0B6FE0146304600F0B9FB51
:10D3C00008B070BD2178601C03F0EEF801463046CD
:10D3D00000F0AFFB08B070BD207802F0B7FE014648
:10D3E000304600F0A6FB08B070BDA278617812024A
:10D3F00089182379E2781B02D21820786379A479FE
:10D4000089B292B2009403F0AFF80146304600F0C2
:10D4100090FB08B070BD6178207803F087F8014672
:10D42000304600F086FB08B070BD617820780902B4
:10D43000411868460180E178A078090241186846E1
:10D4400041802179017161798171A41D0294A179D2
:10D450004171E079217A1AE00AE2FFE1EEE1E3E1CD
:10D46000C5E1A2E190E178E157E149E13EE135E132
:10D4700025E110E1FAE0DDE0D0E0BAE0ADE099E0CE
:10D480008FE05EE053E048E03FE032E029E009024F
:10D49000411868468181A17A607A0902411868467C
:10D4A000C181217BE07A0902411868460182A17B93
:10D4B000607B0902411868464182217CE07B0902B9
:10D4C000411868468182A17C607C09024118684647
:10D4D000C18203A902F0F6FC314600F03AFB08B025
:10D4E00070BD02F017FD0146304600F022FB08B087
:10D4F00070BD2570651C02F021FD287002222146B6
:10D50000304600F0F9FA08B070BD02F084FC014624
:10D51000304600F00EFB08B070BD611C207802F0B0
:10D5200076FC0146304600F004FB08B070BD611C7B
:10D53000207802F0F3FD0146304600F0FAFA08B018
:10D5400070BD6178207809024018E278A178120253
:10D550008A1869460A806279217912028A18694616
:10D560004A80E279A17912028A1869468A80627A31
:10D57000217A12028A186946CA80E27AA17A1202D6
:10D580008A1869460A81627B217B12028A186946E1
:10D5900080B24A8102F044FC314600F0DAFA08B069
:10D5A00070BD204602F0CAFE0146304600F0C1FAC6
:10D5B00008B070BD617820780902401880B26070B0
:10D5C000020AA270E11C02F01BFD20700822214615
:10D5D000304600F091FA08B070BD617820780902F9
:10D5E000401880B202F06CFD314600F0B2FA08B08B
:10D5F00070BD002000900190029003906D46049051
:10D600002870214622461031681C02F087FC112246
:10D610002946304600F070FA08B070BD2570601CD5
:10D62000082106F0F9FF09222146304600F064FA8D
:10D6300008B070BD61782078A41C637A227A1B023E
:10D640000902D2184018234680B292B20A3321460A
:10D6500002F0BEFF314600F07CFA08B070BD000059
:10D66000FFDFFFFFD8950020202B00206178207875
:10D670000902401885B2A11C284602F07BFC00215B
:10D680000091694608704D70280A88700322304660
:10D6900000F032FAE1E7617820780902401884B29C
:10D6A000204602F04FFC00210091694608704C7042
:10D6B000200A88700322304600F01EFACDE725705C
:10D6C000651C06F0EDFA02460B46284609F096FA6C
:10D6D00009222146304600F00FFABEE72078FDF718
:10D6E000D3FC0021304600F024FAB6E720786178B8
:10D6F000A278FDF779FD0021304600F01AFAACE778
:10D70000FDF776FE002222706070000AA0702146AC
:10D710000322304600F0F0F99FE761782078090293
:10D72000401885B2E178A0780902401881B2627988
:10D7300020791202801882B2284602F067FD014665
:10D7400000200090684601704570290A817003220C
:10D750006946304600F0D0F97FE703A902A802F03D
:10D76000E3FB00210091684601910170018941703D
:10D77000090A81708189C170090A0171052269460F
:10D78000304600F0B9F968E761782078090240185E
:10D79000E278A1781202891880B289B202F07CFD89
:10D7A0002946304600F0C5F957E706AB05AA04A99B
:10D7B00003A802F04BFC0021009101916846029100
:10D7C000017081894170090A8170018AC170090A5A
:10D7D0000171818A4171090A8171018BC171090A44
:10D7E000017201460922304600F086F935E761787A
:10D7F00020780902401884B203AA02A9204602F048
:10D8000047FC01460020009001906846017044707A
:10D81000210A8170017AC170017B0171052269467C
:10D82000304600F069F918E720786178A27802F0B4
:10D8300061FD0146304600F07CF90EE76178207802
:10D8400009024018A178E2782379647980B20094C3
:10D8500002F0C0FD314600F07CF9FEE620786178E8
:10D86000A278FDF761FC0021304600F062F9F4E691
:10D8700020786178A278E378FDF726FD0021304614
:10D8800000F057F9E9E631460120E4E770B5104CA5
:10D89000657A207A854216D0A84214D0002C15D083
:10D8A000207AA17A0840616848432168401881784D
:10D8B000C91CFFF7CBF9002C02D0207A401C207243
:10D8C000207AA842EAD100F0A9F870BD0020EEE766
:10D8D0009095002070B50646002920D008780128D0
:10D8E0001DD1214C657A207A854216D0A84214D0E9
:10D8F000002C35D0207AA17A08406168484321681D
:10D9000040188178C91CFFF7A1F9002C02D0207AB9
:10D91000401C2072207AA842EAD100F07FF8F0077C
:10D920001DD0114C657A207A854216D0A84214D0B9
:10D93000002C17D0207AA17A0840616848432168FA
:10D9400040188178C91CFFF781F9002C02D0207A99
:10D95000401C2072207AA842EAD100F05FF870BD26
:10D960000020CEE70020ECE79095002010B503489A
:10D970000121007906F064FA10BD0000D095002066
:10D98000F7B50F4F1546F86B002816D0EE1CB0B255
:10D9900006F01EFD040010D0042020700099617074
:10D9A000A5702A46E01C0199FDF74CF8711EFA6B30
:10D9B000601C9047204606F031FD03B0F0BD00002A
:10D9C00090950020014AD163106470479095002023
:10D9D00010B50E480C4A00214260C9430160002185
:10D9E0008160C16000221F214261016108494968CC
:10D9F000C9790183074806F017FC0748417D017586
:10DA000004F07AF810BD0000FF1F0020D895002018
:10DA10001C2B0020F495002090950020F8B5324C86
:10DA2000607D217D0C34884254D00090814251D0D9
:10DA30002E4D002C1CD0207AA17A08406168484302
:10DA400021684218507811780002081881B2D07805
:10DA500093780002181883B2032000030E050840D3
:10DA60000121360D0903121D884203D1012102E074
:10DA70000022E7E7022128781F46074301D1022947
:10DA800014D0002801D0012918D000202870304679
:10DA900004F0AAFB3A281ED007281CD0002C02D084
:10DAA000217A491C217200280CD00FE00120287037
:10DAB000002C0BD0207A401C207207E00020287038
:10DAC0000221E4E70121304600F053F8217A009862
:10DAD0008142AED1F8BD064800780028FAD1042171
:10DAE000044806F0FDFAF8BD909500201C2B00209C
:10DAF000F8950020F4950020F8B50646D01C154690
:10DB00000F4680B206F064FC041E11D001210170A2
:10DB10006670310AA1702A463946E01CFCF792FF74
:10DB2000EA1C21460E20FFF72BFF204606F076FC6C
:10DB3000F8BD38B50023009301246B461C70587063
:10DB4000000A9870D970042269460E20FFF718FF6A
:10DB500038BD08B5002300936B461870012058703B
:10DB60009970080AD870042269460F20FFF708FF51
:10DB700008BD00B583B000220092019201236A46DD
:10DB800013705070000A9070D170080A107105224D
:10DB900069461320FFF7F4FE03B000BDFFB5174F31
:10DBA00081B0386C1D46002823D06E1DB0B206F03F
:10DBB0000FFC04001DD0022020700299601C022975
:10DBC00019D00122120301990905090D11430170B1
:10DBD000090A41708570290AC1702A46001D0399FF
:10DBE000FCF730FF711E3A6C601C9047204606F02F
:10DBF00015FC05B0F0BD01225203E4E7909500202A
:10DC000070B50446007884B012287DD201007944B2
:10DC1000097949188F44081E345764798B9AAEE30A
:10DC2000FEFDA2FCFBFAF9F80520FFF74BFA0028ED
:10DC30006AD000200090217968460170A179417076
:10DC4000E0880422010A68468170217AC170694621
:10DC50000520F5E00820FFF735FA00287ED00020E7
:10DC60000090217968460170A1794170E088042212
:10DC7000010A68468170217AC17069460820DFE098
:10DC80000C20FFF71FFA002868D0002000900190B8
:10DC9000217968460170A1794170E0880822010A63
:10DCA00068468170217AC170A17A01716089010A88
:10DCB00068464171217B8171A089010A6846C17162
:10DCC00069460C20BCE01020FFF7FCF9002845D085
:10DCD0002079002100916946087001221020AFE0F0
:10DCE0003020FFF7EFF9002838D00020009021798C
:10DCF00068460170A1794170E0880322010A6846F4
:10DD00008170694630209BE028E0E288218900206C
:10DD1000009001900123684603704270120A8270DD
:10DD2000C170090A017105226946132088E0572055
:10DD3000FFF7C8F9002811D000200090A08869469C
:10DD40000870000A48700222572079E00A20FFF785
:10DD5000DBF9002804D02046FFF733FA04B070BD89
:10DD60000120FFF7D1F90028F8D02046FFF7E6F9A7
:10DD700004B070BD0220FFF7C7F90028F8D08B4827
:10DD800040780028F4D0207A0C3006F021FB061EE3
:10DD9000EED00221017001217170A17AB170E17A97
:10DDA000F170351D214606220C312846FCF74AFE4B
:10DDB000207AA871ED1D227A28466168FCF742FEA0
:10DDC000207A617A40190170227A31463E200C3265
:10DDD000FFF7D6FD304606F021FB04B070BD0320EE
:10DDE000FFF792F90028F8D00020009001900290EF
:10DDF00003216846017021794170A1798170E08822
:10DE0000010A6846C17006E099E0B6E092E08FE052
:10DE10005EE039E018E0217A017120890A22010AC6
:10DE200068464171A17A81716089010A6846C171B1
:10DE3000217B0172A089010A6846417269463E2031
:10DE4000FFF79EFD04B070BD0420FFF75DF90028C8
:10DE5000F8D00020009001900290684604230370DF
:10DE600023794370A3798370E28801A8130A6A4674
:10DE7000D3700822A118FCF7E5FD0C2269463E206C
:10DE8000FFF77EFD04B070BD0520FFF73DF90028C7
:10DE9000F8D000200090019002900390684605227F
:10DEA000027022794270A188C01C0A0A69468A70F1
:10DEB0000822A11DFCF7C6FDA07B6946C872E08957
:10DEC0000D22000A08733E20FFF75AFD04B070BD12
:10DED0000720FFF719F90028F8D0002000900190E2
:10DEE000029068460722027022794270A1880A0ACD
:10DEF00069468A70A279CA70E1880A0A69460A717D
:10DF0000227A4A7121890A0A69468A71A27ACA71FB
:10DF100061890A0A69460A72227B4A72A1890B2228
:10DF2000090A817269463E20FFF72AFD04B070BDE0
:10DF3000082000E00920FFF7E7F804B070BD0C20CE
:10DF4000FFF7E2F80028F8D00020009001900C21A3
:10DF50006846017021794170A1798170E0880622BC
:10DF6000010A6846C170217A0171617A417169467E
:10DF70003E20FFF705FD04B070BD1420FFF7C4F884
:10DF80000028F8D000200090142168460170217903
:10DF90004170A0880422010A68468170A179C1708D
:10DFA00069463E20FFF7ECFC04B070BD509900209C
:10DFB00070B58205120F0F2A04D001460120FFF729
:10DFC000C8FD70BD0446002580060A46800E06D0B6
:10DFD00003280DD021460120FFF7BBFD70BD0621AF
:10DFE000104605F095F829462046FFF7A2FD70BDC2
:10DFF0000878FDF74BFB29462046FFF79AFD70BDD8
:10E0000001490861704700001099002070B50E4B5F
:10E01000DA889C88A24201D3072070BD012810D85D
:10E0200000290ED0D5001C68521C6419DA80A0713A
:10E030002046FDF7D5FB01212046FDF70DFB002012
:10E0400070BD122070BD0000B82B002070B50E46C8
:10E05000040001D0012000E00020FF23393313A287
:10E060001C490BF0FFFC8E20005D25466035012821
:10E070000FD0AC786C7025213046FCF763F9E87856
:10E080002522511A484300191146FCF771F9A9706D
:10E0900070BDA8786870218FE08C012201F008FB28
:10E0A00060872521FCF74EF9F1E700002E2E5C2E4B
:10E0B0002E5C737461636B5C636F6E74726F6C6CF7
:10E0C00065725C6C6C5F636F6E6E5F636F6D6D2EFF
:10E0D000630000000000060270B501290DD006465D
:10E0E0000025203675720446357006F081FAC104A9
:10E0F000B078C90C012803D003E005F075F970BDB4
:10E100000021104A206B504341182046FCF7CAFCFE
:10E11000B17A606B4843FCF7CBFC21684018606023
:10E120000020FCF7CBFC0120FCF7CEFC022004F021
:10E13000CDFA05480570757002F03CFF0020FCF731
:10E14000C9FC70BD710200002C2B002010B50A78AC
:10E1500082B01407240F6A4614700A789206D30F0F
:10E160006A4653700A785206D30F6A4693700A784B
:10E17000D3096A46D3704B78091D1371032C03D061
:10E18000052C01D1222B02D0002002B010BD0A467E
:10E19000694600F07BFB02B010BD7047F1B50098F6
:10E1A000002800D00120C72318A222490BF05AFCF6
:10E1B000009D2846643086460020024658350021DE
:10E1C0000426D3009C460123AC5C1F468F403C4292
:10E1D00005D067467F1874462754401CC0B2AC5C1B
:10E1E0004F1CBB401C4206D063465B1874465B1C48
:10E1F0002354401CC0B2891C761EE4D1521C052A4F
:10E20000DDDB009980314873F8BD00002E2E5C2EB6
:10E210002E5C737461636B5C636F6E74726F6C6C95
:10E2200065725C6C6C5F636F6E6E5F636F6D6D2E9D
:10E23000630000000000060270B5044660300578F7
:10E240001C480068002800D00120FF235F331A4AD1
:10E250001A490BF007FC01F025FA082D00D3072519
:10E26000174A6900515A62690818216885B200206E
:10E27000891A00290DDD0846FCF732FC7D26F600E0
:10E280003146FCF75FF80146284648433146FCF723
:10E2900059F84034218A0B4A5143FF22F53296390E
:10E2A000814200D210460849097B002900D046224D
:10E2B000101870BD282B00200CE2000000000502A1
:10E2C000A62B00207102000078950020F8B504000C
:10E2D00001D0012000E00020324B334A33490BF0DB
:10E2E000C1FB2546FF358135A87F697F884201D370
:10E2F000012000E000206923DB002B4A2C490BF0B1
:10E30000B1FBA87F697F0027401AC3B22046FF30C7
:10E31000A13006798278964207D14770C77087701E
:10E32000002B3CD00121A17739E0002B09D09A4283
:10E330000AD8238C5B07DF177F1C4770DB0FA3779E
:10E3400013E04770A77710E0278C931B7F0700D559
:10E350005B1C994201D2012700E0002747709942D7
:10E3600001D3012300E00023A377238C921B5B07DA
:10E3700003D5002901D0491E6977FF34C134697F74
:10E380002678914201D9134600E00B46F31823701A
:10E39000C378914200D91146511A5918C170C178F9
:10E3A0008170F8BD470300000CE200000000060287
:10E3B0006666FFFFF8B50446407E0D46002812D081
:10E3C000E889A18C401A012180B2C903884202D891
:10E3D000491E88420CD91D48694640680090204675
:10E3E00004F0C4FCF8BD0121204604F0E3FCF8BDB4
:10E3F000697A2B7A0A0E0E0200209B190146AE7A2A
:10E400005141320C36049E19EB7A51411A0A1B060F
:10E41000F31851412A7B1818514101F0EFFC0028F4
:10E420000ED00121A420015520469C30EA68A9683D
:10E4300042600160A220015B204600F025F8F8BD93
:10E440001E220121204604F0E9FAF8BDA0E30200F3
:10E4500010B505480021C180818800688A0100212B
:10E46000FCF71AFB002010BD6097002010B505488E
:10E470000021C18081880068CA000021FCF70CFBE4
:10E48000002010BDB82B0020F3B50446C38C81B02A
:10E49000808C02991A1A2546081A4035298A894E15
:10E4A000401E71432646FF36A136904229D2029F74
:10E4B000BB4226D0171A79432046FCF717FBE08CA5
:10E4C000B9B2C01BE0842046FFF7C0FD2046FFF72D
:10E4D000B3FE7D49C83009684A8B898B51180818EA
:10E4E000FCF7E6FAA06021680B1A7849CA68402058
:10E4F0008243CA608B61CA68012382431043C860AB
:10E500007371E18C029881427DD127468037F87B78
:10E51000002820D0A98A0A2041433846DC3005F083
:10E52000DFFD288AB98A884203D02146002002F004
:10E53000C3FD0020F873387CA881788AE881B88A06
:10E540002882F88A6882388BA882207F40084000A1
:10E550002077012070712146A031087900281FD052
:10E56000002008717D7F3B7F2A0E2D025D19BB7F45
:10E5700050411A0C1B04EB18FD7F50412A0A2D064E
:10E580005B1950410A78191C5041A165E06520468D
:10E59000FFF704FE207FFD210840207701207071E5
:10E5A0002746FF378137B87D00282CD0BD7C68070F
:10E5B00000D50325F87E03214903A84205D0226A2D
:10E5C00001238A435B03D21822620022BA7538778E
:10E5D000FD76207FFB22104020770122206AD202A4
:10E5E000904342042062920F10D088432062384842
:10E5F000FF210068D131201AFBF7BAFE81B22B4609
:10E600001A46002000E05AE002F0FCFDF87E2546A4
:10E61000C035032803D0387F032827D04DE03A7F48
:10E6200069682868032A07D0A9221201130480B25E
:10E63000184389B2120411436B88020C9A4203D129
:10E64000EB880A0C9A4238D0696028602048FF2184
:10E650000068D131201AFBF78BFE6988009180B2E7
:10E660002B88EA88A98802F047FD26E02988A88837
:10E670000A04520B703292B289B213041943030494
:10E680005B0B70339BB280B21F0438436F88BA4271
:10E6900002D1EA88934210D0296068600C48FF21BB
:10E6A0000068D131201AFBF763FE6988009180B2BF
:10E6B0002B88EA88A98802F01FFD0120707103B041
:10E6C000F0BD0000E2040000282B002000000250F2
:10E6D000242B0020F8B50446407F002822D1E07E9C
:10E6E00001261F4F1F4D002821D00020E0766677BD
:10E6F000607E012817D02A68002A02D00021204617
:10E70000904719488069002802D0204602F0ACFCEE
:10E710003868FF21201AD131FBF72AFE80B2002190
:10E72000FCF7EAF9F8BD6A68002AE7D1E9E738683A
:10E73000FF21201AD131FBF71BFE80B20121FCF72B
:10E74000DBF9E676607E012806D02A68002AE9D047
:10E75000012120469047F8BD6A68002AF8D1F8BD2B
:10E76000242B0020089600201099002070B504008A
:10E7700001D0012000E00020364B37A240490BF0C9
:10E7800071F92046FFF7A2FD0020FCF797F9012060
:10E79000FCF79AF9A08E0025E16800283AD0A586FA
:10E7A00020686061607E012828D1A06A002825D0F9
:10E7B00034480068818B408B0818FCF779F9A16810
:10E7C00022680B1AA16A0126881AB607B04200D93E
:10E7D000501A984205D3E08C012802D9208C0006FB
:10E7E00013D5FF209C30005D274940004018403879
:10E7F000C08FFCF75DF9A16A081A2060E08E02283C
:10E8000006D380B2801EE08619E00420E086F8E797
:10E81000E58614E0E08E062801D2401CE08680B236
:10E82000401E012804D8487D062801D2401C4875A6
:10E83000E08E062803D30120400203F047FFA562C3
:10E84000206A80218843206201212046FCF75AF982
:10E8500070BD0000E30400002E2E5C2E2E5C73744D
:10E8600061636B5C636F6E74726F6C6C65725C6C11
:10E870006C5F636F6E6E5F636F6D6D2E6300000083
:10E8800000000602282B0020A02B0020F0B5064631
:10E89000F5480D4681799DB0F4480068007C8142BE
:10E8A0007ED253781178180E1B0294781943230CEA
:10E8B00024042143D4781843230A184313792406E7
:10E8C0001843537921431B0218430091019019907A
:10E8D000D4798C469179200E2402177A21433C0C7E
:10E8E00020433F04547A3943270A2406931D2143C9
:10E8F000947A5B79384320431B02184302910390BA
:10E9000016911790517B107B09024018917BD37BA5
:10E9100009041B06C91840180490507C917C000221
:10E9200009044018117C40180590D17C08A8817119
:10E93000517D107D0902411868460185D17D907D89
:10E940000902411868460184517E107E090241186F
:10E9500068464184D17E907E0902411868468184D0
:10E96000547F137F210E24021C321B19002094783F
:10E970004841210C24041B19D4784841210A24065B
:10E980001B1948411479191C604106910790507970
:10E99000C106C90E08A881725079410908A800E093
:10E9A00096E0C17200200E900F900C900D90B76809
:10E9B0003C4620342279D00703D0AB498868C96827
:10E9C00002E0AB49886AC96AD207E378D20F062B06
:10E9D0007ED0022B7CD0EB78934279D1169A179B8C
:10E9E00042404B401A4373D1A8781490604619995D
:10E9F0001191109010AA0120149901F0CBF9002870
:10EA000066D1E07801280CD15020C15D1498814274
:10EA10005ED1B96CF86C109A119B5140584001437B
:10EA20007ED16846018D008C814279D808A9897908
:10EA3000002975D0421E082A00DD082291426FDCB1
:10EA40008C4A811F91426BD26946898C8A4B0A4657
:10EA50000A3A9A4264D26A46528CFF23F4339A42AD
:10EA60005ED8864B521C5A4350439A005143814210
:10EA700056D900207C496072087020702879C00047
:10EA80002830FCF715F8396C47180120FCF740F8DE
:10EA9000044600F0C7FE0420B46030750020F07515
:10EAA000022070756846E660149001206076A978AF
:10EAB0003D200155204606223E301499FBF7C2FF47
:10EAC000049860640598A06408A88179204600E055
:10EAD00026E04030169081816946098DC1816946E2
:10EAE000098C01826946498C41826946898C818200
:10EAF00007990698E165A06508A8C17A20466030AC
:10EB0000017008A9897AC1702046FFF747FB2046AB
:10EB100080300021179081736878012803D00CE0C1
:10EB200000201DB0F0BD5648007B012805D1179983
:10EB30008873606C010C41402187204603F02AFB5A
:10EB400016985049C089401C4843FBF7B1FFC019D3
:10EB5000206019204001FBF7ABFFA0601698818A66
:10EB60000A2041432046FF305D3005F0B9FA2646C1
:10EB7000C036B1882046FBF7D1FFF788B84204D2EF
:10EB8000B1882046FBF7CAFF074631882046FBF7CD
:10EB9000C5FF01467088814203D231882046FBF7C9
:10EBA000BDFF3A18169837498089FF32484349100B
:10EBB00041182E482D320068007E5043884200D80C
:10EBC0000846FBF775FF2168401860602046FF305B
:10EBD000B93001D0417A0172302005F0C1FB2A4FD3
:10EBE00006002FD007203070002030713868FF21D8
:10EBF000201AD131FBF7BCFBF080607E3072A87820
:10EC0000707201990098716130616846008C3083A0
:10EC10006846408C70836846808CB08308A8C07AB0
:10EC2000B0771499304606221F303831FBF70AFFBF
:10EC300014993046062225303031FBF703FF304669
:10EC400003F0E2FE3868FF21201AD131FBF790FB78
:10EC5000179980B2897B02F0CAF903488179491C6F
:10EC6000817101201DB0F0BD50990020282B00209B
:10EC7000109900207B0C0000770C0000C4090000F4
:10EC800008970020E2040000242B002010B500F0BB
:10EC9000F3FE04F0DFFF054800210160416001211F
:10ECA00001720349062006F045FE10BD08960020BB
:10ECB000D5E6000038B5427E002A11D04A8A838CFE
:10ECC000D21A012392B2DB039A4202D85B1E9A4207
:10ECD0000AD91C4909680091694604F047F838BD13
:10ECE000002104F067F838BD4B898A89934224D803
:10ECF0000B7A002B21D0541E082C00DD0824A342DF
:10ED00001BDC114B921F9A4217D20A8A1B1F0A3A28
:10ED10009A4212D2CA89FF23F4339A420DD802468E
:10ED2000CD688C6880320969556114610123916155
:10ED3000D373518BFFF7A8FB38BD1E22002103F0CF
:10ED40006DFE38BDA0E302007B0C0000F0B5054667
:10ED5000B8228889525B08318FB0904201D20646B2
:10ED600000E016461B2E01D21B2002E0904200D389
:10ED70001046260C36040A90384C0643088824684E
:10ED80000C94647CA04201D2074600E027461B2F6A
:10ED900001D21B2002E0A04200D320461B0C1B0422
:10EDA00003430890D0009E467030FF2783B29C3703
:10EDB000E0007F5D7030032F06D13D2093010001FC
:10EDC0001B18A4019BB22018CC889C4200D91C4679
:10EDD000B6B227043E4300964988A446814200D932
:10EDE000014674460E04A4B23443A6460B912C4649
:10EDF000C03427880A990126B9420BD1A7880899FF
:10EE0000B94207D161888C4504D1E1880B9F8F42BC
:10EE100000D10026774600996760216069460A8222
:10EE20000C994A7C69468A824B82C88204A928468A
:10EE300003F076FB002E0ED00948FF210068D13187
:10EE4000281AFBF795FA6188009180B22388E2883E
:10EE5000A18802F051F90FB0F0BD0000282B00206E
:10EE6000242B0020F0B50446012083B00246009018
:10EE700008892346FF33054681331B3D0831019342
:10EE8000E12D25D28B881B2B22D3FB2B20D8CD88BC
:10EE9000FF264936B5421BD3494B4A4FEB18BB42BC
:10EEA00016D3494B9D4213D84B88B34210D3444EDE
:10EEB0009E19BE420CD3444EB34209D8019EF67E41
:10EEC000032E07D1A9263601B34201D3B54201D2A0
:10EED000002200922546C0356F682E68002A44D073
:10EEE000224680328B889646128F9C46934201D2EE
:10EEF000634600E013461B2B01D21B2304E094451C
:10EF000001D2634600E01346360C36041E437346B6
:10EF10009B8FB446984201D2064600E01E461B2E47
:10EF200001D21B2002E0984200D318463F0C3F0458
:10EF3000019B07437046DB7E408F032B04D1900179
:10EF40003D221201801880B2CA88824200D8104641
:10EF5000624696B2000406437046C08F49888842D4
:10EF600000D30846BFB2000407432988B0B28842E4
:10EF70000DD1A988B8B2884209D16988300C88427D
:10EF800005D1E988380C884201D1002000906F60DB
:10EF900020462E6001F0EFFB009800280ED00B48B1
:10EFA000FF210068D131201AFBF7E2F9698800914E
:10EFB00080B22B88EA88A98802F09EF803B0F0BDE1
:10EFC000B7F7FFFF4702000090420000242B00200B
:10EFD000F8B50A4605460978854C501C61711A2916
:10EFE00079D2844B8A009A58002A74D0192972D297
:10EFF0000A007A441279921897440C29369CB9D9A0
:10F00000D9364D4DD9D93ADE48F5F5E29797536E8A
:10F01000737F8600764902780A72837842781B02F1
:10F02000D2184A810379C2781B02D2188A81837967
:10F0300042791B02D218CA81037AC2791B02D21804
:10F040000A82427A807A000210184882A4E06A4E4E
:10F050000746014605223046FBF7F4FCB97978797A
:10F0600009024018F08094E061490078087293E04A
:10F070005F4902780A72837842781B02D2184A816B
:10F08000C278007900021018888185E05B48008C06
:10F09000000720D580E0564EFCF7BCFBF160B06065
:10F0A00077E0564A128C920615D54378027850497B
:10F0B0001B02D2180A81C37882781B02D2184A81B7
:10F0C000437902791B02D2188A818279C0790002C1
:10F0D0001018C88160E072E0484A128C92066ED522
:10F0E000E3E7464A0923126A1B021A427BD04049D1
:10F0F00002780A72407848724EE0404A0923126A48
:10F100001B021A426FD0F2E73C4A0923126A1B0223
:10F110001A4268D0364902780A7242784A72827876
:10F12000C07800021018488136E03448008CC006D0
:10F1300059D531E0314A128CD20754D02E4E0746B1
:10F14000014608223046FBF77DFC797A387A0902BD
:10F15000401830810A373046082239460A30FBF71A
:10F1600071FC394608310422304612300FE0234A40
:10F17000128CD20737D0204E07460146082230466F
:10F18000FBF760FC39463046083104220830FBF7B3
:10F1900059FC60791A2805D26079194A2179125CE4
:10F1A000914217D0C1B2284603F004FEF8BD1348BF
:10F1B000008CC00717D0EFE70D4900789BE712E0FD
:10F1C0000E4A128C52070ED5094902780A7240780D
:10F1D0004872E1E7810007484258002AE6D0044916
:10F1E00028469047F8BD284603F0E4FDF8BD00002E
:10F1F00040970020ACE302004897002010990020BF
:10F2000014E4020070B50446407E1849002802D07C
:10F21000012807D00CE04879002809D04879401E21
:10F22000487105E08879002802D08879401E8871ED
:10F230002646FF368136F079B579002802D1132DA4
:10F2400000D116250A48FF210068D131201AFBF7AA
:10F250008FF880B2294601F067FF2046FF305D300D
:10F2600004F0E2FF0020F06070BD00005099002023
:10F27000242B0020FF22D132504308B50E4A1268D9
:10F2800080180AD0027E002A07D00246FF3281325F
:10F29000D379002B03D0132008BD022008BDD2680B
:10F2A000002A01D0002008BD6A461170694603F0AB
:10F2B0005DFD002008BD0000242B0020F0B50446B1
:10F2C000407E89B000287BD020460831E4300F46CC
:10F2D00008220646FBF7B6FB25463889C035688408
:10F2E0003946284608220A314C30FBF7ABFB28464A
:10F2F00039465C30042212310290FBF7A3FB08214F
:10F3000004A805F089F906A80421074605F084F948
:10F3100004A9204603F06DF920460121E030017078
:10F320004170082204A93430FBF78CFB284639468B
:10F33000603004220746FBF785FB28460D2200219A
:10F340007030FBF7A9FB2846082275300299FBF7BD
:10F3500079FB607E012839D0802038752046FF3047
:10F360000D2200214D30FBF797FB2046FF3008228D
:10F3700052300299FBF766FB607E012828D00021FD
:10F38000FF20513001551348FF210068D131201A68
:10F39000FAF7EEFF87B26D8C102004F0E1FF040055
:10F3A0000BD00B202070A78008223146A01DFBF750
:10F3B00049FBE581204603F027FB09B0F0BDFFE7DC
:10F3C0000321204603F0F6FC09B0F0BD0020C4E79D
:10F3D0008021D5E7242B002070B50446407E88B0FC
:10F3E000012861D020460831FF300D460822153033
:10F3F000FBF728FB20462946FF3021300422083144
:10F400000546FBF71FFB002000900190029003903F
:10F4100004900590069007902046FF301022694620
:10F420000D3008F099FF2046102204A9EC3008F0B6
:10F4300093FF204604AA6946FC30FBF7AFFC204648
:10F44000FF300D2200213130FBF726FB2146FF3132
:10F450001D31084608220E461930FBF7F3FA607E8C
:10F46000012827D0802028752046FF300D2200215A
:10F470004D30FBF711FB2046FF3008223146523059
:10F48000FBF7E0FA607E012816D00021FF20513002
:10F4900001550121E1200155204604F031FA2046B2
:10F4A00001F058F908B070BD0421204603F082FC39
:10F4B00008B070BD0020D6E78021E7E70149C860A9
:10F4C000704700001099002030B5427E83B0002ABA
:10F4D00015D00D4A0D7A116A546A0A462A4005462B
:10F4E000002380356B63090A2A6309020A43234318
:10F4F00069460193009203F0D0F803B030BD49791A
:10F5000003F058FC03B030BD1099002030B504461C
:10F5100016480B7A006A83B01840234600228033D5
:10F520005A6318632033DD79002D19D0DA718B68A6
:10F53000C9681B0A1B02034311430D480191009344
:10F540000068FF21201AD131FAF712FF81B26A4612
:10F55000002001F06AFE204601F00DF903B030BD35
:10F560004979204603F026FC03B030BD10990020F5
:10F57000242B0020F8B50446002503216846009599
:10F5800005F04AF8684680782E028106890E6846A2
:10F5900040318170427803782804000E360E000452
:10F5A000360230432D0E12020904284351182070F0
:10F5B000020A6270000CC918A070E170080A20717C
:10F5C000080C6071F8BD000010B50C46FF21D13168
:10F5D00048430849096840180AD0017E002907D02D
:10F5E0008030C06D0A21FAF7ADFE2080002010BDEA
:10F5F000022010BD242B00200149886AC96A704787
:10F6000010990020FF308130C07E012804D00228EC
:10F6100002D0032801D0002070470420704700006A
:10F62000F0B40546C035EC881D4E2B466103C0334F
:10F630008919DA7E090C0127521E9740FAB2477EDB
:10F64000002F04D0077F7F0706D5DA7D08E0008C05
:10F65000000505D59A7C03E0008CC00400D5DA7C57
:10F66000900703D5A0038019010C13E0500711D5B2
:10F67000987E1B21012802D0022806D00AE0FF3C18
:10F680007F3C2011093881B204E0FF3C913CA0117D
:10F69000093881B2A888884200D30846F0BC704778
:10F6A0000000F2FF01488088704700002C2B0020EA
:10F6B000F8B50C46604007461646C0B2FCF794F811
:10F6C0000546380AFCF790F801022943080108189A
:10F6D000001987B2F8B2FCF787F80546380AFCF73C
:10F6E00083F80102294308010818001987B2F8B20B
:10F6F000FCF77AF80546380AFCF776F80102294348
:10F7000008010818001980B2002E00D06040F8BD32
:10F7100005490120096ACA0500D50320090501D55C
:10F7200004210843704700001099002010B4064BD4
:10F730001C682478047018684088088018688088DD
:10F74000108010BC70470000282B00200148007971
:10F7500070470000B82B002070B5040001D00120D4
:10F7600000E00020284EF0231EA231460AF07AF96C
:10F77000264D002C2C6001D0012000E00020D92370
:10F78000234A31460AF06EF92868417C1B39E12989
:10F7900004D2007E002801D0012000E00020F523E3
:10F7A00010A21C490AF05EF91B49002008701B4892
:10F7B00004F002FB1A490876FBF792FB00F07EFF8B
:10F7C0002868407EFBF728FE05F048FF04F036FA73
:10F7D00003F0A8FD01F0DCFB01F0A8FBFFF756FAEF
:10F7E00070BD00002E2E5C2E2E5C737461636B5C0A
:10F7F000636F6E74726F6C6C65725C6C6C5F696E5B
:10F8000069742E630000000000000A02282B00200B
:10F810002807010000000F022C2B00209D0701008B
:10F8200030990020F0B5044683B0012060760025B1
:10F83000A576E5762577A5776077E5772020E560E2
:10F840002062A584E584656125602561A560A562C7
:10F85000E5622563A586E58656200553204660307F
:10F8600045708570658725872030009085735F48D7
:10F8700027460290FF37007E613738736620B870E4
:10F880005B48FF210068D131201AFAF771FD01466B
:10F8900038462038019081841C3004F0C5FC029861
:10F8A0003E46007E203630706720B8755048FF21F4
:10F8B0000068D131201AFAF75BFD014601980187F3
:10F8C0003046B580103804F0AFFC00982246C5736E
:10F8D0002046A030057145718571C57100208032C8
:10F8E0001063506343480168487CFB2800D3FB2029
:10F8F000009A1087C000009A70305087487CFB281F
:10F9000000D3FB20009927468887C00000997030FB
:10F91000C8871B20C037FF21388049317980B880E3
:10F920003548F98081797176C179F175007A307640
:10F930000120F0763077B076B5750298FF21007E11
:10F9400038766B20B8732A48D1310068201AFAF74C
:10F950000FFD388200982949C1652046C83004F05F
:10F9600063FC2046E030457005700198FF21457624
:10F9700001980D2285760198C1762146FC310F1D34
:10F9800000917962FF2104202D310855384630302E
:10F990000021B862FBF780F80099396401990420CE
:10F9A000087238464C300D2200217864FBF774F859
:10F9B000B571F5711248F560B0603846C0304178D5
:10F9C0000170B562F562356375637577B577FF349D
:10F9D000F577A13425706570A570E57025716571A6
:10F9E00085720572457203B0F0BD000030990020A9
:10F9F000242B0020282B00200099002030750000C7
:10FA000020A10700104A1268D37B127C9B1801D1F9
:10FA10000020704710B50246840702D08208920089
:10FA2000121D0A4C2260FF24D13463439A18141A21
:10FA30008C4207D90648611A0143A22305A200207F
:10FA40000AF010F8204610BD282B0020242B00209F
:10FA5000000003022E2E5C2E2E5C737461636B5CBF
:10FA6000636F6E74726F6C6C65725C6C6C5F636FED
:10FA70006E6E2E6300000000F8B5FCF7BFFF07466E
:10FA8000FCF7B6FF574D01462868574EC27B007CF5
:10FA9000101816D03C46BA0702D0BC08A400241D9A
:10FAA000FF22D132504300193460C41B8C4207D965
:10FAB0004E48611A0143A2234D4A002009F0D2FFAB
:10FAC0002046FCF767FF2868417C877C0E31890857
:10FAD00089001331CC08E40020467843FBF744FD4D
:10FAE0000090002800D00120DC2342A24A4909F0FE
:10FAF000B9FF3B46224649480099FCF7FFF8002829
:10FB000043D000244449DF2341183AA2204609F09B
:10FB1000A9FF28680024C17B007C081800284CDD60
:10FB200030480068417CC67C0E31890889000B3161
:10FB3000CD08ED0028467043FBF716FD0090002825
:10FB400000D00120EE232BA2354909F08BFFFF20C6
:10FB5000D130274647432448334600682A463818A0
:10FB6000FF30B9300099FCF7C9F801000FD0002030
:10FB70002B4DF1231FA2491909F074FF6814FCF7FB
:10FB800017FF060005D0012004E00124BAE7012098
:10FB9000EEE70020F52317A2294609F063FF12487B
:10FBA000641C00683818FF30813046640D480068D6
:10FBB000C17B007C0818A042B2DC1820FBF7D4FC03
:10FBC000040001D0012000E00020FF23013309A23E
:10FBD000144909F047FF012020710020607112488C
:10FBE0000460F8BD282B0020242B00200000030215
:10FBF00054FA00002E2E5C2E2E5C737461636B5CD5
:10FC0000636F6E74726F6C6C65725C6C6C5F636F4B
:10FC10006E6E2E63000000000000020210990020AA
:10FC200000000102AA0001029C2B0020F8B5082662
:10FC30004027B001FBF798FC040001D0012000E050
:10FC400000208325AD0464231BA2294609F00AFF86
:10FC500033463A4621462148FCF750F8002820D088
:10FC600000244119672314A2204609F0FBFEFF205F
:10FC70000130FBF779FC002800D001206A230EA296
:10FC8000174909F0EFFE174D1448002168614172D1
:10FC9000686901722020FBF767FC040003D0012093
:10FCA00002E00124DDE70020722303A20E4909F0DF
:10FCB000D9FEAC61F8BD00002E2E5C2E2E5C737454
:10FCC00061636B5C636F6E74726F6C6C65725C6C9D
:10FCD0006C5F7363616E2E630000000070970020FC
:10FCE000FF000C0280970020EE000C0270B51A4D48
:10FCF0002868002800D001203B2318A2214909F0E0
:10FD0000B1FE28688079002824D0C000FBF710FCE1
:10FD1000040005D14121452310A2C90409F0A2FE27
:10FD2000286800218079C2002046FAF7B5FE1648FF
:10FD3000164A04602968897981800021C18011698F
:10FD40007F20C0008143124BE000C0188005800D69
:10FD50000843106170BD0000282B00202E2E5C2E61
:10FD60002E5C737461636B5C636F6E74726F6C6C2A
:10FD700065725C6C6C5F77686974656C6973742E0E
:10FD80006300000000000A02B82B00204008025067
:10FD90000000EC7FF7B50E461349002409680128DE
:10FDA000CD7B02D1087C2C462D18AC4216DA0F4FC1
:10FDB000FF20D130396860434018017E00290AD005
:10FDC0003D21095CB14206D106223E300299FAF784
:10FDD000ABFE002805D0641CAC42E9DB002003B078
:10FDE000F0BD012003B0F0BD282B0020242B002003
:10FDF0000148007970470000342B002010B504F052
:10FE000065FA022801D3012010BD002010BD10B5F5
:10FE1000FEF7FCF810BD10B5FEF728FB002010BD62
:10FE2000FF2230B5D1325043244A83B01268801883
:10FE300009D0027E002A06D0427E012A03D0002A81
:10FE400004D0012303E0022003B030BD00236A4642
:10FE50005380032313704B8893808B88D380CB8887
:10FE600013810246FF32C1325378127889889A1A78
:10FE7000D3B2134A1268D47B127CA21806246243C0
:10FE80009A18C38C591851186A46891D5181016A04
:10FE9000402211430162014601228031CA73029D52
:10FEA000019C009B8D614C610B61017F11430177C7
:10FEB000694602F0B6FA002003B030BD242B0020C2
:10FEC000282B002070B50D46044603F029FF0028BA
:10FED0000AD06079C00703D00D48C079002810D03F
:10FEE0002079002802D00EE00C2070BDA268002A04
:10FEF00007D0A1790020FFF74DFF002803D00B2089
:10FF000070BD122070BD2946204600F063FD70BD13
:10FF10005099002010B500F055FE10BD10B5FAF74D
:10FF20003DFF002010BD0000034A538803809088E5
:10FF300008800020704700000099002010B5FFF7EE
:10FF400005FC10BDFF21D131484310B508490968AF
:10FF500040180AD0017E002907D00022E0210A546F
:10FF6000062102F072FD002010BD022010BD00002D
:10FF7000242B002070B50E46FF21D13148431F4984
:10FF800088B00968441836D0207E002833D0002578
:10FF90002046009501950295FF300395049505953F
:10FFA0000695102269460D30079508F0D5F9102204
:10FFB00004A9304608F0D0F9204610223146EC3032
:10FFC000FAF740FD204604AA6946FC30FAF7E6FE3F
:10FFD0002646E0363570204602F08FFE0120FF21D4
:10FFE00030705A3108550121206A09040843206203
:10FFF000002008B070BD022008B070BD242B002086
:020000040001F9
:10000000FF22D1325043104A126880181AD0027E63
:10001000002A17D0826D0A70C36D826D1B06120A0A
:100020001A434A70C36D826D1B04120C1A438A7006
:10003000C36D826D1B02120E1A43CA70C06D087127
:100040000020704702207047242B002030B40F4D51
:100050002C68647CFB2C03D81B2C02D21B2400E0F0
:10006000FB240480E000703008802868407CFB2876
:1000700003D81B2802D21B2000E0FB201080C00008
:100080007030188030BC002070470000282B002002
:1000900070B50D46FF21D13148430849144609681F
:1000A000401808D0017E002905D0FFF7ABFA287070
:1000B0002070002070BD022070BD0000242B0020A5
:1000C000FF21D13110B54843124982B00968441864
:1000D0000DD0207E00280AD00F49086A496A019194
:1000E0000090607E002805D0012808D00BE0022097
:1000F00002B010BD6946204602F0A4FA03E069464A
:10010000204602F0CFFD0120A034E071002002B0B3
:1001100010BD0000242B00201099002010B501F024
:1001200083FC10BD70B50C46054603F0F9FD0028B0
:1001300003D01F2C03D9122070BD0C2070BD2146A6
:10014000284602F07FFE002070BD000010B5044676
:1001500003F0E6FD00280CD00848407AC00703D021
:100160000748C079002806D0204602F07DFE002016
:1001700010BD0C2010BD122010BD0000989800206A
:1001800050990020FFB506461F4889B00078139C9F
:1001900017460D46002808D103F0C2FD002804D000
:1001A000AE4205D911200DB0F0BD0C200DB0F0BD50
:1001B000012F01D106263546684600960195077243
:1001C0000C9941721299817262782178100E120294
:1001D000A37811431A0C1B041943E37810431A0A3D
:1001E000104322791B06104362791943120210430F
:1001F000059004916846149901761599417602F0AC
:100200004BFF00200DB0F0BD50990020FF2370B5CA
:10021000D13358431B4B1B68C01815D0037E002BED
:1002200012D00B461B3BE12B12D2FF2349339A42DB
:100230000ED3154B154DD418154BAC4206D2852361
:100240001B019A4204D105E0022070BD9A4201D9F7
:10025000122070BD0F4B1B685B7C8B4201D21C4689
:1002600000E00C461B2C01D21B2102E08B4200D285
:100270001946034680339987DA8702F003F9002094
:1002800070BD0000242B0020B7F7FFFF47020000DD
:1002900090420000282B0020024610B41B3AE12AAD
:1002A00015D2FF224932914211D30D4A0D4C8B18C1
:1002B0000D4AA34204D285221201914207D101E0E6
:1002C000914204D8094A1268527C824202D210BC80
:1002D00012207047064A5080918010BC0020704761
:1002E000B7F7FFFF4702000090420000282B0020D4
:1002F0000099002030B40F4B1C6A0B46E5051343F0
:10030000002D01DB9D0705D4240501D45B0701D432
:100310008A4202D030BC11207047C30700D00021B0
:10032000830700D50022044B9871D9711A7230BC32
:10033000002070471099002000990020F1B5224854
:10034000224E0468707982B00025A84238DD204F23
:10035000207E00282ED0607E00282BD10522684602
:100360000299FAF76FFB2046FF30C13041780078E0
:10037000081AC1B23868C27B007C101806225043AC
:1003800009185220E28C005B101808186946801D7D
:10039000C88020469C30019A00994260016001208B
:1003A000A4210855207F0221084320776946204672
:1003B00002F018F87079FF34D1346D1CA842C7DC04
:1003C000002003B0F0BD0000242B00205099002035
:1003D000282B0020F8B5FF248646D13460433D4CDD
:1003E0000D462468069904190AD0207E002807D0FB
:1003F0002046FF308130867D002E03D00C20F8BDD2
:100400000220F8BD344E1746366A1F43B446F6053F
:10041000002E01DBBE070BD46646360501D47E07ED
:1004200006D40126002D01D1934201D1FF0801D04D
:100430001120F8BDEF0700D00022AF0700D5002340
:100440009A420FD1C77EBC467F1EBE40964211D154
:100450006646032E03D1867E8E4200D08176667E6C
:10046000012E16D1C27E71461346002000F0CAFE4E
:100470000020F8BDB343DA0701D0012208E09A0753
:1004800001D5022204E05A0701D5042200E000222F
:10049000134616461E4308D06E463270737045767A
:1004A000C2750376002907D007E0C27E7146134665
:1004B000002000F0A7FE0BE001218176C374837455
:1004C000207F0421084320773146204602F02EF990
:1004D0000020F8BD242B00201099002030B4124BCE
:1004E0001978002902D15978002902D030BC0C209B
:1004F000704744780178220E2402857821432C0C21
:100500002D042943C57822432C0A224304792D0661
:10051000407929432243000202439960DA600120B6
:10052000D87130BC002070475099002070B50C463F
:10053000054603F0F5FB00280DD009484079C007B7
:1005400003D00848C079002807D02146284602F089
:1005500003FE002070BD0C2070BD122070BD000095
:10056000C099002050990020FFB583B014460D4675
:1005700006460C9F03F0D4FB002803D009484078BE
:10058000002802D00C2007B0F0BD68460671058037
:10059000448006994171877102F064FE002007B023
:1005A000F0BD00005099002070B50C46054603F0E0
:1005B000B7FB002803D01F2C03D9122070BD0C20DC
:1005C00070BD2146284602F059FE002070BD000093
:1005D000FFB5FF21D1314843374987B00968154637
:1005E000441808D0207E002805D0607E002805D061
:1005F0000C200BB0F0BD02200BB0F0BD2746FF373A
:100600004137787E012600281ED0204602F068F887
:10061000E0200655BE7620460822E4300899FAF715
:1006200011FAE220055320461022EC300A99FAF71D
:1006300009FA38460821343803F0EEFF3846042121
:10064000243803F0E9FF33E0082268460899FAF7F6
:10065000F9F9684605810A300821069003F0DCFFAD
:1006600004A802300421074603F0D6FF694620465D
:1006700001F07FFFE020065520460822E43008996B
:10068000FAF7E0F9E220055320461022EC300A99EF
:10069000FAF7D8F92046FF3008220D300699FAF70C
:1006A000D1F92046FF30042239461D30FAF7CAF945
:1006B00000200BB0F0BD0000242B002010B5194C19
:1006C0002068002800D00120802317A21F4909F0CC
:1006D000C9F92068808A02F039FD03F0E7FA1C4866
:1006E00000210161C160016241622268117806291E
:1006F00003D301210023436201621178082903D347
:10070000036A3C24234303621178092904D3492353
:10071000026A1B021A4302620021C9438A0D426326
:10072000016310BD282B00202E2E5C2E2E5C7374CE
:1007300061636B5C636F6E74726F6C6C65725C6C22
:100740006C5F696E69742E630000000000000A028D
:100750001099002010B5FF217531095C002904D0E3
:100760000121FF308130818010BDFF3028217130A0
:1007700003F006FD10BD014610B5FF3181318A88B6
:10078000FF307130002A05D000228A80282103F032
:10079000F7FC10BD03F048FD10BD0000F8B5784E21
:1007A0000C00054647D0207865380B287FD2010021
:1007B0007944097949188F4405083F357A284468F7
:1007C0007A70610000F0FEF9B6E06088FF21D13157
:1007D00048436C4909684418207E00282BD02046E5
:1007E000FF308130C168002925D16749496901225C
:1007F0001143C16008218171204605F0C5F8002829
:1008000019D02046FEF7FEFC96E06088FF21D1312A
:1008100048435C4909684018017E00290BD001F06B
:1008200031FE89E06088FF21D1314843554909688C
:10083000401803F0E1F87FE060882221FEF71AFDFE
:100840007AE050496788FF20D1300968784344181E
:10085000204601F0E9FF207E00280BD02046FF3023
:100860004130417E002902D1807E002802D02046FE
:1008700002F07AFF384600F0ADFB5DE0B269002A75
:100880005AD061786088904756E003F073F93F488A
:10089000818A03F075FC4FE009E06088FF21D131C7
:1008A000484338490968401803F040F844E020788C
:1008B000002802D001281ED039E0E088FF21D13184
:1008C00048433049096847183846FF30713003F013
:1008D000ABFC3846FF305D3003F0A6FC3846C8302C
:1008E00003F0A2FC384603F01BF9384601F0B2F9D8
:1008F000002038761BE0E088FF21D13148432149B0
:100900000968471822480068807F00280CD0306AA8
:100910001121084208D0207A0028384602D002F07F
:1009200023FF01E002F090FF384601F065F9F1681D
:100930002046002900D08847002D1FD0E80601D5A9
:1009400001F004F9A80601D502F094F8680603D571
:100950007069002800D08047A80705D502F09EFCEA
:10096000FDF71BFC02F0ACFE280703D500F0C2FA2D
:1009700000F05EFB680501D5FAF7DCF8F8BD000071
:1009800010990020242B002000000250A89900207C
:10099000282B002010B5012903D0040004D0012029
:1009A00003E0FAF7CDF810BD00208223064A07497C
:1009B00009F058F82046FDF7D9FE00200449A06050
:1009C000087000F0F7FA10BD340A0020000006029B
:1009D0002C2B0020F0B56B4F0446787889B00D467B
:1009E000002803D00021084602F0B6FB664EB07E18
:1009F000012815D065480022654982770B8C5B047D
:100A000001D5012383776148807FF076637961485F
:100A1000079043726079C00705D0B868F96804E0B0
:100A20000C2009B0F0BD886AC96A039102905A4946
:100A30000020C866207900281BD1A079C007C00F0C
:100A40003076A26853781078190E1B0297781843F5
:100A50003B0C19433F04D37838431F0A1B06184345
:100A60001379527939431943120211434A4A5167A3
:100A700010670020454F01463877079841707D2068
:100A8000C000FAF715F845494969401838602088D0
:100A9000B8846088F8840798217981720020786092
:100AA0003F48983707613F48298801866988418611
:100AB000A9888186E988C186298901876989418752
:100AC00003F096FD0090FAF7DBFFB8620098000291
:100AD000000AF86203990298F961B861324803216B
:100AE0008177009841073148490F0090018068885C
:100AF0003887A8887887E888B88700201F21C043F6
:100B000079633863FAF7E0FF01460098284D817059
:100B10000521C1700020B864F864386578652868DC
:100B2000007A00280ED0234801AA006801902248CC
:100B3000017E2248009003F053FA2868017A009859
:100B400003F01EFB1448002700680097051D2220B3
:100B5000019060790521C3070C48DB0F827F28468E
:100B600000F092FB1649281D00F09FFB0A48032164
:100B700047600120B076054804F046FB002009B02C
:100B8000F0BD000050990020789800208097002048
:100B900010990020A0970020189800200000025013
:100BA00000980020F09700203898002058980020E6
:100BB000282B002030E4020030990020709800209B
:100BC0003098002010B5184C8CB0A07E012802D0BF
:100BD0000C200CB010BD154804F0D6FE002820D023
:100BE000134803F021FB0020124AA0765168002927
:100BF00001D0087650601048014608311EC90091A6
:100C0000014603940293019218311EC907942830BB
:100C10000693059204910FC808AC0FC4684600F013
:100C2000F5F900200CB010BD7898002080970020C6
:100C3000709800201898002030E40200F0B50746B4
:100C400080300669FD6874688DB0002C7ED000206D
:100C50007060786900287AD0417A837A19404368B5
:100C600000685943091808790307100A1B0F00028E
:100C70000A7918439206FF23D20F1B0212029843EF
:100C80001A4010430A791B025206D20F12049843ED
:100C90001A4009791043C9090002000A09060843ED
:100CA0000690002038772046FEF7BCFD0420AC609B
:100CB00028750020E875022068757948E5600068AD
:100CC000318AC08A814200D9084676492546403596
:100CD00048430495E882304660300890C17E204643
:100CE0008030099081739620F9F7E2FE396BAD1ED2
:100CF00040180A9000206076069837460002010EE0
:100D00003D200155B08C316A03060A0A1A43297046
:100D1000030A6A709C460A0C03041A43AA70020272
:100D2000090E1143E9702871634618376B713869F1
:100D300060647869A064384620300290049D81790F
:100D4000A981398DE981398C298201E014E016E00E
:100D5000798C6982B98CA982FA69B969E265A16561
:100D60002146C27A60310A70807AC870099803906F
:100D7000807B012805D008E000200DB0F0BD0021E7
:100D800071E7606C010C414021872046FDF706FAAF
:100D9000204601F0FFF90020A060E889424948435D
:100DA00042494018F9F784FE0A9940182060E88A01
:100DB000FF38F538F9F77CFE216840186060384844
:100DC0000068C07B012809D1288A37494843FF3889
:100DD000F538F9F76DFE216840186060A98A0A208D
:100DE00041432046FF305D3003F07AF92046FF3062
:100DF000B93001D0417A0172302003F0B1FA050018
:100E00002FD007202870002028712948FF21006872
:100E1000D131201AF9F7ACFAE880607E2872069882
:100E200006220002000E6872F968B86869612861DC
:100E3000388C2883788C6883B88CA88302983946CC
:100E4000C07AA877284638311F30F9F7FBFD3946BC
:100E50002846062230312530F9F7F4FD284601F006
:100E6000D3FD1348FF210068D131201AF9F780FA29
:100E7000039980B2897B00F0BAF80899002088763F
:100E80003046583003F0D0F90A494879401C48717F
:100E9000F9F7DEFD0020F9F759FE01200DB0F0BD95
:100EA000282B002071020000E2040000CA080000A4
:100EB000242B00205099002010B5094803F0B4F904
:100EC00008480021084A81765068002801D0017640
:100ED000516006484170064804F056FD10BD000000
:100EE00070980020789800201898002050990020D1
:100EF0008097002010B5064803F096F905490020B8
:100F0000054A88765168002901D00876506010BDE6
:100F10007098002078980020189800200249014815
:100F200008607047950901000896002010B5382028
:100F3000FAF71AFB040001D0012000E00020212173
:100F4000952308A2090508F08DFD0F48382204609A
:100F500000212046F9F7A0FD0C490C2004F0EAFC22
:100F600010BD00002E2E5C2E2E5C737461636B5CD2
:100F7000636F6E74726F6C6C65725C6C6C5F7363C4
:100F8000616E2E630000000018980020151E0020DE
:100F900010B502F0D1FEFEF749FE04490A2004F024
:100FA000C9FC0349022004F0C5FC10BD1D1E010050
:100FB000451D010010B5064C6078002807D0207848
:100FC000002804D1A078FAF761FB0020607010BD02
:100FD0002C2B002010B50446062003F0C1F9002890
:100FE00004D006210170848001F00EFD10BD70B5A3
:100FF00005460C46082003F0B3F9002805D010215F
:1010000001708580847101F0FFFC70BD70B50446ED
:10101000302003F0A5F9002808D02ECC2EC02ECC0D
:101020002EC01ECC1EC0303801F0EEFC70BD00009A
:101030000C4810B5014608311EC98CB0009101461C
:1010400003940293019218311EC907942830069325
:10105000059204910FC808AC0FC46846FFF7D6FF8D
:101060000CB010BD30E4020070B50546042003F05A
:1010700077F904000ED06F2020700748FF21006828
:10108000D131281AF9F774F96080287E6070204603
:1010900001F0BAFC70BD0000242B002010B50446FE
:1010A000042003F05DF9002804D06E210170448013
:1010B00001F0AAFC10BD000070B506460D460E20DA
:1010C00003F04EF9040014D009202070094826715D
:1010D0000068FF21281AD131F9F74AF9E0808035FC
:1010E000A88A2081E88A6081288BA081204601F0AF
:1010F0008BFC70BD242B0020FFB581B00646144642
:101100000D460E200A9F03F02BF9002809D00D216F
:1011100001708680C580048104994181878101F036
:1011200073FC05B0F0BD000070B505460C460A2002
:1011300003F016F9002807D000210170C580047261
:10114000017101F061FC70BD034B04A20C49002049
:1011500008F088FC70BD00005D0200002E2E5C2EA1
:101160002E5C737461636B5C636F6E74726F6C6C16
:1011700065725C6C6C5F636F6E6E2E6300000000C6
:101180000099FFFF70B5064614460D460A2003F08D
:10119000E7F8002806D0012101700671C5800472AD
:1011A00001F032FC70BD70B505460C46082003F016
:1011B000D7F8002805D0042101700571C48001F022
:1011C00023FC70BD70B50446FF308130816A002970
:1011D00014D0C06A002811D0042003F0C1F8050023
:1011E0000CD0682028700648FF210068D131201AF1
:1011F000F9F7BEF86880284601F006FC70BD0000D3
:10120000242B0020F8B507461C4615460E460A203A
:1012100003F0A6F8002807D0112101700771C680DD
:101220000572447201F0F0FBF8BDF8B507461546AB
:101230000E46102003F094F804000DD00A20207010
:101240002771E680002D04D008222946A018F9F75E
:10125000F9FB204601F0D8FBF8BDFFB581B006468A
:1012600014460D460E200A9F03F07AF8002809D094
:10127000022101700671C580047204994181878141
:1012800001F0C2FB05B0F0BD70B40907090F5201AF
:1012900011439A01039C11430225E2011143049E6C
:1012A00001704670284670BC704770B40A7C0270AA
:1012B0000A8A1623120A42700A69120C82700A699D
:1012C000120EC2700A7D02718A8A120A42714A693C
:1012D000120C82710A4620329479C4710C8D04720A
:1012E0000C8D240A44720C8C84720C8C240AC472F7
:1012F0004C8C04734C8C240A44738C8C84738C8CBB
:10130000240AC4730C7E04740C7F0D8B26062C0AF1
:10131000344344740C7F8D6926042C0C344384744C
:101320000C7F8D6926022C0E3443C474097F01752D
:10133000917AD27A52010A43427570BC18467047BE
:101340001023194312020A430270110A417002204D
:10135000704710B50446407E00280DD001280AD100
:10136000204601F0D0F90120E02108550021FF348A
:1013700041346176A07610BD4979204601F01AFD0E
:1013800010BD30B50446417E25460020E03587B0CB
:10139000002904D0012900D1287007B030BDFF21F9
:1013A0005A3108552870204601F0ADF9214608222F
:1013B000E4316846F9F746FBE220005B69460881A4
:1013C0002146FF3102A808220D310230F9F73AFB1D
:1013D0002146FF3104A804221D310230F9F732FB07
:1013E0006946204601F0C5F80120287007B030BDDD
:1013F000F8B50D46040001D0012000E00020544B58
:1014000054A25E4908F02EFB6B782A781B02D21892
:1014100092B25B4893079B0F03705307DB0F437037
:101420001307DB0F8370D306DB0F160AC370A91CEA
:101430000671002E24D00778FF232046514AD1336D
:10144000E030032F1DD04578002D02D0657E002DA1
:101450006DD00078002802D0607E012867D0106827
:101460000D46201A1946F8F783FF80B2012F6CD081
:101470000221454A1469002C02D033462A46A0476F
:10148000F8BD4678002E13D0667E002E10D10E785F
:10149000032E0DD0042E0BD0052E09D0062E07D01A
:1014A0000A2E05D00B2E03D00D2E01D0112E3ED1C9
:1014B0000078002845D0607E002802D0012825D081
:1014C0003FE0087803283CD004283AD0052838D0DB
:1014D000062836D00A2834D00B2832D00D2830D038
:1014E00011282ED026466C78A41C204602F038FF26
:1014F0000700C5D022462946F9F7A4FA3046FF3046
:101500003A460021B13002F040FFF8BD08780328C8
:1015100017D0042815D0052813D0062811D00A2882
:101520000FD00B280DD00D280BD0112809D0106832
:101530001946201AF8F71CFF80B23D21FDF79AFEEC
:10154000F8BD2046FDF744FDF8BD012191E70000FC
:101550003E0600002E2E5C2E2E5C737461636B5C65
:10156000636F6E74726F6C6C65725C6C6C5F7064D0
:10157000755F636F6E6E2E63000000000000060250
:1015800040970020242B002010990020F0B504463D
:10159000007F83B0002802D0627E002A0FD00E4662
:1015A0005B492546627EFF350836C8798135012AB8
:1015B00010D0E875097A2976002836D037E0400740
:1015C00001D5232200E02A224979204601F026FA9B
:1015D00003B0F0BD0122216A120311432162E875B4
:1015E000002801D1FEF794F87178EA7E01400120CD
:1015F000521E904088420DD08143CA0701D001217C
:1016000008E08A0701D5022104E0490701D5042139
:1016100000E0C1B2684601714171E974A97401A981
:10162000204601F0AEF803B0F0BDFEF771F8717816
:1016300008400746287E002801D1FEF769F8317876
:10164000FB2608400740E87E012804D0022805D088
:10165000032806D006E07F087F0003E0FD20074056
:1016600000E03740F80701D0012708E0B80701D5AE
:10167000022704E0780701D5042700E00027684628
:1016800007704770002F22D02046FF30C1304178CC
:101690000078081AC1B21F480068C27B007C10188D
:1016A0000622504309185220E28C005B10180818DB
:1016B000801D694648802046FF30833009880182BA
:1016C000694649884182002F03D0012002E00020B2
:1016D000EFE70020A8756946204601F07DF8002F4D
:1016E00011D1207F41070ED5304020770A48FF21D5
:1016F0000068D131201AF8F73BFEEA7E81B213462A
:101700000020FFF77FFD2046FFF735F803B0F0BD5E
:1017100000990020282B0020242B0020F8B5054636
:10172000407E012808D02E46FF3681360F46F07DD8
:101730000837002805D006E01721284601F03AFBBB
:10174000F8BDFDF7E5FF797808400446307E0028B3
:1017500001D1FDF7DDFF3978FB2708400440F07E1A
:10176000012804D0022805D0032806D006E064082A
:10177000640003E0FD20044000E03C40E00701D0AD
:10178000012408E0A00701D5022404E0600701D588
:10179000042400E00024684604704470002C22D029
:1017A0002846FF30C13041780078081AC1B21E487F
:1017B0000068C27B007C1018062250430918522092
:1017C000EA8C405B10180818801D6946488028463E
:1017D000FF30833009880182694649884182002CA4
:1017E00003D0012002E00020EFE70020B075694639
:1017F000284600F0F1FF002C11D1287F41070ED5BB
:10180000384028770948FF210068D131281AF8F7B5
:10181000AFFDF27E81B213460020FFF7F3FC2846AD
:10182000FEF7A9FFF8BD0000282B0020242B002084
:1018300038B50446407E002817D008460A7A08309A
:10184000002A17D04288A38CD21A012392B2DB035C
:101850009A4202D85B1E9A420CD923486946806896
:101860000090204601F082FA3AE01821204601F06B
:10187000A1FA38BD2246FF3283320B89138249898F
:1018800051820078951E002807D0E97E0122491E6A
:101890008A40904201D0012000E00020A875002875
:1018A0001AD10121206A090388432062207F410761
:1018B00016D5FB21084020770C48FF210068D13164
:1018C000201AF8F755FDEA7E81B213460020FFF793
:1018D00099FCA87D002803D0A98A2046FCF7D4FDF6
:1018E0002046FEF748FF38BDA0E30200242B00206D
:1018F00010B500F0BEFF10BD10B5FEF73CFF10BDE7
:10190000014A106011717047342B0020FF21D13142
:1019100000B54843104983B00968401818D0017ECB
:10192000002915D00D496A4609680B7813704B8859
:1019300053808988918001460122A0314A718A79B9
:10194000521C8A71694601F04AFA002003B000BDBA
:10195000022003B000BD0000242B0020282B002013
:10196000FF22D1325043064A1268801806D0027E08
:10197000002A03D0807E0870002070470220704744
:10198000242B002001494861704700001099002075
:10199000F8B50D460446FEF7EEFE2E46287A0836C8
:1019A000124F16280ED1607E01280BD13868FF2116
:1019B000201AD131F8F7DCFC81B2002370781A4686
:1019C000FFF720FC2046E030017801290DD10021ED
:1019D000017041703868FF21201AD131F8F7C8FC36
:1019E00081B2687A0022FFF7CDFBF8BD242B0020DE
:1019F00070B50D460446FEF7BEFE2046E030017885
:101A000001290ED10021017041700648FF210068B4
:101A1000D131201AF8F7ACFC81B2687A0022FFF7C6
:101A2000B1FB70BD242B0020F3B581B0074601281F
:101A300053D80298002850D02E4C0025E08800286A
:101A400054DD2068E900461831460298F9F7BEFED9
:101A5000002847D0B079B84244D1E088411B4A1EE3
:101A6000002A2EDD0027401EA84239DD01268E43C4
:101A700008D0E8000146226808315118101805F016
:101A800073F90127E188491B491EB14219DDE819A4
:101A9000C000034622680833D118101805F064F915
:101AA0007F1CE919CA00134620680833C118801842
:101AB00005F05AF9E088B61C401B401E7F1CB0425E
:101AC000E5DCE0882168C000083808180021F9F733
:101AD000C3FDE088401EE08008E0122003B0F0BDA6
:101AE0000026CFE7E0886D1CA842AADC002003B0E6
:101AF000F0BD0000B82B002010B5FCF7B7FC114872
:101B00000178002908D14178002905D1C1700E481B
:101B100002F08AFBFCF79CFC002001F0A5F90021F3
:101B2000084601F019FBFFF7C7F904F02BF802F0A3
:101B3000BDF802F001F902F021F902F08BF802F091
:101B400011F910BD50990020A8990020F8B5274C34
:101B5000657A207A854225D0A84223D0244E002CD5
:101B600021D0207AA17A0840616848432168411851
:101B70004A780878120280188B78CA79891D80B259
:101B8000002A29D0FF27D13778433768C019076A60
:101B9000BF030AD50122016A520491430162102059
:101BA00000F094FDF8BD0021E2E7077E002F13D07E
:101BB000FF275A373F5C002F0BD0002B09D03D2167
:101BC000FF30813081710B49496901221143C160A5
:101BD00002E0921CFFF70CFC002C02D0207A401C83
:101BE0002072207AA842BAD1F8BD000010990020D6
:101BF000242B00200000025070B504462546FF3516
:101C0000B135007E2E46303E002816D0F068002800
:101C10001FD1E020005D00281BD10021284602F0E2
:101C2000A8FB060015D0727801462046921CFFF7EB
:101C3000DFFB304602F0B1FBEFE70021284602F05F
:101C400098FB002802D002F0A8FBF6E700203063E2
:101C5000706370BD10B5FF30B1300021044602F052
:101C600088FB002807D002F098FB0021204602F0F4
:101C700080FB0028F7D110BDF0B4034660331A7E14
:101C8000022A5CD3521E002A54DD52070021520F53
:101C900094460C46012A0BD46246521ECD002D18E4
:101CA0006F6C2E6C491C641CEF63AE639442F5DDCF
:101CB0001C7E6246641E94423CDDCC002418666C97
:101CC000256CE663491CA563CC002418666C256C62
:101CD000E663491CA563CC002418666C256CE6639A
:101CE000491CA563CC002418666C256CE663491C6E
:101CF000A563CC002418666C256CE663491CA563BB
:101D0000CC002418666C256CE663491CA563CC00E6
:101D10002418666C256CE663491CA563CC00241866
:101D2000666C256CE663A5631C7E491C0832641E44
:101D30009442C2DC187E002801D0401E1876F0BC08
:101D400070470000F8B501292ED000252E4C00293F
:101D50002DD061694268891A62031031914222D301
:101D60006669E16849084900E1606169B1420DD1E5
:101D70000523002200950099491C00910729FADBF0
:101D8000521C9A42F6D36169B142F1D06169091DD2
:101D90002161E26853085B0001221A43E2601B4B99
:101DA00000221A620163F8BD00F076F8F8BD060063
:101DB00001D0012000E00020BD239B00144A1549FA
:101DC00007F050FE0020F8F7C1FE75601248357725
:101DD0000570FFF7EFF86269E06840084000E060D6
:101DE000606990420DD10523002100950098401CA8
:101DF00000900728FADB491C9942F6D360699042AB
:101E0000F1D0F8F725FEF8BD000002504004025062
:101E1000B8FC0000000006022C2B0020F8B5027D63
:101E2000022A35D18068097844692030007A012877
:101E300030D00126607A227A821AD2B25318A27A5E
:101E4000521CD2B2921B934204DC401860722020D4
:101E500000F03CFC657A207A281AC1B2A07A401CB6
:101E6000C0B2801B814213DC002007460090002E88
:101E70000EDDA07A626828402168504341186D1C2D
:101E8000EDB2091D0098F8F767FE7F1CB742F0DB42
:101E90000020F8BD0226CDE7F0B583B0040001D0E4
:101EA000012000E00020A34BA3A2AC4907F0DAFD1B
:101EB0000120F8F74BFEF9F703FF0090A84801272F
:101EC00007700220F8F700FE0120F8F7F7FD012166
:101ED00000220846F8F7C8FDA24E357EF8F742FE0C
:101EE0004119A14D2869020A1202C8B210432861A3
:101EF000367FF8F73DFE69698019090A0902C0B208
:101F0000084368610120F8F739FE984D6E69E8686A
:101F1000B8430022E8606869B0420DD10523002172
:101F200001920198401C01900728FADB491C994254
:101F3000F6D36869B042F1D08C494869093008612C
:101F4000CA6853085B003A461A43CA60884A0021AF
:101F500011622063844E8748B063874870632546CA
:101F6000203568780321F8F7EDF908462530F8F7B1
:101F70000BFE687AC207D20FC00703D07F4988687A
:101F8000C96802E07E49886AC96A12040B041B0E04
:101F90001B021A43C9B20A437349CA630204120EF0
:101FA000C1B2120289180202120E000E12040006BB
:101FB00010180918734801602646803631690029D7
:101FC0006CD0AA7A012A78D07822525C70314B7991
:101FD00012040F791B023B431A43C2614B780A7803
:101FE0001B02D2188B78C9781B040906591851189E
:101FF00001624169CA08D2000521114341615B4871
:10200000416962680123881A9B07984200D9501AD7
:10201000F8F766FD544FF86160207862386BFF2155
:10202000090388432521090301433963564A51694D
:10203000102081430843506130690028606942D014
:10204000002875D0417A827A114042685143026873
:10205000891842680020091DF8F77EFD30692022AA
:1020600001680020091DF8F795FDF86801090901CC
:1020700006200843F86045480C2142690A43426142
:1020800042698A43426182698A4382610098F9F712
:1020900025FE0020F8F772FD03B0F0BD3CA10968F1
:1020A0000191A97A01AA515C42694907D208D2007C
:1020B000490F11434161A2E7FFE74169C908C9001F
:1020C0000F4347619BE700280FD0417A827A114085
:1020D000426851430268891842680020091DF8F7D8
:1020E0003BFD287A012802D00FE00021F4E7606967
:1020F000417A827A491CC9B2114042680068514352
:1021000009180120091DF8F727FDA16920220020E8
:10211000091DF8F73FFD287A012807D00520F96846
:10212000090909010843F860A5E701E00420F6E782
:1021300000218EE72F0200002E2E5C2E2E5C737481
:1021400061636B5C636F6E74726F6C6C65725C6CF8
:102150006C5F7363616E2E63000000000000060276
:102160002C2B002034960020000802500000025062
:102170004004025055555500D6BE898E5099002016
:102180001099002040080250400902508008025077
:102190000001060470B5040001D0012000E0002019
:1021A000EF230F4A0F4907F05DFC8E20005D2546A6
:1021B00060350128A878687006D0E9784018252194
:1021C000F8F7C0F8A97070BD218FE08C0122FDF7EF
:1021D0006FFA60872521F8F7B5F8A97070BD000087
:1021E0000CE2000000000602FFB50146714AFF2024
:1021F000D1301268484387B01F46841809D0207E2A
:10220000002806D06C480068C27B007C1018884209
:1022100002D802200BB0F0BD099800280BD0002F87
:1022200009D02046FF3081300190C168002905D0D7
:1022300080790BB0F0BD1E200BB0F0BDE020005D3A
:10224000002804D1FF205B30005D002802D03A2036
:102250000BB0F0BD2546FF35C135A87A002861D105
:102260002046FDF7DDF9C421095B814200D2084612
:10227000014604903846F8F765F886B20804000C69
:1022800001D0761CB6B2002E61D0FF34B934607A2A
:10229000217A401AA17AC0B2491CC9B28219491EDA
:1022A0008A420CDD401C88423CDA01983A46406C78
:1022B0000999F8F7C7FB0120A8722F726F72012EDF
:1022C00033D00498002C80B2059030D0607AA17A87
:1022D000084061684843216840180599CAB24270B5
:1022E000001D01900899FFF72BF801460198059A07
:1022F0000818801C0999F8F7A5FB05990998761E1E
:1023000040187F1AB6B20990002C02D0607A401CA7
:102310006072A87A00281BD0697A0598814208D398
:10232000012007E007200BB0F0BD3846CAE70020C7
:10233000D3E70020214B22A2002107F093FB697A0A
:102340000598081A0006000E68722DD1A8722BE0BD
:10235000002E29D00498874200D8384685B2002C38
:1023600025D0617AA07A014060684143206809184D
:10237000EAB24A70091D019101210198FEF7E0FFC0
:1023800001992A464018801C0999F8F75BFB0998C7
:10239000761E40197F1BB6B20990002C02D0607ADD
:1023A000401C6072002ED5D100200BB0F0BD002182
:1023B000DEE70000242B0020282B002099040000D9
:1023C0002E2E5C2E2E5C737461636B5C636F6E7477
:1023D000726F6C6C65725C6C6C5F636F6E6E2E639B
:1023E00000000000F8B506460D46052001F0F0FF9C
:1023F000071E15D0012101707C1C052229462046AC
:10240000F8F720FBA8796071E8880823000AA0711A
:102410003A460321304600F03FFA384601F0FEFF0D
:10242000F8BD70B506460C460C2001F0D1FF051E24
:1024300026D00021017021786970A178A970618887
:10244000681C090AE97021792971A1880C23090AFD
:102450006971A179A971E1882A46090A8171217AF5
:10246000C1712189090A0172A17A41726189090A3F
:1024700081720321304600F00FFA284601F0CEFFAA
:1024800070BD0000F8B50546092001F0A1FF041E4B
:1024900042D02946214B80311B6ACE1D4A8F9F06B0
:1024A000F936002F0ADA1B0508D5F37E032B05D178
:1024B0000A8F3D2392011B01D21892B2142303709C
:1024C0000B8F63700B8F601C1B0AA370E270120AE3
:1024D00022718A8F62718A8F0923120AA271CA8FB0
:1024E000E271C98F2246090AC1710321284600F012
:1024F000D3F900280DD1FF217531495D002902D0A3
:102500000120B08005E02846FF302821713001F01D
:1025100037FE204601F082FFF8BD00001099002030
:1025200070B506460C46092001F052FF051E1FD06B
:1025300015210170217869702188681C090AA97029
:10254000A178E97061880923090A297121796971E3
:10255000A1882A46090AA971A1798171E188090A2D
:10256000C1710321304600F097F9284601F056FF6B
:1025700070BDF8B505460E46172001F029FF071E6D
:102580002FD0032101707C1C082231462046F8F729
:1025900059FA307A207230893146000A60720A3462
:1025A00008220A312046F8F74DFA20463146083015
:1025B00004221231F8F746FA17233A460321284637
:1025C00000F06AF90446384601F028FF002C08D1D3
:1025D000FF217531495D002904D00121FF2085309C
:1025E0004153F8BD2846FF302821713001F0C8FD65
:1025F000F8BDF8B505460C460D2001F0E9FE061EB3
:1026000017D004210170701C074608222146F8F7F4
:1026100019FA38462146083004220831F8F712FA30
:102620000D2332460321284600F036F9304601F0EA
:10263000F5FEF8BD0249C968002900D00847704777
:102640001099002070B505460E46092001F0C0FE25
:10265000041E21D008210170601C7368326804F0E8
:10266000CDFA092322460321284600F015F9002857
:102670000FD1FF217531495D002904D00121FF20D0
:102680008530415305E02846FF302821713001F0A4
:1026900077FD204601F0C2FE70BD70B506460D46BE
:1026A000092001F095FE041E0FD009210170601C65
:1026B0006B682A6804F0A2FA0923224603213046F7
:1026C00000F0EAF8204601F0A9FE70BD014610B501
:1026D0000248007E01F0B4FB10BD000030990020DC
:1026E00070B50546012001F073FE041E0AD00A21D0
:1026F0002170024601230321284600F0CDF8204630
:1027000001F08CFE70BD70B50546012001F060FE41
:10271000041E0AD00B212170024601230321284602
:1027200000F0BAF8204601F079FE70BD70B504469D
:102730000D46032001F04CFE061E1AD01621017032
:10274000297871706978B1700323324619462046A2
:1027500000F0A2F80546304601F060FE002D08D1D9
:10276000FF217531095D002904D00121FF2085304A
:10277000015370BD2046FF302821713001F000FD6B
:1027800070BD70B504460D46032001F021FE061E03
:102790001AD017210170297871706978B1700323FC
:1027A00032461946204600F077F80546304601F0DB
:1027B00035FE002D08D1FF217531095D002904D0B7
:1027C0000121FF208530015370BD2046FF302821B4
:1027D000713001F0D5FC70BD70B505460C46052082
:1027E00001F0F6FD061E1ED01821017021787170CF
:1027F0006178B170A178F17061880523090A31719F
:1028000032460321284600F047F8304601F006FE24
:102810006088002807D02078002804D00121286A89
:10282000C9020843286270BD70B50546012001F059
:10283000CFFD041E1CD0122121700246012303216A
:10284000284600F029F800280FD1FF217531495D95
:10285000002904D00121FF208530415305E028469E
:10286000FF302821713001F08BFC204601F0D6FDAD
:1028700070BD70B50546012001F0AAFD041E0AD006
:1028800013212170024601230321284600F004F899
:10289000204601F0C3FD70BDFFB585B005000DD029
:1028A000287E00280AD02846FF3081300190C06879
:1028B000002806D00198807909B0F0BD022009B047
:1028C000F0BDE020405D002802D03A2009B0F0BD04
:1028D0002C46FF34B934607A217A401AC2B2A17A08
:1028E00020461038491C00908A422ED200210098C0
:1028F00001F03FFD060028D0002C4AD0607AA17A72
:1029000008406168484321684718B01C02907078FD
:1029100078703F1D727831783846FEF711FDC01986
:102920007278801C0299F8F78DF8002C02D0607A3A
:10293000401C6072304601F030FD607A217A401A06
:10294000C1B2A07A401C8142D0D3607A217A089E1D
:10295000411ACBB2A17AF6B24A1C93421DD2002C86
:1029600019D0084061684843216845186E702D1DD4
:10297000324628460699FEF7E3FC4019801C089A67
:102980000799F8F75FF8002C39D0607A401C607224
:1029900035E00027B9E70025E8E7069803902F46C1
:1029A0000798089D0290A81C80B201F0D9FC040091
:1029B00025D0039820706670A01C2A460299F8F76B
:1029C00041F822460021009801F0DFFC0198816A5D
:1029D000002914D0C06A002811D0042001F0C0FCE6
:1029E00004000CD0682020700648FF210068D13117
:1029F000381AF7F7BDFC6080204600F005F800208B
:102A000009B0F0BD242B0020014610B50248007E1D
:102A100001F04AFA10BD000030990020F8B50746D1
:102A200015460E46032001F0D3FC041E0CD01121E4
:102A3000017066700323A570224619463846FFF7D9
:102A40002BFF204601F0EAFCF8BD70B506460D46A6
:102A5000022001F0BDFC041E0BD00D210170657039
:102A60000223224603213046FFF716FF204601F0DD
:102A7000D5FC70BDF0B58848A3B040691390417A89
:102A8000149100284BD0007A884248D08348807E39
:102A9000012842D08248407800283ED07E48014636
:102AA000203160302291199006A90AA81F91219027
:102AB000139800287ED0017A827A1140426800681B
:102AC00051430C1876D06079241DC01D8008800009
:102AD000205801F025FF209068461A90207869461A
:102AE0000007000F087020788006C00F487020781B
:102AF0004006C00F88702078C009C87060780871DF
:102B00002178241D4906CA0F69468A701590801FD6
:102B10000294202805D31398B3E01398017223B0D0
:102B2000F0BD22980078002875D0029902984B7861
:102B30000078190E1B021843029B12049D78564C14
:102B40002B0C19432D04029B2843DD782B0A1943D3
:102B5000029B2D061B7928431943029B5B791B02BC
:102B600019430A431999097E8C46002901D0C907E7
:102B7000C90F00234D1E0BD42F46DD002E19B56B57
:102B8000F66B45405640354354D05B1CBB42F4DDE8
:102B900063468C4513DDCB001E19B36BF56B4340C8
:102BA00055402B4346D0336C756C434055402B4306
:102BB00040D000E068E0891C63468C45EBDC1A9845
:102BC000354D8678199C082B02D32846FFF754F818
:102BD000029902984A780078110E12021043029A64
:102BE00093781A0C11431B04029A1843D3781A0ADB
:102BF0001143029A1B06127918431143029A527923
:102C00001202114332040A43217ECB005B19491C96
:102C10002176DA6398633C2103A8F7F762FC082069
:102C2000694608731A9803AC0078022806D0062873
:102C300006D006E01398002826D022E0032000E00A
:102C4000022088751A9806228078C87520984875E1
:102C500002991F98F7F7F6FE0299159A891D921F9F
:102C600021981F2A01D91F2300E013466D462B75BA
:102C70000490F7F7E7FE2046FFF7DCFC13980028E6
:102C800002D0017A491C01721398017A149881428A
:102C900000D00DE723B0F0BD809700207898002089
:102CA0005099002070B505460E46092001F090FBB2
:102CB000041E21D00E210170601C7368326803F07D
:102CC0009DFF0923224603212846FFF7E5FD002842
:102CD0000FD1FF217531495D002904D00121FF206A
:102CE0008530415305E02846FF302821713001F03E
:102CF00047FA204601F092FB70BD70B505460120F1
:102D000001F066FB041E16D0052121700246012346
:102D100003212846FFF7C0FD0646204601F07EFB52
:102D2000002E08D1FF217531495D002904D0012111
:102D3000FF208530415370BD2846FF302821713077
:102D400001F01EFA70BD70B50546012001F040FB90
:102D5000041E0AD0062121700246012303212846C1
:102D6000FFF79AFD204601F059FB70BD70B504468F
:102D70000E46022001F02CFB051E18D00221017026
:102D80003178697002232A4603212046FFF784FD2B
:102D9000FF348134E068002806D13078A0710448FF
:102DA000406901210843E060284601F037FB70BD0F
:102DB0000000025070B506460D46022001F008FBE7
:102DC000041E0BD0072101706570022322460321E7
:102DD0003046FFF761FD204601F020FB70BD70B565
:102DE00006460C46062001F0F3FA051E28D00C21F9
:102DF000017021786970A178A97061880623090A99
:102E0000E97021792971A1882A46090A697103218B
:102E10003046FFF741FD00280FD1FF217531895D54
:102E2000002904D00121FF208530815305E0304680
:102E3000FF302821713001F0A3F9284601F0EEFAA5
:102E400070BD000070B50C460A46014604480546B0
:102E5000F7F7F8FD0348EC770121017070BD000021
:102E6000B8980020D8980020F0B57C4C002683B09C
:102E700000281AD020460078002822D1784838222D
:102E800000210446F7F708FE764D7748296801636C
:102E90002A7AA270012A16D0042A14D0002A17D048
:102EA000032A12D0022A12D012E02078002808D07B
:102EB0006D4802F069FD002802D120780028FCD17D
:102EC000267003B0F0BD012202E0022200E00622DB
:102ED000E270697A0020CB07DB0F23716073687E94
:102EE000E07261486F692E69C7648664A87A5F4E94
:102EF000C707FF0F3774002626735D4E368C7604A5
:102F000001D501262673C90702D054498E68C968C5
:102F10008446554800262946466410318E46217B5A
:102F200017073F0F49019B0140690F431F43001DD5
:102F3000F9B20193012A03D16346DB010B43D9B2F5
:102F400001704C4F001D012A68D04B490091CA7F87
:102F5000F7F778FD3E700099C87F4349801D4969A5
:102F6000464F4871217B40484901019AC069091DBB
:102F7000114301713A7842490830F7F763FD7E70DA
:102F800039493878C969801D4871A672297E3D4843
:102F9000CA076171002A03D0252333540122A2728B
:102FA0008A0705D5A37A26221A54A27A521CA27245
:102FB000490705D5A27A27211154A07A401CA07296
:102FC0000020294E60727069F16940794979401892
:102FD0002D49C0004018706301F00AFB2B49F7F738
:102FE000B1F90846F7F764FD2949496947187D207A
:102FF000C000F7F75DFDC01C38183060A17A706B17
:103000004843F7F755FD3168401870600020306183
:103010002070B063287A012807D010E0062271469C
:10302000F7F710FD06203E7097E77D20C000F7F708
:103030003FFD174949694018B0631648F063962070
:10304000F7F736FDB0600549012008700020F060F8
:103050000121054802F0D8F803B0F0BD50990020D6
:103060000897002098980020E896002028970020D4
:1030700010990020D8980020B8980020F8980020D7
:10308000D99800200E9700208A0300001027000026
:10309000000002500088130030B43CC802493CC113
:1030A0001DC81DC130BC704798980020FF2270B524
:1030B000D1325043134A1268801813D0027E002A7E
:1030C00010D002464032138A528A0F4C521C62437F
:1030D0005343024680320D4DD46D6C43A34203D955
:1030E000112070BD022070BD0A235943D165FF2213
:1030F0005A32125C002A02D0C83000F0F1FF0020E2
:1031000070BD0000242B0020E20400001027000006
:1031100010B4437801781A0E1B0284781943230CEB
:1031200024042143C4781A43230A1A4303794079BB
:1031300024061A430002024303482143C26281620B
:1031400010BC0020704700001099002001498880C1
:10315000704700002C2B0020F8B50025354C0F4699
:1031600000285ED020464078002859D13248807E21
:10317000012855D00020F7F7E9FC7C2200212F48D8
:10318000F7F78AFC2E4C012660694572606905726A
:103190002C48A577008C4004002800DAA6772A493D
:1031A0002A480A46138883865388C38693880387F0
:1031B000D38843874879C207D20FC00702D01D4881
:1031C0008168C068A17F92014901C91CA0691143AF
:1031D00001710C21417138461D4F257738707D20D3
:1031E0007D70C000F7F764FC1A49496925614018F1
:1031F00020603E737E73E08C17494843F7F758FC14
:103200002168A5604018606014480576144805617F
:1032100008484670867002210948E56001F0F4FF15
:10322000F8BD6078002803D0054802F0ADFB65705A
:10323000A570F8BD50990020789800209C97002038
:103240008097002010990020C099002070970020DE
:10325000A09700200000025071020000E0970020BB
:1032600000980020044902880A8042884A808288A7
:103270008A80C288CA807047C099002010B50C4669
:103280000A4601460348F7F7DDFB034801210470B5
:10329000417010BDD9980020F8980020F8B51B4D5A
:1032A000002628781A4F1B4C002814D01A49606950
:1032B000CA7F001D1F2A00D31F22931D4370001DCB
:1032C000F7F7C0FB2E706069E169407949794018D1
:1032D000C000C0196063114D6878002814D0E069FF
:1032E0002A78001D1F2A00D31F22911D41700C490E
:1032F000001DF7F7A7FB6E706069E16940794979B5
:103300004018C000C0196063F8BD0000D8980020C4
:103310008A030000E8960020B8980020F898002062
:10332000D998002010B500F029FD4020F8F71CF9CD
:103330001B4C0028A06100D001201A4B1AA2224980
:1033400006F090FBFF200130F8F70EF9002800D0BE
:1033500001201E4B14A21E4906F084FB3820F8F70A
:1033600003F96061002800D0012093239B000EA286
:10337000184906F077FB3820F8F7F6F8E0610028E6
:1033800000D00120144B08A2144906F06BFB14492D
:10339000082002F0CFFA1349002002F0CBFA10BD4A
:1033A000E8960020460200002E2E5C2E2E5C7374E0
:1033B00061636B5C636F6E74726F6C6C65725C6C76
:1033C0006C5F6164762E630001000E02490200000A
:1033D00002000E0204000E024F02000008000E025E
:1033E0004DE10000D9E00000F0B5044683B00120B3
:1033F000F7F770FB0120F7F7C1FBF8F761FC0190CC
:103400007F49012026460870203670700220F7F7A9
:103410005BFB0120F7F752FB012100220846F7F77A
:1034200023FB784F7D7DF7F79DFB4119764D286989
:10343000020A1202C8B210432861FF7EF7F798FB18
:10344000C1196869020A1202C8B2104368616F4963
:103450008A68022002438A608A6882438A606C4BD1
:103460005869001D1861DA6857087F0001223A4345
:10347000DA6000220A6220646648A86366486863CE
:103480007079E968702240079143400E0843E86074
:103490003079C207D20FC00703D060498868C96875
:1034A00002E05F49886AC96A12040B041B0E1B0202
:1034B0001A43C9B20A43EA630204120EC1B21202ED
:1034C00089180202120E000E1204000610180918C4
:1034D0005448016054A109680091F17A6A46525C2F
:1034E00041695207C908C900520F0A434261296B5A
:1034F000FF2212039143112252030A432A634C21F3
:103500006962F178012923D0022948D0A1694022BB
:103510000020091DF7F720FBA16940220120091DA9
:10352000F7F71AFBA16940220220091DF7F714FBE7
:10353000616938220020091DF7F72CFBE169382268
:103540000120091DF7F726FBF07806283AD03AE06B
:1035500036498A8842604B780A781B02D2188B78E9
:10356000C9781B040906591851188160A1694022C5
:103570000020091DF7F7F0FAA16940220120091D7A
:10358000F7F7EAFAA16940220220091DF7F7E4FAE9
:10359000616938220020091DF7F7FCFAD4E7616958
:1035A00038220020091DF7F7F5FA61693822012059
:1035B000091DF7F7EFFA616938220220091DF7F7B4
:1035C000E9FAC1E70320E968000709090901000FCA
:1035D0000843E86016480C2142690A434261426987
:1035E0008A43426182698A438261707A401C7072A8
:1035F0000198F8F773FB0020F7F7C0FA03B0F0BDAD
:103600002C2B002034960020000802504004025069
:103610000000025055555500D6BE898E50990020A5
:10362000109900204008025000020301309700204A
:1036300080080250F8B5012902D000F00BF9F8BD5E
:10364000040001D0012000E000203023174A18496F
:1036500006F008FA0120F7F791FAF8F731FB154D5B
:103660000646A96802200143A960A9688143A960B0
:1036700011480068418B808B0818F7F719FA0F4A38
:10368000516940181061D16801234F087F00194625
:103690003943D1602B62A0622046F7F781FA0020FF
:1036A000F7F76CFA3046F8F719FBF8BDDC0A002092
:1036B0000000060240040250282B002000000250A7
:1036C0001148807801281ED110B510488CB0C16B0C
:1036D000806BF7F76BFA002813D00020FFF7C4FBCC
:1036E0000B481EC803940293019200911EC80794D0
:1036F0000693059204910FC808AC0FC46846FDF705
:1037000085FC0CB010BD704708970020E89600209B
:1037100070E3020030B5427E83B0012A15D00D4A15
:103720000D7A116A546A0A462A40054600238035FC
:103730006B63090A2A6309020A432343694601931A
:103740000092FEF7AAFF03B030BD4979FFF732FBC4
:1037500003B030BD1099002002490148486070470D
:10376000353601000896002010B5DC210958C83014
:1037700000F0B6FC10BD70B50446407E002818D19C
:103780002546E0352878002813D0FF2001265A303E
:103790000655002028702046FFF7D5FA2E702046E7
:1037A000FDF710FD204600F0ABF82046FCF7D2FFF5
:1037B00070BD05212046FFF7FDFA70BD70B50446C7
:1037C000407E25460026E03501280ED128780028C5
:1037D0000BD02E700121206A090488432062204604
:1037E000FFF7B1FA2046FDF7EDFC2246FF322E70BE
:1037F0004132937EFF211348D131002B0DD09676B4
:103800006E700068201AF6F7B3FD81B20020FDF754
:10381000CAFC607E00280BD00FE06E700068201A92
:10382000F6F7A6FD81B201220020FDF7ABFCF0E720
:103830000121206A4904084320622046FCF79BFFCF
:1038400070BD0000242B002010B5C83000F0ECFC47
:1038500010BD0000F8B50446FAF788FF2746403748
:1038600000903D8AE08EAD1E042800D30120A842BE
:1038700000D205462046FAF7DFFC1F4E02463168AB
:103880004B7E002B02D0FF20F53001E07D20C000F0
:10389000002B06D13B8AFF279137BB4201D37D2005
:1038A0000001E38C032B02D3009B002B02D0FF30DE
:1038B000F53005E0E38E002B01D0684300E01046B0
:1038C0004A8B898B0546511864354819F7F7F0F88B
:1038D000A060FF209C30005D032807D13068418B39
:1038E000808B08184019F7F7E3F8A060034900201F
:1038F0000870FDF75FFBF8BD282B00202C2B002063
:1039000010B5FF30713000F08FFC10BDFF308130FA
:10391000C268002A07D10122034BC2715B691343BD
:10392000C360097A8171704700000250F0B5064605
:103930003546007EFF35C13583B0002850D0A87AC7
:1039400000284BD03046FBF76BFE2C46083C00901D
:10395000607A217A401AA17AC0B2491CC9B2401CCF
:10396000491E88423ADAFF3681360296687A009913
:10397000884200D80146CFB2002C36D0617AA27AB4
:1039800011406268514322688E18297A3A46091A12
:103990000298406C081801907770361D012130465E
:1039A000FDF7CEFC80193A46801C0199F7F74AF8DA
:1039B000687AC01B6872002C02D0607A401C60726A
:1039C000687A002813D0607A217A401AA17AC0B2AE
:1039D000491CC9B2401C491E8842C7DB03B0F0BD78
:1039E0000020A872687203B0F0BD0026CDE7002069
:1039F000A872287203B0F0BDF0B583B004000DD0FA
:103A0000207E00280AD02046FF3081300090C06818
:103A1000002806D00098807903B0F0BD022003B0E2
:103A2000F0BDE020005D00281CD000982546816A8A
:103A3000002914D0C06A002811D0042000F090FCA6
:103A400004000CD0682020703448FF210068D13178
:103A5000281AF6F78DFC60802046FEF7D5FF3A2045
:103A600003B0F0BD2546FF35B935687A297A401A8A
:103A7000C1B2A87A401C814231D228461038029047
:103A80000021029800F075FC060028D0002D43D0DC
:103A9000687AA97A08406968484329684718B01CC1
:103AA0000190707878703F1D727831783846FDF754
:103AB00047FCC0197278801C0199F6F7C3FF002DEE
:103AC00002D0687A401C6872304600F066FC687A62
:103AD000297A401AC1B2A87A401C8142D0D30098FA
:103AE0002546816A002914D0C06A002811D004201C
:103AF00000F036FC04000CD0682020700748FF213D
:103B00000068D131281AF6F733FC60802046FEF7B2
:103B10007BFF002003B0F0BD0027C0E7242B00206E
:103B200010B5FF30A9300021044600F022FC002827
:103B300007D000F032FC0021204600F01AFC0028DB
:103B4000F7D110BD70B50C460546FCF714FE207A7F
:103B50000E280BD10648FF210068D131281AF6F74C
:103B600007FC81B200221A20FDF75FFB70BD000048
:103B7000242B0020F8B5124F0026F88800281DDD00
:103B80003868B101441815D025462035A87E002894
:103B900006D0214610312046FBF7ECFC01202877A7
:103BA000E87E002806D0204629460830FBF7E2FCD4
:103BB00001206877F888761CB042E1DCF8BD00008F
:103BC0006097002030B50546044683B0A0350889CB
:103BD0002881488968818889A881164869460068D3
:103BE00002780A714288CA8080880881A8790028F2
:103BF00005D10120A87101A92046FFF7F0F8204661
:103C0000FCF7B9FD6879002811D0002068710A48D6
:103C1000FF210068D131201AF6F7AAFB81B2803467
:103C2000A08D0090638D2A7A0020FDF716FB03B06B
:103C300030BD0000282B0020242B002010B50822C6
:103C400000210348F6F728FFFCF750F810BD0000EC
:103C5000B82B002010B50A2200210A48F6F71CFFF5
:103C6000094801680748CA7C0270897C41701B21A1
:103C70004180FF2149318180032181710021C1717F
:103C8000017210BD00990020282B00200149086A0C
:103C9000496A7047109900200048704760990020D9
:103CA0000149086B496B70471099002070B5582284
:103CB00000211848F6F7F0FE164800210170C17087
:103CC0004170817041718171C171134A11745174D5
:103CD0002022027480228274C024447504228276D9
:103CE000282383772223C3770C488271F7234372FA
:103CF000FF238372C3727F250573302505744474D6
:103D0000F9248474C3740123037541758175C275E8
:103D100070BD0000509900209099002070990020FB
:103D20000448017C002901D0002070470121417422
:103D3000084670479099002010B50A2200210748D4
:103D4000F6F7AAFE0648054A016840681180090C8A
:103D500051809080030CD38010BD0000C0990020DA
:103D600088E4020010B5E1200349800088820846FB
:103D700000F05AFA10BD0000A8990020F8B568229A
:103D800000210748F6F788FE0648FEC8006884460A
:103D900003481EC08760466061460560C160F8BD8B
:103DA0009898002068E402004069704742689208D1
:103DB00092000A434260704770B5050001D00120AF
:103DC00000E0002083230DA2114905F04BFE114CA9
:103DD000207E401C082801D2012000E0002084231E
:103DE00006A20D4905F03EFE207E0C4A810089188E
:103DF0008D60217E491C217670BD00002E2E5C2E28
:103E00002E5C7574696C735C6D64632E63000000D6
:103E1000000005078496002000000B076496002030
:103E200010B53C2200210248F6F736FE10BD000016
:103E3000649600200149C863704700006496002022
:103E400070B50E460446082801D2012000E000208B
:103E500055230DA2114905F005FEF7F731FF054680
:103E60000F48610009180A8D022332430A850D4963
:103E70004A7E1A434A76C06B002800D08047284605
:103E8000F7F72CFF70BD00002E2E5C2E2E5C757493
:103E9000696C735C6D64632E6300000000000507AD
:103EA000649600208496002070B50C00054601D071
:103EB000012000E00020442311A2164905F0D2FDA4
:103EC000082D01D2012000E0002045230CA2124958
:103ED00005F0C8FDF7F7F4FE0646224629460F48CE
:103EE00000F053FA0E480122417E114341762038FA
:103EF000C06B002800D080473046F7F7EFFE70BD5A
:103F00002E2E5C2E2E5C7574696C735C6D64632E52
:103F10006300000000000907000005076496002008
:103F200084960020F0B587B0002768460773F6F73F
:103F300043FEF7F7C5FE284D6C7E6F76F7F7CEFE91
:103F4000264EE00718D003A9304600F012FA01907F
:103F5000002811D06846007B019980008019826892
:103F600000209047019800F018FA03A91B4800F0C0
:103F700000FA01900028EDD160070AD500F074F82E
:103F8000002806D0017C890089198A68811D0020DB
:103F90009047A0071ED5287E002400281ADD0F496F
:103FA00060004618308D002810D0A0004718B8686F
:103FB00000280BD0F7F784FE318D00910021318568
:103FC000F7F78CFEBA68002100989047287E641CA1
:103FD000A042E4DC07B0F0BD849600206496002087
:103FE00070B515460E46040001D0012000E0002007
:103FF000E1219B2304A2C90405F034FD267428881E
:10400000E0806888208170BD2E2E5C2E2E5C757439
:10401000696C735C7374696D65722E6300000000D7
:10402000FFB581B00A9F1D460E46040001D0012055
:1040300000E00020E121A32305A2C90405F012FD40
:1040400026740398A071E571278105B0F0BD0000CA
:104050002E2E5C2E2E5C7574696C735C7374696DA6
:1040600065722E630000000070B5F7F729FE054663
:104070000B4800220468002C02D0E068002804D01D
:104080002846F7F72BFE002070BD2146044800F0BB
:104090000DFC002020712846F7F720FE204670BD59
:1040A000902B0020044900220A604A6003494869B5
:1040B00003494A6008607047902B002000000250BE
:1040C000882B002010B5F7F7FBFD044904234A7E36
:1040D0001A434A76F7F702FE10BD000084960020CE
:1040E000F8B50E46040001D0012000E00020E121D7
:1040F000B4231CA2C90405F0B5FC0025761CF7F713
:10410000DFFD009020791D4F002813D03A68002071
:10411000002A0FD02146A24204D010461268002A7D
:10412000F8D107E0002A05D00246144800F0BEFB93
:1041300000202071012020710020E6602060386896
:10414000002806D0C1688E4203D3054600680028C7
:10415000F8D12A462146094800F000FB0098F7F7FD
:10416000BDFDF8BD2E2E5C2E2E5C7574696C735CE3
:104170007374696D65722E6300000000902B00203F
:10418000F8B50E46040001D0012000E00020E12136
:10419000AD231EA2C90405F065FC7D20C000464386
:1041A0000025761CF7F78CFD009020791D4F002824
:1041B00013D03A680020002A0FD02146A24204D032
:1041C00010461268002AF8D107E0002A05D00246FE
:1041D000144800F06BFB00202071012020710020AA
:1041E000E66020603868002806D0C1688E4203D39C
:1041F000054600680028F8D12A462146094800F003
:10420000ADFA0098F7F76AFDF8BD00002E2E5C2E7F
:104210002E5C7574696C735C7374696D65722E6362
:1042200000000000902B002070B5040001D0012098
:1042300000E00020E121BB230FA2C90405F012FC1D
:10424000F7F73EFD0546124800220368002B0ED00A
:10425000A34204D01A461B68002BF9D107E0002BBB
:1042600005D021460A4800F021FB00202071284695
:10427000F7F734FD70BD00002E2E5C2E2E5C757499
:10428000696C735C7374696D65722E630000000065
:10429000902B00200A4A41081140401A0949024661
:1042A00080080A400840101801090818064908400B
:1042B000010A0818010C08188006800E70470000DB
:1042C00055555555333333330F0F0F0F30B4204C42
:1042D0000246CD070B4640082843490822402040AB
:1042E0002340214012184B411A4C11469D07184695
:1042F00092082A439B0821402240204023408918ED
:104300005841154C0B460507024609092943000987
:104310002340214022402040591842410B460F4C77
:104320001506090A29431046150A234021405A1848
:10433000204025406841140C93B2050481B22C43FF
:10434000020CA0B218185141401830BCC0B27047DE
:1043500055555555333333330F0F0F0FFF00FF0003
:1043600010B5083080B200F033F8002800D00830D3
:1043700010BD10B50C4600F091F9002804D0002CB7
:1043800001D001792170083010BD0B4610B51146DF
:1043900008390B7100F0ACF910BD10B5083800F009
:1043A0003DF810BD5621095C2030CA060749D20EDF
:1043B0000A7002781207120FCA70027E5206520F5C
:1043C0004A7000790007000F887070472725002089
:1043D00000281FD070B506460F4805784468002DA8
:1043E00016D02088B04210D3F7F76AFCA1680029E4
:1043F00009D00D460968A160E168491CE160F7F742
:104400006DFC284670BDF7F769FC10346D1EE8D1CD
:10441000002070BD704700007C2B002070B514494F
:1044200005460878020148681418103C844218D3E5
:1044300089688908890009186268AA420ED8A942C9
:104440000CD9F7F73DFCA1682960A560E168002957
:1044500001D0491EE160F7F741FC70BD103C844279
:10446000EAD2D92303A20949002005F0FBFA70BD66
:104470007C2B00202E2E5C2E2E5C7574696C735C78
:10448000706F6F6C5F6275662E6300000000070737
:10449000F3B583B0F8F7B2FA4D4E7060009004980F
:1044A000010100980C1804983070F8F7A1FA8108FF
:1044B000706889000818A04212D2F8F799FA8008AB
:1044C000716880004018A04201D2012000E0002065
:1044D000482340A2454905F0C5FA002005B0F0BDCB
:1044E0000498411EC9B20491002868D0039800883E
:1044F000042803D200990420088009E0810705D030
:104500008107890F401A001D009900E0009908807A
:1045100003988578009885700398001D0390009893
:104520004460009884600098008880080190012D04
:1045300021D98700F8F75CFA80087168800040187C
:10454000A04212D2F8F754FA80087168800040182F
:10455000A04201D2012000E0002069231DA22349CE
:1045600005F080FA002005B0F0BD381920606D1EFE
:104570000446012DDED8F8F73BFA80087168800008
:104580004018A04212D2F8F733FA80087168800010
:104590004018A04201D2012000E0002073230DA2A8
:1045A000124905F05FFA002005B0F0BD0020206040
:1045B00001988000041900981030009075E7706829
:1045C000201AB060F8F7E6F9B06805B0F0BD000059
:1045D0007C2B00202E2E5C2E2E5C7574696C735C17
:1045E000706F6F6C5F6275662E63000000000407D9
:1045F00008494868C202424088684860C8688860C4
:104600000B68CB60D80C5840130A534058400860E0
:1046100070470000402C0020F0B4002939D01E4A19
:104620009368D768566815689C46F20272406646E1
:10463000BC462F46EB0C5D40130A53405D402A46B2
:1046400004290AD30270130A4370130C8370120EEC
:10465000091FC27089B2001D13E0002913D0431E48
:10466000CC0702D05A70120A5B1C4C0806D05A7054
:10467000120A9A70120A9B1C641EF8D14018491A3B
:1046800089B20029D1D104486146C76046600560FF
:104690008160F0BC70470000402C002070B5040021
:1046A00001D0012000E000205F230AA20F4905F09D
:1046B000D9F9F7F705FB25680146002D04D02868D5
:1046C0002060002800D160600846F7F707FB284605
:1046D00070BD00002E2E5C2E2E5C7574696C735CB0
:1046E0007871756575652E63000000000000020793
:1046F00070B50C46050001D0012000E000203C23ED
:104700000EA2144905F0AEF9002C01D0012000E002
:1047100000203D2309A2104905F0A4F900202060E3
:10472000F7F7CEFA2968002905D069680C606C603B
:10473000F7F7D4FA70BD2C60F9E700002E2E5C2E3E
:104740002E5C7574696C735C7871756575652E6324
:10475000000000000000020700000307F8B517463C
:104760000C46050001D0012000E00020384E9D23BA
:1047700031A2314605F076F9002C01D0012000E08D
:1047800000209E232CA2334905F06CF9F7F798FA24
:1047900000902868002802D06868B84222D1002D15
:1047A00001D0012000E000203C232B4A314605F0D7
:1047B00059F9002C01D0012000E000203D23264AB9
:1047C000244905F04FF900202060F7F779FA2968AD
:1047D000002905D069680C606C60F7F77FFA06E085
:1047E0002C60F9E7002F06D0386820603C60009804
:1047F000F7F774FAF8BD002D01D0012000E0002089
:104800007E23154A314605F02DF9002C01D00120F8
:1048100000E000207F23104A0E4905F023F9F7F746
:104820004FFA296821602968002900D16C602C604A
:10483000F7F754FADBE700002E2E5C2E2E5C757421
:10484000696C735C7871756575652E630000000096
:1048500000000207000003073C47010070B50D4649
:10486000040001D0012000E000207E230C4A0D4905
:1048700005F0F8F8002D01D0012000E000207F2392
:10488000074A094905F0EEF8F7F71AFA2168296096
:104890002168002900D165602560F7F71FFA70BD17
:1048A0003C470100000002070000030770B51646F0
:1048B0000C46050001D0012000E00020BF2310A21B
:1048C000154905F0CFF8002C01D0012000E00020B0
:1048D000C0230BA2114905F0C5F8F7F7F1F92968D3
:1048E000A14202D12168296003E0002E01D0216895
:1048F00031606968A14200D16E60F7F7EFF970BDD1
:104900002E2E5C2E2E5C7574696C735C78717565E7
:1049100075652E6300000000000002070000030719
:10492000801040B2704700000D4881B0C26B012179
:104930000A43C2630B4802680A43026042680A43A2
:1049400042600A2200210B4600930098401C009010
:104950000728FADB491C9142F6D301B070470000EA
:104960000000074040000740F0B42F4C2C4A246858
:104970002C4B002112681B68A508A6080846002DCC
:1049800012D0121FF50702D05168090E121D002522
:10499000E40808D057683F0E7918976808323F0E30
:1049A0007D19641EF6D14919204A126894089508A9
:1049B000002C14D01B1FEC0703D05C68240E2018B9
:1049C0001B1D0024D20809D05F68521E3F0E381804
:1049D0009F6808333F0E3C19002AF5D10019382290
:1049E0005643324638235D432B46423252090A363B
:1049F00052187409423361180A355B096C091B1897
:104A000024180B489B1C921C436002608A1C826025
:104A1000A21CC260074801814481F0BC70470000BD
:104A20000C2C00201C2C0020CC2B0020E02B002084
:104A300054960020642B002008B52B48C26B01213E
:104A40000A43C263294802680A43026042680A4373
:104A500042600A2200210B4600930098401C0090FF
:104A60000728FADB491C9142F6D300F087F820486A
:104A70000022006881081F48F6F7A4F813F05CF8DC
:104A8000002802D015F028FE06E01B48002200682E
:104A900081081A48F6F796F819480022006881083C
:104AA0001848F6F78FF81848C16A7F22920391439D
:104AB000C162C16AD2019143144A12889208520617
:104AC00012090A43C262816AFF2252019143104ACD
:104AD000127852010A438262816B0E4A090A1278E7
:104AE00009021143816308BD0000074040000740F0
:104AF00050EA020090E40200C82B0020B0E402005B
:104B000054EA0200A4E4020000040250DC2B00205E
:104B100061EA020060EA020010B511F01FFF0128EF
:104B200020D015F011FE022000F078F900200F4C83
:104B30000A2120716171A071E0710D492073886AAA
:104B40000C22904388620B480022006881080A48C2
:104B5000F6F738F8207BFFF76FFFFFF705FF12F03D
:104B60005DF810BD15F0DEFEDDE70000642B0020CF
:104B70000004025058EA0200A8E4020030B5934C49
:104B8000914821688A0819D04907914AC90F03D072
:104B900013681B680360001D23689B088B420DD9B6
:104BA00015688B00ED58056015685B195B684360FC
:104BB000236808309B08891C8B42F1D8854C2168FA
:104BC0008A0818D04907844AC90F02D013681B68A5
:104BD00008C023689B088B420DD915688B00ED58DF
:104BE000056015685B195B684360236808309B08A3
:104BF000891C8B42F1D8794C21688A0818D0490762
:104C0000774AC90F02D013681B6808C023689B0845
:104C10008B420DD915688B00ED58056015685B193E
:104C20005B684360236808309B08891C8B42F1D87D
:104C30006C4C21688A0818D049076B4AC90F02D00A
:104C400013681B6808C023689B088B420DD9156840
:104C50008B00ED58056015685B195B68436023683D
:104C600008309B08891C8B42F1D8604C21688A0867
:104C700018D049075E4AC90F02D013681B6808C0E4
:104C800023689B088B420DD915688B00ED58056091
:104C900015685B195B684360236808309B08891CB2
:104CA0008B42F1D8534A11688B0818D04907524BF0
:104CB000C90F02D01C68246810C01468A4088C4274
:104CC0000DD91D688C002D5905601D686419646834
:104CD000446014680830A408891C8C42F1D8474C01
:104CE00021688A0818D04907454AC90F02D01368BD
:104CF0001B6808C023689B088B420DD915688B0080
:104D0000ED58056015685B195B68436023680830DF
:104D10009B08891C8B42F1D83A4C21688A0818D02C
:104D20004907394AC90F02D013681B6808C02368B5
:104D30009B088B420DD915688B00ED5805601568EE
:104D40005B195B684360236808309B08891C8B42B1
:104D5000F1D82E4C21688A0818D049072C4AC90F6F
:104D600002D013681B6808C023689B088B420DD9CA
:104D700015688B00ED58056015685B195B6843602A
:104D8000236808309B08891C8B42F1D8214C21688C
:104D90008A0818D04907204AC90F02D013681B6837
:104DA00008C023689B088B420DD915688B00ED580D
:104DB000056015685B195B684360236808309B08D1
:104DC000891C8B42F1D830BD00100250DC2B002032
:104DD0002C2C0020F02B0020302C0020CC2B00208D
:104DE0000C2C0020D42B0020102C0020D02B0020D5
:104DF000142C0020E02B00201C2C0020E82B00208D
:104E0000202C0020E42B0020242C0020D82B002074
:104E1000182C0020EC2B0020282C0020044A916A3A
:104E20001F235B03C0069943800B084390627047C1
:104E300000040250F0B5D64D0446286885B000281D
:104E400005D18F239B00D3A2D84904F00BFED8488C
:104E50000390D8480490002C01DC641E64B2D6484C
:104E600044710168002901D020468847D349D448BD
:104E70000A78002A03D1826B9206120F0A703C2234
:104E8000092C0CDB09784B1D0F2B01D90F2100E0F9
:104E9000491D836B890093430B43836305E0836B58
:104EA0000978934389000B438363283464B212F07A
:104EB00043FE002808D00A2044430246A3B26946B4
:104EC000002012F03FFE07E00A204443BD480A22BA
:104ED00021186846F5F7DDFA6846BB4980888A687C
:104EE0008001BA4B1A4002438A606846C078C2000B
:104EF000B748016878239943114301606846807977
:104F000003990004084303900022012103A8F5F748
:104F100059FE6846C07904990005084304900022B0
:104F2000012104A8F5F74EFEAA4900200A68AA4903
:104F300093080AD093082A688400145B2404240E82
:104F40007A2C7DD0401C8342F6D8A44A00201268F7
:104F5000A34C93080AD0960822688300D35A1B04F6
:104F60001B0E7A2B6DD0401C8642F6D89D4A00203D
:104F7000126893080BD09C4E930832688600965BAB
:104F80003604360E7A2E7DD0401C8342F6D8974ADE
:104F9000002013689A080BD0954A9B081268860077
:104FA000965B3604360E7A2E6DD0401C8342F6D8BE
:104FB000904A00201668B3080BD08F4BB6081B68C8
:104FC0008700DF5B3F043F0E7A2F7DD0401C864276
:104FD000F6D869464878097A80004901084369464D
:104FE00089787C4B08431E680021844BB7080AD09F
:104FF0002D68B6088F00EF5B3F043F0E702F74D012
:10500000491C8E42F6D8754D00212D68AE080AD095
:105010002468AD088E00A65B3604360E702E6ED066
:10502000491C8D42F6D86F4C00212468A5080ED08B
:105030006D4EA50834688E00A65B3604360E01E07E
:105040004AE053E0702E76D0491C8D42F3D8674C6D
:1050500000212568AC080BD0654CAE0824688D0093
:10506000655B2D042D0E702D7CD0491C8E42F6D828
:1050700014680021A2080ED05F4AA50812688C00AF
:10508000145B01E03CE044E02404240E702C71D059
:10509000491C8D42F3D868464078594984006846D7
:1050A000007A096840010443684680780443002080
:1050B0008A080DD0534A8D08116882008A5A12045A
:1050C000120E702A5DD000E02CE0401C8542F4D81E
:1050D000FFF754FD05B0F0BD80006C4613582478EE
:1050E0008B436405234313502FE725E083006E466E
:1050F000D0583678884376053043D05036E722E0E2
:1051000080006E46135836788B4376053343135030
:105110003DE783006E46D0583678884376053043A5
:10512000D05045E786009859884369460978490573
:10513000084398514DE70EE089006E5807049E43DE
:105140003E436E505FE78900655806049D43354332
:10515000655068E706E08D006159060499433143C4
:10516000615174E78D0061590604994331436151DF
:105170007EE7FFE78C001159000499430143115168
:1051800089E780000A589A4323041A430A509FE78C
:105190000C2C00202E2E5C2E2E5C737461636B5CD5
:1051A00072665C72665F7068792E63001111EEEEB4
:1051B00012570000124E2000642B0020602B0020AC
:1051C000000007407CE10200400003403F00FFFF79
:1051D00040000740CC2B00200000E000D02B002036
:1051E000142C0020D42B0020102C0020D82B0020C1
:1051F000182C0020FC2B00203C2C00200000ED008F
:10520000DC2B00202C2C0020F8B5164D0F466C68C6
:105210000646002C24D0F6F753FD009068684068DD
:1052200068600020A66060752775E0750120E06069
:105230000421F4602161A9686160AC60092F02D18A
:105240002036F17861752969491C296106490A7B74
:10525000002A00D1087300F0E5FC0098F6F73EFD47
:10526000F8BD00003C2B002034960020F0B5D84D4E
:105270008FB0E868002871D0D64AD168C900490CBF
:105280000191D268520F0492D34A536A0693D34BCA
:105290001B691B06DC17037D641C012B0CD0022B41
:1052A0002FD0032B41D0042B6ED18468607F01285E
:1052B0006AD000286AD06CE08668B7693F1D002973
:1052C00012D0002C10D00698F5F7F2FB316C401884
:1052D0003064C3480368002B06D07A783946121D23
:1052E000E8689847002808D1BD48C268002A04D061
:1052F000E86800218068904765E10020F5F7EAFB47
:1053000061E1491E8568012908D8002C06D0B449FE
:105310004B68002B02D0012201A99847B0480269CE
:10532000002A31D0022128462DE086680120400263
:10533000FDF7CCF9E868C17D002910D080363069CE
:105340004268002A02D00021117641605830FEF7F1
:105350006BFFA3480269002ACAD134E114E0019925
:1053600000290AD0002C08D09D498B68002B04D05E
:1053700000221146984700287ED199480269002AE8
:1053800002D00221304690470FB0F0BDE07E0028E9
:10539000FAD09148C06AC003400EFEF77BFF02902E
:1053A000002003900198002804D00698F5F780FBB0
:1053B000A16A4018A06200200C90019800287DD0BE
:1053C000E16A1022491CE162216A11432162090449
:1053D00075D4844900260B91002869D92046FF30F6
:1053E0004D300D900C3808900B98002806D0417A6B
:1053F000827A114042680068514308180546071D2B
:105400000079B8707978F970002910D001200C90DB
:105410000898407E002800D001208000C01D081898
:10542000800880003858FFF77BFAA07603E07868A0
:10543000FFF776FAA0767878002809D00398401C08
:1054400003900898407E002802D0F878001FF8707A
:105450006548FF210068D131201AF4F789FF2870D0
:10546000000A68700020A8700199701CAD1C884269
:1054700014D10898407E00E0A5E000280ED00299E3
:105480000398814206D1002808D00D98026851186F
:10549000016003E0002801D03D2028700B9800280F
:1054A00002D0417A491C41720198761C86429BD3F6
:1054B0002046FF30A1300178019A01E029E01BE08D
:1054C0005140C907C90F01701020FDF7FFF80C9873
:1054D000002811D0FF205A30005D00280CD043482E
:1054E0000068807F002807D03E481121006A0842EA
:1054F00002D02046FEF738F9A08E01994018A08608
:105500005420015B0A2041432046FF305D30FEF706
:10551000E7FD0498002844D001462046FF30813042
:105520004177C27F04994A40D107C90FC177216AE8
:10553000480702D50498401E04902046FF30A13051
:1055400082780079101A049A904200D91046FF22FE
:105550005A32125D002A07D0C90305D42146FF3113
:1055600031310A6812180A60002802D04020FDF785
:10557000ADF8FF20CB30005D002809D01A48FF218C
:105580000068D131201AF4F7F3FE80B2FBF786FDF4
:105590005420015B0A2041432046FF305D30FEF776
:1055A0009FFD0D48826804210A43826082688A4315
:1055B00082600021C1620A484169002903D0044881
:1055C000C0688068884700F02DFB0FB0F0BD000078
:1055D0003C2B00200008025040040250800802507A
:1055E0001496002010990020242B0020282B002046
:1055F0001848C06800282BD010B5017D0A2910D2A8
:105600000A007A441279921897440B040C0C140B7C
:105610000B0B0B1B1049CA68002A02D080680121BD
:10562000904710BD0C490A69002A0ED080680021FD
:1056300090470AE008494969002906D080688847F0
:1056400003E005490A6A002AF0D100F0EBFA10BD28
:10565000704700003C2B00201496002070B53A4C97
:105660002068002800D001206E2338A2404904F0B1
:10567000F9F9402200213F48F5F70EFAF7F7BEF995
:105680000646F7F7B5F901463046B20702D0B00832
:105690008000001D384D28602268D37B147C1B19C4
:1056A000547AD27FA2189C181822A41C62431018A6
:1056B000861B8E4207D93148711A0143842323A2E5
:1056C000002004F0CFF93046F7F764F900210A46CC
:1056D000012C36D00020641E002C09DD2E68182114
:1056E00041438B1919461831401C5960A042F6DB22
:1056F0004A602868AA60EA602A61686020482149F7
:105700000273CB7843750B7983754B79C3758B79AD
:105710000376CB7943760B7A83760B7883734D7857
:10572000C5738C78047443748374C57404754B7AA0
:10573000C3768B7A0377C97A417713480260426057
:1057400070BD28684260D4E7282B00202E2E5C2EE6
:105750002E5C737461636B5C636F6E74726F6C6CE0
:1057600065725C7363685F6D61696E2E6300000033
:1057700000000209149600203C2B002000000702C4
:1057800034960020FC2A0020502B0020F3B52C4832
:1057900081B00068019900288C6815D085681920AF
:1057A0008001F5F785F90146AA6828680126801A64
:1057B0006268411A511AB607B1420AD920480199C4
:1057C000FFF74CF803B0F0BD1D48FFF747F803B0F2
:1057D000F0BDA3682168C91A6B68CB1AB342F6D929
:1057E000821AB242F3D9081AB042F0D919208001C6
:1057F000F5F75EF9AA682968891A0F1A4B20C000CC
:10580000F5F756F902994018391AB14201D9C71B68
:1058100000E00F46C820F5F74BF922686168891A45
:105820004618B742D3D919208001F5F741F9AA6883
:105830002968891A081A801B206080196060BDE7FA
:10584000502B0020F8B50446F6F73AFA00901748B6
:105850000568A368002D0ED0A9685E688A6808688C
:10586000821A0120B71A800787420AD921460F48B9
:10587000FEF7F4FF15E0002221460C48FEF76EFF0C
:105880000FE01F689B684968FB1A591A814202D9C8
:10589000911B814201D8964203D1607D697D884287
:1058A000E4D80098F6F71AFAF8BD0000502B002053
:1058B00010B51F48C068017D0A2935D20A007A4414
:1058C000127992189744300410171C303030302170
:1058D000816820310A78012A26D1C07D002825D090
:1058E0004878002821D021E08068007F01281BD162
:1058F000FFF77EFE18E08068007F012815D013E0D6
:105900008068407F002811D00EE0816820314A78FD
:10591000012A09D1C07D002808D00020487088786D
:10592000002801D0F5F794F8002010BD012010BD2B
:105930003C2B00200F280ED202007A4412799218D4
:10594000974407090A0909090D10130916091909CD
:105950001C000C48C16070470A4801617047094843
:10596000416170470748016270470648016070470F
:1059700004484160704703488160704701484162B4
:10598000704700001496002070B50125C468F6F732
:1059900097F906461C480121C06800282BD0002C2E
:1059A0002DD0A04204D1227D022A0CD0012A0AD097
:1059B000A04202D1227D092A19D0A0421DD0204642
:1059C00000F0A8F81BE0E17500F02CF9207D01281B
:1059D00008D10E480078002804D03046F6F77EF94A
:1059E000002070BD3046F6F779F9012070BDE175F1
:1059F00000F018F9F6E7002C01D0E17500253046DB
:105A0000F6F76CF9284670BD3C2B00205099002019
:105A1000F8B53D4EB568002D75D0F6F751F90090F8
:105A20006C680027002C33D0E07D00282CD0E7756F
:105A3000207D012804D0032808D0042818D109E0CB
:105A400032480770A0682030477011E00820FCF74A
:105A50003DFE0DE0A06800280AD00246FF328132E8
:105A6000D168002904D09179082901D1F9F7CAFB3E
:105A7000606868607068606074603069002801D098
:105A8000401E30616C6801E025466468002CCBD173
:105A9000B068002830D0C17D002931D0C775017DA4
:105AA000012904D0032908D0042918D109E0174995
:105AB0000F7080682030477011E00820FCF706FE68
:105AC0000DE0806800280AD00146FF318131CA68A4
:105AD000002A04D08979082901D1F9F793FBB0682D
:105AE0004168B1607268426070603069002801D01E
:105AF000401E3061002903D10548F7600773376104
:105B00000098F6F7EBF8F8BD3C2B002050990020E8
:105B100034960020F8B5194E0500B7682CD038002F
:105B20002AD0F6F7CDF8B168A94208D16968B1600A
:105B3000716869607560316900290DD113E07C6876
:105B4000002C10D0AC420AD1616879607168616044
:105B500074603169002906D0491E316103E027468F
:105B60006468002CEED1B168002903D1044AF160C9
:105B700011733161F6F7B2F8F8BD00003C2B00203C
:105B80003496002070B5F6F79BF822490646CA689D
:105B900020200243CA60C868402290430024C860A5
:105BA000CA6810200243CA60CA688243CA601A4B9E
:105BB0009968002913D05A68087D042802D0092862
:105BC00003D005E08868047602E08D6820352C70EB
:105BD00048684A600A46011EEED15A6099601C610D
:105BE0000E48DC600473F4F733FF0020F4F766FF1F
:105BF0000120F4F769FF0A480C2142690A43426117
:105C000042698A43426182690A4382613046F6F7FB
:105C100065F870BD000002503C2B00203496002037
:105C200080080250F0B58FB0F6F74AF8FD4D0890A5
:105C3000E868002808D0FFF73BFE002804D0089849
:105C4000F6F74CF80FB0F0BDFFF7E2FEA868F64E8D
:105C5000F64C002830D00120F4F7BAFF0120C00232
:105C600030602046C26810210A43C260C2688A437D
:105C7000C260C26840218A430021C260406901902D
:105C8000EB48016041601438EA4AC160116051601C
:105C90008468029106910791002C6FD04B20C000C0
:105CA000019DF4F705FF4619207D01281BD004282B
:105CB00047D0092844D16DE00120C0023060E1687E
:105CC00010200143E160E1688143E160E168202048
:105CD0000143E160E06840218843E0600898F5F7FF
:105CE000FDFF0FB0F0BDA5682968A868081A811BE0
:105CF0000120800781421AD90127CF48296B4143EF
:105D00002846F4F7CFFE6775A9682868401A811BFA
:105D1000012080078142F0D82220405D012806D072
:105D2000FEF766FCC104C90C2846F4F7BBFE2A2026
:105D3000405D696B4843F4F7BBFE29684018686012
:105D400042E0A5680127A9682868BF07401A801BA0
:105D5000B84239D900212846F4F7D4FE607D0628E0
:105D600011D2697E002907D001214018C0B26075A8
:105D7000697E002903D006E00221F6E78DE00628BF
:105D800001D906206075A9682868401A801BB842AE
:105D9000E0D819E0A06882680168891A0122891B8D
:105DA0009207914210D9617D062901D2491C617583
:105DB00043690168C9180160C369CB1843608368EF
:105DC000C91A891B9142EED8E07D002803D001203A
:105DD0000790646853E0207D042803D002990029CD
:105DE00032D035E0F5F76CFF0D9091480268A3685A
:105DF000002A0FD09568A9682868411A5868074694
:105E0000461A0120800786420AD921468848FEF7B3
:105E100025FD15E0002221468548FEF79FFC0FE096
:105E20001E689B686D68F31A5B1B834202D9CB1B0B
:105E3000834201D88F4203D1617D507D8142E4D8F5
:105E40000D98F5F74BFF19E0012805D0052803D080
:105E50000699002902D005E002940FE0022804D040
:105E6000032802D0092802D008E0069406E073480F
:105E7000426A002A02D02046019990476468002CAB
:105E800000D00BE70798002801D0FFF7C1FD02986A
:105E9000002802D00199FFF779FC664800680028C5
:105EA00002D00199FFF7CEFC614800685D49644E5D
:105EB000C8606449099100287ED080680A900698DD
:105EC00000287AD084685C4920680790E08C4843B9
:105ED000F4F7EEFD2168451830466560F4F7E8FDFB
:105EE00001994618A08C544948430390E08C4843DC
:105EF000F4F7DEFD274620370B900BE02046039990
:105F0000F4F7D0FD20680B99451865607978491C35
:105F1000797007900120A91B80078142EED8B54215
:105F2000ECD04B20C000079EF4F7C2FD0199401849
:105F3000311A01208007814206D94B20C000F4F7B6
:105F4000B7FD0199401807900A98076886681920DC
:105F50008001F4F7ADFDB91B4B270E1AFF00384640
:105F6000F4F7A6FD01994018811B012080078142AA
:105F70006ED9A91B81420FD93846F4F799FD0199D2
:105F800040182E1A3048F4F793FD864273D96560A5
:105F900024490698C8606EE04B20C000F4F788FDE5
:105FA000014601980818351A2848F4F781FD854202
:105FB00061D30798371A01E019E072E00125AD07B7
:105FC000AF4258D87D200001F4F772FDB84252D894
:105FD0004B20C000F4F76CFD014601980818801BA7
:105FE000A84248D966600F490698C86043E0069801
:105FF00000284BD00B49C860069884683046F4F7F7
:1060000057FD01994718A08C0B4948430190E08C3B
:106010004843F4F74DFD216806468819254620358A
:10602000606020E03C2B002080E200E00000025095
:10603000502B0020582B00207102000014960020E5
:106040003408000034960020DC050000B80B000086
:1060500011E020460199F4F725FD20688019606061
:106060006878401C687060680121C21B89078A42F9
:10607000EFD8B842EDD05F48C068002806D0069936
:1060800000290ED0884209D1012008E0099900209A
:1060900008730898F5F722FE0FB0F0BD0020F4F762
:1060A00055FD5548416953480024C068C160007DD2
:1060B0000A284AD201007944097949188F444504D5
:1060C00010102145454545384A480021C068202226
:1060D0004175806801211154016880680C1A3EE006
:1060E00044490020C96801224875069880680277F3
:1060F000446842480269002A31D0886801219047EB
:106100002DE03C480121C068417581688B680A68B0
:10611000D41A00224A7739498C62016900291ED0BD
:1061200002291CD8491E016119D10421016116E020
:106130003048C168886802462032D3784B750168C0
:1061400080680C1A0120507009E00998007B012832
:1061500005D12B4B2BA23449002003F083FC264EA3
:1061600075697003671B874205D9291B2F4B25A230
:10617000002003F077FC01208007874200D92F1B05
:10618000032F01D87469241DF1684025A943F160EB
:10619000B461F1682846A9430843F060F168202003
:1061A0008143F160224980010860B069A04205D0B6
:1061B000204B14A22049002003F054FCF068202159
:1061C000084205D01D4B0FA21D49002003F04AFCD8
:1061D000F068284205D11B4B0AA21B49002003F09E
:1061E00041FC0020F4F7F4FC0898F5F777FD0FB0B8
:1061F000F0BD00003C2B002000000250149600204F
:106200009D0400002E2E5C2E2E5C737461636B5C0B
:10621000636F6E74726F6C6C65725C7363685F6DD4
:1062200061696E2E6300000000000109A5040000F2
:1062300000E100E0B9040000BBBBFFFFBE040000AA
:10624000CCBBFFFFC3040000DDBBFFFF10B500F0B7
:1062500001F810BD10B5024800F010F810BD0000A4
:106260003025002010B500F001F810BD10B502482F
:1062700000F004F810BD00006425002010B501688E
:106280000446C8690122C007C00F002803D0086A6D
:106290001043086210BDC8690422104226D0C868A5
:1062A000400723D520688168608B62694300D2185B
:1062B000401C60831180618B208B814212D3236A42
:1062C0002046002B03D0428B10206169984721683B
:1062D000042248699043486122680221506988433A
:1062E000506103E02068C0684007DBD421680222C7
:1062F000C869104226D0C868400723D52068816845
:10630000608B62694300D218401C60831180618BEE
:10631000208B814212D3236A2046002B03D0428B6C
:106320001020616998472068042142698A434261CC
:106330002168022248699043486103E02068C068F0
:106340004007DBD420680821C2690A42A2D0C06895
:10635000800737D5608A218A884217D2608A2168EF
:10636000E2684300D218401C608210888860206870
:10637000C16849070AD5A17A112907D18168608BC4
:1063800062694300D218401C60831180618A208AB0
:10639000814213D32079002803D12068C168C9063F
:1063A000FCD4636A002B03D0628A1020E16898470E
:1063B0002268082150698843506103E02068C06862
:1063C0008007C7D4A07A012800D063E72068C1689D
:1063D0004907FAD58168C1684907FBD410BD7047E9
:1063E000401E0AD300BF00BF00BF00BF00BF00BFF8
:1063F00000BF00BF00BF401EF4D270470349CA6F00
:106400009207D217521CFAD1086070470030004042
:106410000168074802684A40026042684A40426098
:1064200082684A408260C2685140C1607047000083
:10643000402C0020F8B51F4D28780A2801D90A20E1
:10644000287064211C48F4F74CF81B4C5520207030
:10645000AA20607028788100891CA1701749E0701B
:1064600042000F46201DF4F714F828781449420022
:1064700010190E46001DF4F70CF8287866218200EA
:1064800010190171BB2141717D23DB0021460D48AC
:10649000921DF6F7F1F90020287064213846F4F7D0
:1064A00020F864210848F4F71CF864213046F4F71A
:1064B00018F8F8BDF68F0020928F00202A90002057
:1064C0005691002028260020EC91002010B510489D
:1064D00041690904090F0ED0491C42690D4C92050F
:1064E00010D5806A04221040042806D00A48F3F729
:1064F00029FF606010BD0121EFE70848F3F722FF94
:10650000606010BD0648F3F71DFF606010BD00001D
:10651000000004401C250020006CDC020090D00329
:106520000048E801F8B50546FF2701372B463B2216
:106530000021A5480097F5F745FE2846AA7F1E30A2
:10654000002113462E244678B2188678801C7118D4
:10655000D2B2C9B2641EF6D1501829466031CA7E43
:10656000C0B282427ED1C87D022812D32031087881
:1065700000223F244E7830188E78891CB218C0B2A1
:10658000D2B2641EF6D1FF218018495DC0B28142AB
:1065900075D18E49086A8E4A2C4610405A07920ED1
:1065A00010432034A27A5206520F1204104308629C
:1065B000486A884A104022781207520E1043A27986
:1065C0005207520A10434862886A834A104022796F
:1065D0001207D20E1043A2781207D20A1043886223
:1065E000C86A237A78221B0790435B0E1843C8625F
:1065F0007A480368267A93433609F60033430360EA
:106600000B6B667A93433607760E33430B63CB6B83
:10661000667A93433609F6003343CB63416891436E
:10662000A27A1207520E11434160C168E27AC9088A
:10663000C9005207520F1143C160694FF969FF2227
:1066400012029143E27C12021143F961B969654A71
:106650001140227E1207120E1143627E1202114374
:10666000B96100E00BE02A464032117DCE064B09AD
:10667000F60E5B01361D1F2E0AD91F2109E05A496B
:106680000020087039462846F3F72BFF0020F8BD9C
:10669000091DC906C90E0B431375016901235B056A
:1066A0009943937DDB079B0A1943016147498B6B33
:1066B0004E4E3340967DF606360FB6003343167DB8
:1066C000527DF606B60CD2063343520B13438B634E
:1066D000826813022A46603216791B0A3606334353
:1066E0008360D37D022B1FD3042B08D2237E072681
:1066F000F341012676079B191926F34123768B6A0D
:1067000007267605B343267E7606760F7605334355
:106710008B62066901231B061E430661D07D072894
:1067200002D3886A18438862D07D062836D3086A67
:1067300006229043227C9209520010430862386A74
:1067400070218843A17B4907490E08433862786A63
:10675000012189028843A17B0907C90F89020843E7
:106760007862F86930218843A17B8906890F090185
:106770000843F861B96A1E480140E07B4206920F67
:1067800012011143C206920F920140071143400DBE
:106790000143A07B8009C0020143B9622846F4F797
:1067A00077FA2846FDF7FEFD2846F5F703FD064C6F
:1067B0002046F5F7E3FC2046F5F7BAFC2046F5F74E
:1067C000A3FD0120F8BD00000000054000000740C7
:1067D000C7FFF8FF87FF8FFFE1FFE1FF40000740A1
:1067E000000004400F00FFFF1C250020C301F8FF3C
:1067F0000FE0FFFF70B51B480025C5611A4CE06A29
:106800000F2109048843E062184E2A4602213046CF
:10681000F5F7CAFD02213046F6F7FCF9F5F706F95F
:106820001348816B3C229143124A114349084900A5
:10683000816311490D61616A3F22120191436162D6
:10684000416B4908490041630C490A6810239A4387
:106850000A60016A062211430162206A702108431E
:10686000206270BD40000740000004400000054069
:1068700000000740180000020000084080010240AC
:1068800070B50446006881680125C907002903D056
:106890008560E16A0120884720688169C907C90FBE
:1068A00003D08561E16A022088472168104A0E23DF
:1068B00002268868914201D1184000E0304000284B
:1068C00014D08868914201D1184000E030408860BF
:1068D00020688168904201D1702200E004221140BA
:1068E000816020688560E16A0320884770BD0000F0
:1068F0000080004010B500F001F810BD10B502484E
:10690000FFF7BEFF10BD00009825002010B500F075
:1069100001F810BD10B50248FFF7B2FF10BD00002E
:10692000C825002010B500F001F810BD10B50248D0
:10693000FFF7A6FF10BD0000F8250020002904D0B5
:106940000269120E12060A4302617047014908608B
:1069500070470000982B002010B500F001F810BD22
:1069600010B5024800F010F810BD000028260020E5
:1069700010B500F001F810BD10B5024800F004F8A1
:1069800010BD00005C26002070B501688A681307FE
:1069900002461B0F2032042B37D00CDC012B5AD0BF
:1069A000022B0FD1137A002B0CD0C96F8907C9179E
:1069B000491C2CD03DE0062B05D00C2B02D10C211C
:1069C00000F04DF870BD04464869C505507AED0DDC
:1069D0000028F7D06669002EF4D0680704D5E38C50
:1069E00004212046226AB047280705D5E38C666952
:1069F00005212046226AB047A807E3D5E38C6569E4
:106A000006212046226AA84770BD0421D8E7C38B1F
:106A1000818B8B420DD2C18B036884696418491C39
:106A2000C183217819600168C96F8907C917491C9A
:106A3000EDD0C18B838B9942E6D101684B6802246B
:106A4000A3434B60002111724469002CDCD0C38B3E
:106A50008269A04770BD012100F001F870BD70B5DA
:106A600004462030427A002A5BD0257C0022042391
:106A7000002D57D00C2972B60BD113E0E18CA28CFB
:106A800091420DD20168E08C226A1218401CE08409
:106A90001170206884210958C906C90E0129EDD852
:106AA00062B632E02168C96F0907C917491C11D1C4
:106AB000E18CA58CA9420DD221680D68E18C266A73
:106AC0007618491CE18435702168C96F0907C91718
:106AD000491CEDD062B62168CD6F2D07ED176D1CF6
:106AE00013D04D686D086D004D6021684D689D4361
:106AF0004D6072B64272227462B66569002D04D090
:106B0000E38C02212046226AA847E08CA18C8842AF
:106B100007D36569002D04D0E38C03212046226A47
:106B2000A84770BD72B62168C96F0907C917491C0B
:106B300011D1E18CA58CA9420DD221680D68E18CA0
:106B4000266A7618491CE18435702168C96F0907E7
:106B5000C917491CEDD062B6E18CA58CA942E0D1E1
:106B600021684D686D086D004D6021684D689D433A
:106B70004D6072B6427262B66569002DD1D0E38C69
:106B800001212046226AA84770BDF8B50D4604468B
:106B9000F4F776FEE268002180263243E2602A683C
:106BA0000B4697001922F3F727FC3A460023F3F728
:106BB000F3FB0746642801D20020F8BD6421F3F7F7
:106BC000C1FBC1B221600104090E61606421484328
:106BD000381A00013230F3F7B5FBC0210851E068E4
:106BE000B043E060E0688109287989010843E060EA
:106BF0000120F8BD0170090A4170704770B41C068D
:106C0000110A2143027041701D04110C2943817047
:106C10001E02110E31431C0AC1701D0C0371447118
:106C20001A0E8571C27170BC704710B500F002F881
:106C300010BD0000054801680822114301600448A6
:106C40000068002800D00047704700000060004046
:106C50009026002010B500F001F810BD0449012075
:106C6000886004480068002800D000477047000092
:106C700000700040942600200FB410B503A9044B07
:106C8000044A029800F0D6FE10BC08BC04B01847B5
:106C9000D16F0200502C00200FB410B504A9074B8F
:106CA00002AA039800F0C6FE044602A9002001F0E3
:106CB0004EFB204610BC08BC04B018474F830100AF
:106CC00010B5024B024A00F0B5FE10BDD16F0200B4
:106CD000502C00202021020C01D010211046020A65
:106CE00001D010460839020901D01046091F820858
:106CF00001D01046891E420801D0881E7047081A2C
:106D00007047F0B4040C8BB2264682B25E430D0C81
:106D10001046370C58433604801900217941164635
:106D20006E43370C36048019794126466E43891923
:106D3000F0BC70470021017041708170C170017119
:106D400041717047002101804180818070470A783D
:106D500002704B7843708A788270CA78C2700B795F
:106D600003714A79427170470A7802704B78437018
:106D70008A788270CA78C2700B7903714A7942713D
:106D80008A798271CB79C37170470A6802608B88F7
:106D900083808A7982717047C9B20A0211430A045A
:106DA000114301604160704702E008C8121F08C12A
:106DB000002AFAD170477047002001E001C1121F7C
:106DC000002AFBD17047000010B584B0002903D021
:106DD00004682468646900E0094C0093019402ABE4
:106DE00010F0E4FE002804D16846007A002802D0A2
:106DF000002004B010BD0120C00704B010BD000089
:106E0000A97B020010B5044641680068006802686A
:106E10009047E17BC90704D1A17BFA2901D0FB2966
:106E200009D1C106C90E1A2901D01B2903D1C007F7
:106E300003D01B2909D001F0A6FA20686168006818
:106E4000491C82689047002110BD20686168006875
:106E5000491CC268904710BD10B51C4613468C42B1
:106E600005D822461946F3F714FB204610BD002032
:106E700010BD4100C0091B2250434140C8B27047B9
:106E8000F0B51FB486B00998089A030D002102439B
:106E900014D05148514A181850430514119801282C
:106EA00010981AD0281A401C00264D4F4D490096C4
:106EB00001910490002812DA444211E01198012453
:106EC00049A3012801D11098C1430698119A846002
:106ED0000360C26041600BB0F0BD4042E4E704468D
:106EE000210500203F4A001C51410391029012E00D
:106EF000E00707D032463B4601990098F3F7CCFBF8
:106F00000191009032463B4610461946F3F7C4FB08
:106F100006460F466410002CEAD10498039B002813
:106F2000029A0999089806DAF3F7B6FB019B009AD2
:106F3000F3F7B2FB05E0F3F717FC019B009AF3F7B8
:106F400013FC04460E460022284BF3F729FD03D814
:106F50000020C043014607E00022254B2046314671
:106F6000F3F7E8FAF3F7FCFC102409E0002C0ADB45
:106F70000A220023F3F710FA079B30321A55641ED9
:106F800002460A43F2D11122641C079B121B1C19F2
:106F9000119B012B03D0012308430ED10AE00843C3
:106FA00004D0112010900020119077E71098151A46
:106FB0006D1E0BE01098824202DD00236D1C03E081
:106FC000824201DA00236D1E002BEED00698119943
:106FD0008260C16030C07EE701FCFFFF104D000001
:106FE000000014400000F03F300000000000F043BB
:106FF0000000E03FFFB583B00C9E1546040000D1B1
:1070000001BE00200290E0693268801AA2690191F5
:1070100080180090002D2BD03768AF4200D32F4648
:107020003A4601990098F3F734FA3068ED1BC11B1A
:1070300031600098C01900900198C0190190002992
:1070400014D10698A7680168B8697F68A369E269E6
:10705000B8470290002830D1E0693060A069009004
:107060000698E1690068411806980160002DD3D1A7
:107070003168E06981421FD00D9800281CD0069825
:107080000168A0688369026918469047E16932681F
:1070900005468A1A0146501EF3F754F9421C6A430A
:1070A0000698A5680168A8696D68A369A847029059
:1070B000002802D1E0693060029807B0F0BD0000FE
:1070C00030B4002916DD0D4C03781B025A4004230E
:1070D000401C150402D55200624000E05200150425
:1070E00002D55200624000E052005B1EF1D1491E01
:1070F0000029E9DC30BC90B270470000211000008C
:10710000FFB589B01F461646050000D101BE1B4CD5
:107110000A98F3F7FBF90146194A0A98FFF7D0FFDE
:107120003880002030602969002924D93168E86856
:10713000C900411808884A68398880B2814214D34E
:10714000814201D90D4C16E000230A980121129CBE
:10715000029300900394019104AB2846296E00F03D
:1071600029F906490446884205D13068401C306040
:1071700029698842DAD320460DB0F0BD05004209E6
:10718000FFFF0000F3B593B0040000D101BE1498D6
:1071900000280DD0C06800280AD01498216F4068DC
:1071A000091A1498806808186168490881426CD3EC
:1071B000A068656E8269436929461046984706466D
:1071C00060684008B04207D9A368821B98699B6831
:1071D000A9199847002806D1A068324683698768B4
:1071E00029461846B847002850D17048656E006897
:1071F000F3F78CF9A16806460A6988692946904721
:107200000546304617302946F3F79CF8411C694380
:10721000002005910F90206900286AD91498002851
:1072200003D001680F9881425DD00F98E168C000DB
:10723000001D10900858626E216E059E002C00D132
:1072400001BE08180B9090191190A16814220D68C6
:10725000886906AB0B99A847002817D16846A26831
:10726000078C90691269099D0B999047014601901E
:1072700078191330F3F766F80199451C4D437019DE
:107280000D9061684908884202D9494815B0F0BD9F
:107290000B98039011980190002D1ED0E669AE4224
:1072A00000D32E46A168A3690F6888693246039906
:1072B000B8470028EAD1A168A3694F6888693246B7
:1072C0000199B8470028E1D10398AD1B80190390BC
:1072D000019880190190002DE0D1E368109A05997A
:1072E0000D98995005900F98401C0F90216981428C
:1072F00094D814980025002834D0C068002821D0E4
:10730000149909AB09680991818968460185059836
:1073100014990B90C86802268268091D029603938F
:1073200001920491416800910368616E2046059ABC
:1073300000F0BEF90028A9D11498816805980818B2
:1073400005900FE000951498019502950068009053
:107350006A460121204600F068F91498216F4068C0
:10736000081A206721464031888D401C80B28885EC
:10737000616E002C00D101BE6A4655841084042041
:10738000019008A8009009480295039504950368A8
:107390000022204600F08CF900288BD10599A166C7
:1073A000626E216E2266616615B0F0BD1C2A002057
:1073B00006004209F0B58BB01D46040000D101BEA5
:1073C0000020C0438E186B4614229880002D00D1F7
:1073D00001BEA1682B460F6888693146B84700286E
:1073E00019D12868411C18D0002816D0804988423D
:1073F0006FD1288900286CD040286AD212980028C2
:107400000ED0139800280BD00168E868814207D29B
:107410001399086077480BB0F0BD77480BB0F0BD0A
:1074200069468A8804212846FFF74AFE0246012160
:10743000281DFFF745FE02460121681DFFF740FEAB
:1074400002460221A81DFFF73BFE02462846022104
:107450000830FFF735FE0246284604210C30FFF7BE
:107460002FFE69468880E8888019059010980028CA
:1074700043D0119800282DD00598029010980690BE
:107480002E89002C00D101BEF3F740F8B04202D0A3
:107490005A480BB0F0BD002E25D0E069B04200D3B1
:1074A00030460090A168A3690F688869009A029924
:1074B000B8470028EDD1A169009A0698F3F72DF896
:1074C0000028E5D10099029840180290761AE4D17C
:1074D00009E082E0A1682A890E688869109B0599F5
:1074E000B0470028D5D16846828829891098FFF7CF
:1074F000E7FD01466846818027E0059804902E89C3
:1075000001A80A90002C00D101BE002E1DD0E06918
:10751000B04200D330460090A168A3690F68886923
:10752000009A0499B8470028B3D10A9800990288B4
:10753000A069FFF7C5FD01460A98018004990098EB
:10754000081804900098361AE1D12989059809187D
:107550001298002814D01398002811D0A368EA6864
:107560001C689869129BA047070092D168468288E0
:10757000E9681298FFF7A4FD01466846818027E07C
:10758000029101A8EE680990002C00D101BE0027ED
:10759000002E1DD0E069B04200D330460090A168B3
:1075A000A3690F688869009A0299B847070099D1C2
:1075B000099800990288A069FFF782FD01460998A1
:1075C000018002990098081802900098361AE1D1BB
:1075D000694689882869884202D009480BB0F0BD05
:1075E0001398002801D0E968016038460BB0F0BD5F
:1075F000CEFACEFA0700420904004209050042090A
:107600000300420910B574300DD0017900680029DB
:1076100002D015F099FB04E000231A46194615F034
:10762000F9F9002800D101BE10BD70B51546044619
:1076300000291AD0012903D002292DD001BE70BD26
:1076400029682069814200D301BE401E2061116873
:107650008142F4D2401AC200C8000146E3680831F2
:1076600059181818F2F715FF70BD21696069814239
:1076700000D301BE2868884200D901BE884208D2E2
:10768000091AE368CA00C000191808301818F2F780
:1076900000FF2069401C20612A68E168A888D200A8
:1076A00088522868E268C000A968001D115070BDAA
:1076B000FFB58DB01A9D16460F46040000D101BEDD
:1076C0001098002800D101BEB919142007910C9020
:1076D000A2689069126990470146E069142800D2B7
:1076E00001BE4A1E174200D001BEF2F72BFE002950
:1076F00000D001BE169800901798109F0A9002A81B
:1077000018990890002F00D101BE00205C4A029217
:1077100003900490059006906A4610731420D0815F
:1077200001290FD0002050733846F2F7EFFE69466A
:1077300008820A9805900898009909970891002FE7
:1077400002D002E08020EEE701BE4E4A0746042147
:10775000FFF7B6FC02460121381DFFF7B1FC0246D7
:107760000121781DFFF7ACFC02460221B81DFFF78E
:10777000A7FC0246384602210830FFF7A1FC02466A
:10778000384604210C30FFF79BFC02466846018A0C
:107790000998FFF795FC02460898002807D005983D
:1077A000002804D001460898FFF78AFC024606929A
:1077B0006846008A0890A268079990691269059F37
:1077C0009047014600900898C0191330F2F7BAFDAF
:1077D0000099401C4843616830184908884200D924
:1077E00001BEE0690B900BA80027009007AB019742
:1077F00002A920460C9AFFF7FDFB00282DD1384640
:1078000001900BAF00976846028A07AB204610999B
:10781000FFF7F0FB002820D101200097019007AB73
:107820002046059A1699FFF7E5FB070015D1002EB3
:1078300012D01998002801D0002D00D101BE0246B7
:1078400020461899FFF7F1FE1898002812D0012859
:1078500005D0022807D001BE384611B0F0BD206F18
:107860002968401A04E0206F2968401A69684018A6
:107870002067F1E7206F696840182067ECE7000097
:10788000CEFACEFAFFFF0000FFB599B0229D0400AA
:1078900000D101BE0020139013A8009008AB12AADB
:1078A00020461A99FFF72CFC5F49002803D0884234
:1078B00007D1002000E0012029460190814302D039
:1078C00000201DB0F0BD002D01D0012619E00028D8
:1078D00001D0022615E0216960690026814210D39B
:1078E0004700F80013F04EFD05003CD06069E168E8
:1078F000C2002846F2F7CDFDE06814F02FFE676164
:10790000E560276E1A98F2F701FE0090A0681C9DB2
:107910008369026939461846904701460746009830
:1079200040191330F2F70EFD401C78430546002E37
:107930001CD0206E0A901A98F2F7E8FD0390A16817
:10794000139F0A6988690A99904701460090039835
:10795000C0191330F2F7F6FC0099401C4843074663
:10796000022E04D00DE031481DB0F0BD0027206F7D
:107970006168C01B40194908884202D92C481DB0D3
:10798000F0BDA06E616840194908884223D9012ED4
:1079900001D0022E07D11298159716951490012E3A
:1079A00004D0022E04D0002E3BD00DE000200AE0CF
:1079B0001A980E901B980F901C9810906846018C96
:1079C00010A881800EA8179014A92046FFF7DAFBB3
:1079D00001990143D3D1A06E6168401949088842DA
:1079E00000D901BE129805906846018C0183A06EF3
:1079F0000C9707900D951C98019002961B980CA966
:107A000005AA009003920491A26E216E20461A9B53
:107A1000FFF74EFE0028B2D1A16E4919A1661DB034
:107A2000F0BD0021D1E70000050042090200420933
:107A300006004209FFB597B00646002518E2252842
:107A400077D100242746FD49049400E00443761CC6
:107A500032780120203A90400842F7D130782A2825
:107A60000ED00222307801463039092916D80499FF
:107A70000A235943303940181443761C0490F1E727
:107A8000189802C804911890002904DA01204003D4
:107A900004434842049002200443761C30782E2888
:107AA00014D1042004437078761C2A2809D1189830
:107AB000761C80C8189009E00A214F43303FC7194F
:107AC000761C3078014630390929F5D930786C2890
:107AD00010D006DC4C281AD068280ED06A2817D19E
:107AE00004E0742813D07A2812D110E00120400558
:107AF00004430CE00121090501E0032109050C43C1
:107B00007178814203D1012000052418761C761C6F
:107B10003078119066280BD013DC58287DD009DC12
:107B200000287BD04528F6D04628F4D047281AD123
:107B3000A5E118E0632835D0642870D0652812D1FB
:107B40009DE170286CD008DC6728F1D069287BD0D3
:107B50006E280DD06F2806D1BAE073282ED0752874
:107B600071D0782859D01A9A199990476D1C7EE1E6
:107B70006002400F022809D003280DD0042818986D
:107B800001680DD00D60001D189070E11898EA177B
:107B900001680D604A60F6E7189801680D80F2E709
:107BA0000D70F0E718986A4601781172001D189060
:107BB0000020507202A80090012005E0189802C829
:107BC000189000200091C04361070DD5002101E00D
:107BD0000199491C0191B94212DA8142F8DB009AFD
:107BE000515C0029F4D10BE0002101E00199491C0E
:107BF00001918142FADB019A0099895C0029F5D153
:107C0000019904981A9B471A21463846199A00F0A0
:107C100097FA0199401945180BE04FE02CE113E069
:107C20004EE0009800990078491C00911A9A199921
:107C300090470198401E0190401CF2D121463846E1
:107C40001A9B199A10E137E00A2000210090019157
:107C50006002410F022907D0189A01CA1892C21770
:107C60009446032908D00AE01898C01DC108C9002D
:107C700005C91891944607E000B2C217944604293A
:107C800002D140B2C1178C4600226146944506DA03
:107C90000A460021404291418C462D2102E02105F7
:107CA00004D52B216A461173012103E0E10701D0BD
:107CB0002021F7E7029155E00A200AE0102008E0B1
:107CC000102000900021042004430191082703E0C4
:107CD00008200021019100906002410F022907D085
:107CE000189A01CA189200229446032908D008E085
:107CF0001898C01DC108C90005C91891944603E031
:107D000080B2042900D1C0B200210291210729D5F7
:107D10001199702906D0009A1021019B4A401A43FC
:107D200005D00EE040216A461173012108E061464A
:107D3000014306D030216A46117311995173022113
:107D40000291009A0821019B4A401A430AD16146D8
:107D5000014301D1610705D530216A461173012124
:107D60007F1E02911199582904D035A10E910DA9B9
:107D70000D910DE037A1F9E76146019B009AF2F7FA
:107D80000BFB0E9B8C469B5C0D9A521E0D92137042
:107D900061460143F0D10D9805A9081A20300190E1
:107DA000600703D501200004844300E00127019807
:107DB000874201DD381A00E0002001990090411847
:107DC000029809180498401A0490E00306D421464A
:107DD0001A9B199A049800F0B3F94519002706E098
:107DE00003A81A9AC05D199990476D1C7F1C0298D0
:107DF0008742F5DBE0030CD521461A9B199A0498BB
:107E000000F09EF9451904E01A9A3020199990471C
:107E10006D1C0099481E00900029F5DC08E00D98C3
:107E20000D990078491C0D911A9A199990476D1C6B
:107E30000199481E01900029F1DC63E10928010045
:107E400030313233343536373839616263646566D0
:107E50000000000030313233343536373839414292
:107E6000434445460000000000F05AF94519761CCD
:107E70003078002800D0E2E528461BB0F0BD60074E
:107E800000D406271898C01DC108C90048680A68B0
:107E90000831C30FDB071891190001D09CA108E03D
:107EA000210501D59BA104E0E10701D09AA100E0E2
:107EB0009AA1430011985B08109165280CD006DC4C
:107EC000452809D046281DD0472841D141E06628E1
:107ED00018D067283CD13CE00021112F01DB112094
:107EE00000E0781C0191009008A911A8FEF7C8FFD6
:107EF000139905910021119A15927F1C12980197F0
:107F0000009150E00120C00703900120019008A9D2
:107F1000009711A8FEF7B4FF139A14990592002256
:107F2000119B009212981593059A0192002901D095
:107F3000104602E0791C40180190381A01D50198CA
:107F400004E04042401E0090781C0190C01B02904B
:107F500043E0012F00DA01270021112F01DD11205C
:107F600000E038460191009008A911A8FEF788FFAB
:107F700013990591119A0021129815920091019779
:107F800021070CD40599B94201DB019900E0019168
:107F9000012904DD159A491E515C302906D0B842EA
:107FA00001DA011D05DA0121029115E00199491E4E
:107FB000EDE7002805DC0099411800910199091AA4
:107FC00003E0019A411C914200DD01910099401AA1
:107FD000401C02900120C0070390200706D402999C
:107FE0000198814202DB0020C043029000206946D4
:107FF000C87707AF012103980337C907884224D007
:10800000022011902B201290039800280CDA404295
:1080100003902D20129007E00A210398F2F792F9BD
:1080200030317F1E039039701199481E119000293C
:10803000F2DC03980028EFD1791E1298087030788E
:10804000202108404530BF1E387006A8C01BC01D47
:10805000039010980078002800D001200199411861
:108060000298C0170918039809180498401A401E6E
:108070000490E00306D421461A9B199A049800F054
:108080005FF8451910980078002803D01A9A1999BA
:1080900090476D1CE00324D521461A9B199A049839
:1080A00000F04EF845191CE00098002807DB009905
:1080B0000598884203DD1598405C199901E01999EB
:1080C00030201A9A904700986D1C401C009002982E
:1080D000401E0290002804D11A9A2E201999904728
:1080E0006D1C0199481E01900029DDDC05E03878FF
:1080F0001A9A7F1C199990476D1C0399481E03908A
:108100000029F4DC21461A9B199A0498ACE6000079
:108110002D0000002B0000002000000000000000E7
:10812000F8B5044600251E461746880404D405E029
:1081300039462020B0476D1C641EF9D52846F8BD8D
:10814000FFB50446002581B01E46C80301D530277F
:1081500000E02027880404D505E038460399B0479D
:108160006D1C641EF9D5284605B0F0BDF0B56B490D
:1081700093B00A6802924A6801928A680492C968B8
:108180000391674910910168029A5140016041686A
:10819000019A514041608168049A51408160C268EF
:1081A00003994A4000218E46C26000214B1CDC1717
:1081B000A40FE418A408A4001B1B9B001B181B8819
:1081C000584E1B041B0EF55C8B1CDC17A40FE41827
:1081D000A408A4001B1B9B001B181B68CA171B02CA
:1081E0001B0EF45CCB1CDF17BF0F920FFF18521849
:1081F000BF089208BF009200DB1B8A1A9B00920006
:108200001B1812181B6812781B0EB25CF35C7646C2
:10821000092E39DA17466F403E4666405E40B44646
:108220000C923E0603D57E001B277E4000E07E00B8
:10823000F6B267467E402F46724067403E0603D541
:108240007E001B277E4000E07E00F6B267467E403F
:10825000274675405F403E0603D57E001B277E40C3
:1082600000E07E00F6B267467E4074400C9E1F46DA
:1082700077403E0603D57E001B277E4000E07E004F
:10828000F6B267467E4073401B06240423432C024B
:10829000234313438C0008AA491C1351042985DB8E
:1082A000109B204A591C10910399CCB2145D2506ED
:1082B0000C04240E145D2C430D022D0E555D090E89
:1082C000515C2D02254309041A7829434A4002993A
:1082D0005140019A02914A4011460192049A4A4043
:1082E00011460492039A4A400392029A0899514017
:1082F0000160019A099951404160049A0A995140DC
:108300008160039A0B995140C1607146491C8E46A9
:108310000A2900DA49E713B0F0BD0000A09B002055
:1083200020ED020020EB0200044902680A60426866
:108330004A6082688A60C068C8607047A09B00205D
:10834000134610B50A461946F2F7C4F810BD0A687C
:10835000531C0B6010707047002A13D08018491E00
:10836000D30703D0401E03784B70491C520809D034
:108370000346203BDB7F4B70801E03788B70891C8B
:10838000521EF5D17047FEE710B584B004784378EB
:108390008278C17800910394029301920379427923
:1083A00003A10B48FEF778FC094804B010BD00009B
:1083B000253032583A253032583A253032583A254D
:1083C0003032583A253032583A25303258000000C1
:1083D000808F0020FFB58DB0044600206946169DB1
:1083E000087320781E4600280BD003A800900121B6
:1083F00001960295224608460E9B08F0E5FA0028F1
:108400007ED16268002A3AD0217A002937D02089AB
:10841000C00501D5032000E002200B9206910E99C1
:10842000079103A9059101950091069932464906E5
:10843000090E079B08F0EBFA002861D10698002787
:1084400000281CDD002D08D00B98B900081829461B
:108450000DF09CFD002853D10DE00598BA0001787D
:10846000079809180B9810180DF008FD0598059944
:108470000078801C087006987F1C8742E2DBE26867
:10848000002A41D0217C00293ED0208AC00501D598
:10849000052000E004200B9207910E99069103A994
:1084A000059100910799019589063246090E069BB0
:1084B00008F0ADFA002823D107980027002823DD13
:1084C000002D0CD00B99F800401840680C90042245
:1084D0000CA9284610F027FB002811D10EE00B98BC
:1084E000F90008184168059802780698101812F0EB
:1084F00040FF059805990078001D08707F1C00E07A
:108500009DE007988742DBDB6269002A3BD0217E31
:10851000002938D0208BC00501D5072000E00620B7
:108520000B9207910E99069103A905910091079965
:10853000019509073246090E069B08F068FA0028E3
:108540007DD10798002700281DDD002D09D03801B6
:1085500039180B98081829460DF018FD00286ED11F
:108560000DE005980B9A017806980918380138181B
:1085700080180DF083FC0598017810310170079880
:108580007F1C8742E1DBE0692746203784460028CC
:1085900012D0397800290FD0208CC00501D50920D0
:1085A00000E0082003AA00920196029562460E9B05
:1085B00008F00AFA002842D1206AC00112D5022030
:1085C0003856014680316FD06946087403A8009080
:1085D0000196029504AA01210A200E9B08F0F4F9E5
:1085E00000282CD1626A002A0AD003A800900196C4
:1085F0000295042112200E9B08F0E6F900281ED1F6
:10860000A26A002A0CD0397B002909D003A8009067
:108610000196029516200E9B08F0D6F900280ED17F
:10862000226B002A10D0397D00290DD003A80090BC
:10863000062041430196029517200E9B00E081E041
:1086400008F0C2F900287DD1208FC0070CD003A804
:1086500000902246019602953632022119200E9B87
:1086600008F0B2F900287CD1A08FC0072DD00E9958
:10867000029103A9274600911A203A373246019504
:108680000221029B08F0C3F900286AD1002D11D005
:10869000388869468883022207A9284610F043FAE1
:1086A00000285ED111E0FFE704A809F053FA002882
:1086B00057D18BE76846027B02983988101812F070
:1086C00054FE6846017B891C01732746226C4037A3
:1086D000002A0CD03979002909D003A8009001960E
:1086E000029520200E9B08F06FF9002839D1A26C6A
:1086F000002A0CD0397B002909D003A800900196EC
:10870000029521200E9B08F05FF9002829D1226DE7
:10871000002A0CD0397D002909D003A800900196C9
:10872000029524200E9B08F04FF9002819D1A26D64
:10873000002A0ED0397F02290BD303A80196029597
:10874000009000E00DE0FF200E9B08F03DF90028AE
:1087500007D10F98002803D06846017B0F9801705D
:10876000002011B0F0BD70B5044682B000686A46C2
:10877000211D0EF087FB00280FD1A07B002540288B
:1087800001D060280ED1009A0199134653406940E8
:108790000B4302D1E17B490701D5FFF7F4FD616886
:1087A00089186160A168FF264A1C002A06D0C028EB
:1087B0000ED0491EA1600BD1A67313E0206861683A
:1087C0004268914204D0006802689047FF2804D0B4
:1087D000204612F07DF902B070BD6068401C6060F8
:1087E000A673A560002002B070BD000070B50446FD
:1087F000807B88B00E4660280AD0402808D08028A8
:1088000006D0A02804D02046FFF7ADFF08B070BD09
:108810000025802813D0A02811D0681E2E4B079069
:108820000193294607AA2046009406AB0FF0BEF933
:108830000028EBD16846007E00284AD106E00120DE
:108840008002864206D1401C08B070BD0120C007DE
:1088500008B070BD02A920460DF074FF0028F7D1C2
:108860000498002808D0711C02A8FFF7BFFF002859
:10887000EED104980028F6D1A07B802801D0A02852
:1088800003D16846807DFF2801D0FFF77CFD039966
:108890006160A068FF26421C002A07D0A17BC02986
:1088A0000DD0401EA0600AD1A67312E02068426875
:1088B000914204D0006802689047FF2804D0204607
:1088C00012F006F908B070BD6068401C6060A673C5
:1088D000A560002008B070BDA97B020030B59FB034
:1088E000602106A8F1F7FDFD0620694608762848B4
:1088F00080680D90F1F70AFE08A90876FF210E980E
:10890000013108430E9006A803F0EAFA040009D0EA
:1089100020A122A0FEF7B0F9214621A0FEF7ACF974
:108920001FB030BD00256846057505A9284609F029
:10893000A7F9040006D017A118A0FEF79DF921465B
:1089400022A018E002950395022168460495017261
:108950004172284800900195684602AB264A0021E2
:10896000007D03F0E1FA040009D00AA10BA0FEF794
:1089700083F9214621A0FEF77FF91FB030BD29A160
:1089800006A0FEF779F929A0FEF776F91FB030BDF1
:108990003C2A00205B455D2000000000257300009C
:1089A0006572726F722073657474696E672061649A
:1089B000766572746973656D656E74206461746147
:1089C0003B2072633D25640A000000006572726FEF
:1089D000722064657465726D696E696E672061648A
:1089E000647265737320747970653B2072633D25F2
:1089F000640A000085910100FFFFFF7F6572726FBE
:108A00007220656E61626C696E6720616476657262
:108A1000746973656D656E743B2072633D25640AED
:108A2000000000005B495D200000000041647620EA
:108A300053746172742E2E2E0A00000070B5044625
:108A40000078A8B00A2871D008DC00285BD0012883
:108A50006DD0072809D0082854D1CCE00C2867D065
:108A60000F2866D011284DD1F4E0627910A8216951
:108A700007F022FE002845D1211D10A812F0B4F8FD
:108A80000D2020564621241DC8423BDB20780028BB
:108A900001D0012836D1204603F0F0F8002831D06B
:108AA00003F0B4FD050006D077497848FEF7E4F8F6
:108AB000294677A0AFE002A9002009F0E1F80500FF
:108AC00006D071497148FEF7D7F829467848A2E0E8
:108AD00000217848019100900B466846764AA11C17
:108AE000007A03F0E3FB05000CD067496748FEF706
:108AF000C3F8E01CFFF748FC0246A1782B466F48FC
:108B0000FEF7BAF87EE0606800280AD06CA16EA07B
:108B1000FEF7B2F86DA06168FEF7AEF800F0F6FC63
:108B200070E074A168A0FEF7A7F803E06DE056E0DE
:108B300074E086E071A0FEF79FF8208904A903F095
:108B40009DFB00280BD076A15FA0FEF795F8FF22D1
:108B5000754B2E3275A17CA0FEF78EF8FEE707A8B4
:108B6000FFF712FC05460AA80230FFF70DFC064687
:108B70006A46D08E0A214843938E518E754A5143DE
:108B80006A46D27E029300920191039008AA527A1B
:108B90002B4631467048FEF76FF8208911F0D2F964
:108BA00005000AD05EA148A0FEF766F829466BA032
:108BB000FEF762F8002028B070BD208900226E49BF
:108BC00011F0DCFA04001DD055A13FA0FEF754F8C7
:108BD00021466AA0FEF750F8002028B070BD45A1DC
:108BE00039A0FEF749F821796DA0FEF745F8208DF0
:108BF00011F072FA92E73FA133A0FEF73DF86FA0A3
:108C0000616808E0002028B070BD3AA12EA0FEF7F0
:108C100033F874A06168FEF72FF8F3E735A12AA0B6
:108C2000FEF72AF86068008A0090207B2389628919
:108C3000C00701D075A100E077A17BA0FEF71CF86A
:108C4000E0E72CA120A0FEF717F82389E288A1888D
:108C500083A055E7A08804A903F010FB00280BD0DF
:108C60002FA119A0FEF708F8FF222F4B82322FA167
:108C700035A0FEF701F8FEE706A803300CF01DFD55
:108C8000012028B070BD000080950100C897010048
:108C90004661696C656420746F2063616E63656C06
:108CA000207363616E3B2072633D25640A000000FF
:108CB0008C9501003D8A01003075000028EE02000D
:108CC0005B575D20000000002573000043656E7453
:108CD00072616C20436F6E6E656374696F6E20669F
:108CE00061696C65643B207374617475733D2564C0
:108CF0000A0000005B495D200000000043656E74BF
:108D000072616C20436F6E6E656374696F6E20656F
:108D1000737461626C6973686564200D0A000000F9
:108D20005B455D2000000000BCDC02002E2E5C7361
:108D300072635C6170705F626C655F63656E7472B4
:108D4000616C2E63000000002573202564202573CC
:108D50000D0A0000E2040000C4ED02004661696CE7
:108D6000656420746F2061646420706565723B20C7
:108D700072633D25640A0000099601004661696C32
:108D8000656420746F20646973636F766572207305
:108D9000657276696365733B2072633D25640A00E2
:108DA000646973636F6E6E6563743B207265617393
:108DB0006F6E3D3078253032780A00006469736345
:108DC0006F76657279206475726174696F6E206563
:108DD0007870697265733B20726561736F6E3D25B3
:108DE000640A0000656E6372797074696F6E206347
:108DF00068616E6765206576656E743B207374618B
:108E00007475733D2564200D0A000000696E646965
:108E1000636174696F6E00006E6F74696669636187
:108E200074696F6E00000000726563656976656441
:108E30002025733B20636F6E6E5F68616E646C65A6
:108E40003D25642C617474725F68616E646C653D6D
:108E500025642C617474725F6C656E3D25640A0034
:108E60006D747520757064617465206576656E74C7
:108E70003B20636F6E6E5F68616E646C653D256458
:108E8000206369643D2564206D74753D25640A0086
:108E900010B520231A461946012011F01FFB0028A7
:108EA0000BD00BA10CA0FDF7E7FEFF220B4BE63227
:108EB0000BA112A0FDF7E0FEFEE702F0B3FE3B209F
:108EC000C04302F0C5FF06210FA002F099FF10BDBC
:108ED0005B455D200000000025730000D9DC020026
:108EE0002E2E5C7372635C6170705F626C655F6391
:108EF000656E7472616C2E6300000000257320257E
:108F0000642025730D0A0000626C655F68720000C2
:108F100010B5FFF7E3FC00F0F9FA10BD38B51F4CAF
:108F20005A25607800280AD01D490620087020784C
:108F30004870401CC0B22070A0280CD00CE000206B
:108F4000C04300901748002300681A46032114F01C
:108F500047FB257038BD25700222114960880CF04E
:108F600043FE040007D010A111A0FDF785FE2146A5
:108F700010A0FDF781FE7D21C9000A480FF0CEFB4D
:108F80000028E7D013491448FDF776FE134B9E22C4
:108F900013491448FDF770FEFEE700003C2A00204C
:108FA000402A00208C9200205B575D2000000000CA
:108FB000257300006872732073656E64206E6F7491
:108FC000696679206661696C6564202D2072633A58
:108FD00025640A00FC93010004940100EEDC020009
:108FE0000C9401002494010010B50249024810F0CD
:108FF000D1FE10BD118F01008D94010070B50D469A
:109000000646C0B0144614A115A0FDF735FE298808
:10901000324614A0FDF730FE0020694608802888FB
:10902000002816D10CA10EA0FDF726FE606821884D
:10903000028A17A0FDF720FE6B46FA2201A960689C
:1090400008F0C9FF002804D16846018801A800F093
:10905000E9FC002040B070BD5B495D2000000000CD
:10906000257300005265616420636F6D706C6574D8
:10907000653B207374617475733D256420636F6E66
:109080006E5F68616E646C653D25640A00000000D7
:1090900020617474725F68616E646C653D25642044
:1090A0006C656E3A25642076616C75653D0A00003A
:1090B00070B50D460646144605A107A0FDF7DCFD78
:1090C00023882988324605A0FDF7D6FD002070BD13
:1090D0005B495D200000000025730000537562733A
:1090E000637269626520636F6D706C6574653B20A7
:1090F0007374617475733D256420636F6E6E5F6871
:10910000616E646C653D256420617474725F686192
:109110006E646C653D25640A0000000070B50D4664
:109120000646144605A107A0FDF7A6FD2388298859
:10913000324605A0FDF7A0FD002070BD5B495D2013
:109140000000000025730000577269746520636F8A
:109150006D706C6574653B207374617475733D2527
:109160006420636F6E6E5F68616E646C653D25643C
:1091700020617474725F68616E646C653D25640A79
:1091800000000000F0B504460078654D8FB0092856
:1091900052D007DC634E00280BD0012842D00328B0
:1091A0003FD1A2E00D287DD00E284FD00F2838D116
:1091B00089E05DA15EA0FDF75FFD6268002A0AD02C
:1091C0005CA15EA0FDF758FD6068002805D0FFF7A0
:1091D00085FB6E80A0E063A1F3E7208904A903F07A
:1091E0004DF807A8FFF7D0F806460AA80230FFF7A7
:1091F000CBF801466846C38E0A2043436846878EF3
:10920000428E5B4842436846C07E039300900297BB
:10921000019208A8427A33465648FDF72DFD208971
:10922000688079E040A142A0FDF726FD217952A097
:10923000FDF722FD6E8006E03BA13DA0FDF71CFD81
:1092400054A0FDF719FDFFF749FB65E036A138A0F2
:10925000FDF712FD607A584E8007C10F328857A083
:10926000FDF70AFD217A00226348D243012902D08A
:10927000022925D050E0E188338899424CD1617AA7
:109280008907C90F697013D07D21C9005A480FF0B2
:1092900045FA002840D059A15AA0FDF7EDFC5A4BE1
:1092A0009E2200E019E059A15EA0FDF7E5FCFEE773
:1092B0000092002300681A46032114F091F92BE074
:1092C00000216970F4E718A119A0FDF7D5FC2289E7
:1092D000A18857A0FDF7D0FC1EE013A114A0FDF754
:1092E000CBFC5EA0FDF7C8FC16E0208904A902F0C3
:1092F000C5FF0DA10EA0FDF7BFFC6846C08E0A2178
:10930000484300906846838E428E1948424368461F
:10931000018E5648FDF7B0FC00200FB0F0BD0000F4
:109320003C2A0020FFFF00005B495D200000000098
:10933000257300006661696C656400007065726980
:1093400070686572616C20636F6E6E656374696FBF
:109350006E2025733B207374617475733D25640A18
:109360000000000065737461626C69736865640075
:10937000E2040000C4ED0200646973636F6E6E6501
:1093800063743B20726561736F6E3D3078253032B7
:10939000780A0000616476206475726174696F6E8A
:1093A0002065787069726564202D20726573746120
:1093B0007274206164760A00FA2900207375627362
:1093C0006372696265206576656E743B20637572B1
:1093D0005F6E6F746966793D25642076616C756592
:1093E0002068616E646C653B2076616C5F68616EBD
:1093F000646C653D25640A008C9200205B455D200D
:109400000000000025730000EEDC02002E2E5C73CD
:1094100072635C6170705F626C655F7065726970C9
:10942000682E630025732025642025730D0A000033
:109430006D747520757064617465206576656E74F1
:109440003B20636F6E6E5F68616E646C653D256482
:10945000206D74753D25640A0000000073656E641C
:10946000206E6F74696679206F6B0A006CEE0200E3
:1094700010B50FF00FF901460023024A02480FF021
:109480002DF910BD1D8F01008C92002010B517A181
:10949000086882B0496800900191684610F04CF964
:1094A000684610F049FDFFF7E3FFFFF7F1FC00F01D
:1094B00005FA0DF03DFF12F0C3F80E48E1210090CF
:1094C0000023012289000CA013F0F4FF0E4C0028A9
:1094D000606009D013F060FE002100910B46024647
:1094E0000121606814F07CF802B010BD080203048A
:1094F00005060000F9C8020054696D6572277320E3
:109500006E616D6500000000202A002010B584B057
:1095100003A9002008F0B4FB040009D018A11A48E0
:10952000FDF7AAFB214619A0FDF7A6FB04B010BD6C
:109530006846417AF92001406022684682805022C4
:10954000C280002249080272490041720092194B00
:1095500001AA1949007B02F07BFF040007D008A193
:109560000948FDF789FB214614A0FDF785FB20A1E2
:109570000548FDF781FB20A0FDF77EFB04B010BD80
:109580005B455D2000000000C89701006572726FA6
:10959000722064657465726D696E696E67206164BE
:1095A000647265737320747970653B2072633D2526
:1095B000640A00003D8A0100FFFFFF7F4572726F61
:1095C0007220696E6974696174696E6720474150E1
:1095D00020646973636F766572792070726F63655A
:1095E000647572653B2072633D25640A00000000CB
:1095F0005B495D20000000005363616E207374615D
:1096000072742E2E2E0D0A00F0B589B00C0005469E
:1096100015D043A144A0FDF72FFBAA88214643A003
:10962000FDF72AFB4EA140A0FDF726FB4EA0FDF75B
:1096300023FBA888132103F027FD09B0F0BD48A142
:1096400039A0FDF719FBAA8821464DA0FDF714FBB0
:10965000594C04AA206803906068049003A9284626
:1096600010F016FD06000ED0F188A8880023534A9A
:1096700004F066FE07000CD051A153A0FDF7FCFAE0
:10968000394652A03DE04EA14FA0FDF7F5FA59A092
:1096900043E000276548029701970090F188A88869
:1096A000022302AA05F04AFC060007D044A146A006
:1096B000FDF7E2FA31465EA0FDF7DEFAA0680590FC
:1096C000E06806902069079007AB06AA05A928461E
:1096D00010F0CEFE04001BD0012102A8FDF78AFA8B
:1096E0005D4801970090A188A888022302AA05F08E
:1096F00025FC0400A1D032A133A0FDF7BDFA21461C
:1097000056A0FDF7B9FA3AA0FDF7B6FA09B0F0BDD8
:109710002BA12DA0FDF7B0FA5CA0FDF7ADFAF2E7A2
:109720005B575D20000000002573000053657276D2
:1097300069636520646973636F7665727920666119
:10974000696C65643B207374617475733D25642096
:10975000636F6E6E5F68616E646C653D25640A00C0
:109760005B495D200000000053656E6420646973EE
:10977000636F6E6E65637420636D64200D0A000074
:109780005365727669636520646973636F76657289
:109790007920636F6D706C6574653B2073746174C0
:1097A00075733D256420636F6E6E5F68616E646CD7
:1097B000653D25640A000000A8DC0200FD8F010061
:1097C0005B575D2000000000257300004661696C56
:1097D000656420746F2072656164206368617261E2
:1097E0006374657269737469633B2072633D2564B9
:1097F0000A0000005065657220646F65736E2774FF
:1098000020737570706F727420746865207573654D
:109810007220737065636966696320636861726151
:109820006374657269737469630A00001D910100B5
:109830004661696C656420746F2077726974652075
:1098400063686172616374657269737469633B20F4
:1098500072633D25640A0000B19001004661696CA5
:10986000656420746F20737562736372696265202A
:10987000746F20636861726163746572697374697F
:10988000633B2072633D25640A00000050656572E9
:1098900020646F65736E277420737570706F7274B7
:1098A00020746865207573657220737065636966DE
:1098B000696320434343440A0000000010B50CF0E4
:1098C000BFF80CF04FF904480249016000214160E3
:1098D00010BD0000DD980100C427002010B504462B
:1098E00000788AB001280ED0022819D0032828D089
:1098F0001CA11EA0FDF7C0F91D4B2B221DA123A00A
:10990000FDF7BAF9FEE724A118A0FDF7B5F9A068A4
:10991000694640680CF066FB0146A28820A01CE066
:109920001DA112A0FDF7A8F9A068694600680CF017
:1099300059FB0146E388A2882348FDF79DF90AB048
:1099400010BD15A109A0FDF797F9A0686946006848
:109950000CF048FB0146A2881CA0FDF78DF90AB067
:1099600010BD00005B455D20000000002573000075
:1099700008DD02002E2E5C7372635C6170705F62A2
:109980006C655F7376722E630000000025732025DE
:10999000642025730D0A00005B495D200000000073
:1099A0007265676973746572656420736572766940
:1099B000636520257320776974682068616E646C24
:1099C000653D25640A000000C4EE0200202020202E
:1099D0002D7265676973746572696E67206465735B
:1099E00063726970746F72202573207769746820C0
:1099F00068616E646C653D25640A000013460A4682
:109A000010B5014601480EF0C5FD10BD048F0020C1
:109A100013460A4610B5014601480EF00DFE10BD72
:109A2000048F002070B500240D460646002907D893
:109A30000DE0002C04D0200702D107A0FDF71CF98F
:109A4000315D06A0FDF718F9641CAC42F1D302A009
:109A5000FDF712F970BD00000D0A000025303258E4
:109A600020000000002809D170B51C4615460B46A1
:109A70002246294602A0FDF7FFF8FEE770470000E6
:109A80005B455D46696C653A202573204C696E65BF
:109A90003A202564204572726F723A30782530384A
:109AA000780D0A0000B587B000220592009002925E
:109AB000039204920191684600F002F807B000BDDD
:109AC000F0B504468DB0406806900020054602902F
:109AD000A0685049002801DC079100E00790E06889
:109AE000002801DC059100E0059020461030089028
:109AF0000798471B7ED02068405D00287AD06169B6
:109B00000420401A0026009000280FDD2168A819C3
:109B1000095C002976D03D2904D03F48F0F7ECFCE1
:109B200000286FD00098761C8642EFDB87422068C1
:109B30000ADA41196269089810183A46F0F7A9FC48
:109B40006069C019606161E0411962690898101884
:109B5000009AF0F79EFC089800998446002006467B
:109B600004294FDB00276146CA5D80013D2A0BD0E6
:109B7000002E47DC28490B78002B0BD0DBB2934238
:109B800004D1254A891A07E0761C06E04B78491C67
:109B9000002BF3D10021C94308187F1C042FE2DBFE
:109BA000022E2FDC31060143481C2BD000982D18C3
:109BB00000206061059B029A080E9A4226DA029EF6
:109BC000069B0A149A55029A521C0292022809D244
:109BD000059B9A421ADA029E069B0A129A55029A2D
:109BE000521C0292002883D11046059A90420DDA49
:109BF000029A01E00AE005E0069881540298401CB0
:109C0000029075E70020C0430DB0F0BD02980DB082
:109C1000F0BD0000FFFFFF7FB4DB0200FFB581B0A5
:109C20000022039C002932DD1C4E855C521C2D0253
:109C30008A4201DA875C7D192D02521C8A4201DAC0
:109C4000875C7D192F02BF0EF75D2770AF03BF0E33
:109C5000F75D67702F05BF0EF75DAD06A770AD0EFF
:109C6000755DE5702546241D521C8A42DDDB002D02
:109C70000DD0511A00290ADD0420002B05D0401A0E
:109C800040193D22F0F726FC01E0401A441900205B
:109C90002070039805B0201AF0BD0000B4DB02006C
:109CA00010B50248F2F770F810BD00000000054042
:109CB00001200003704700001846134610B5024605
:109CC0000148F2F7E5FC10BD00000540FF2001301F
:109CD0007047000008B500920B220248F2F794FA90
:109CE00008BD00000000054001207047704710B516
:109CF000044608F0DFFC002807D0A189002904D021
:109D00006089884200D3084610BD172010BD70B589
:109D10000C4605460421204608F04BF900280AD1DC
:109D200020680068C278817840780902014328469B
:109D300004F0D0FC002070BD10B5002104F00CFD33
:109D4000002010BDF3B50D468DB00121284608F066
:109D500030F9040046D12868012107680EF08AFE18
:109D60002868008A00283DD03C7804AE012C02D03F
:109D7000022C28D101E0042000E0122001460090CE
:109D8000284608F016F9002801D004462AE0286881
:109D900000680DF05FF969460882012C02D0022CA0
:109DA00013D108E002231A46301D29680CF0A4F8EC
:109DB000002808D109E010230222301D29680CF088
:109DC0009BF8002801D00A240CE0286800990EF0C6
:109DD00051FE002404A90D9804F040FD2868008A73
:109DE0000028C1D121460D9804F0DAFC20460FB0BE
:109DF000F0BDF8B5064608680024008A0D46002824
:109E000021D00421284608F0D4F8002801D00A24E3
:109E100019E028680068417803780A021A43694605
:109E20000A80C1788278080210436946488004217C
:109E300028680EF01FFE6946304604F0AFFD286822
:109E4000008A0028DDD12146304604F03DFD002087
:109E5000F8BD10B506F0DAF9002010BDF8B50E46D1
:109E6000074600250221304608F0A3F804000CD173
:109E70003068066808F02EF86A460021384600F07F
:109E80006FFA040008D008F061FB2A4621463846E4
:109E900004F0C4FD2046F8BD707832780102114309
:109EA000009800F00BFB0098FFF721FF054608F033
:109EB0004DFB2A460421384602F00EFDE5E7F3B5D6
:109EC0000C46002681B035460421204608F071F882
:109ED00007000DD122681068417803780E02C1781E
:109EE00080780D0205431E43042110460EF0C2FD8A
:109EF0002B46324639460094019804F0B5FD3846A9
:109F000003B0F0BD10B50A46002104F0CDFE0020DC
:109F100010BD10B50A46002104F0CEFD002010BD92
:109F2000F3B50C4683B00121204608F042F8050045
:109F300033D1206801680E7801210EF09BFD206866
:109F4000008A002829D0371F3146052E01DA042562
:109F500023E0204608F02DF8002801D005461CE03B
:109F6000206800680DF076F869460880206800686F
:109F7000801C0DF06FF869464880019720680068E2
:109F8000001D0290039804F0B5FD314620680EF0E4
:109F900071FD2068008A0028D6D12946039804F074
:109FA000EDFD284605B0F0BD10B50A46002104F0CD
:109FB00047FE002010BDF3B50C4683B001212046BA
:109FC00007F0F7FF05002CD1226801211068067800
:109FD00010460EF04FFD022E01D20A2521E0206826
:109FE000008A00281DD0B71E3146204607F0E1FF49
:109FF000050016D1206800684178027809021143F3
:10A000006A461180801C029069460197039804F00B
:10A0100071FE314620680EF02DFD2068008A002870
:10A02000E2D12946039804F089FE284605B0F0BD28
:10A0300010B504F0A7FE002010BD38B50C4605464B
:10A040006A460121182000F05FF9002805D004704D
:10A050002846009901F0B9FD38BD062038BD002919
:10A0600001D0914201D903207047F8B50C4615463E
:10A07000064604216A46084600F046F900280AD040
:10A080000470210A41708570290AC1703046009918
:10A0900001F09BFDF8BD0620F8BD002901D09142DA
:10A0A00001D903207047FFB581B00B9E15460C46C1
:10A0B0001F466A460620B11D00F026F9002813D07D
:10A0C0000470210A41708570290AC1700771390A2C
:10A0D00041713246801D0A99F0F7DBF90099019829
:10A0E00001F073FD05B0F0BD062005B0F0BDF8B578
:10A0F00015460C00064612D06A4602211D2000F0CB
:10A1000003F900280DD00470210A417029460098F7
:10A110000EF066FE3046009901F057FDF8BD0324AD
:10A1200000E0062428460EF021FF2046F8BDF8B5D1
:10A1300015460C00064612D06A4602211B2000F08C
:10A14000E3F800280DD00470210A417029460098D8
:10A150000EF046FE3046009901F037FDF8BD0324AD
:10A1600000E0062428460EF001FF2046F8BDF8B5B1
:10A170001C4615460E0007460CD0208A01214019C6
:10A180004902884206D8384600F00EF9218A401F5D
:10A19000884201DA032516E06A460421162000F001
:10A1A000B3F800280ED00670310A41708570290A74
:10A1B000C170214600980EF013FE3846009901F058
:10A1C00004FDF8BD062520460EF0D0FE2846F8BD59
:10A1D000002901D10320704738B50C4605466A4670
:10A1E00002210A2000F090F8002807D00470210A0C
:10A1F00041702846009901F0E8FC38BD062038BDC2
:10A20000002901D103207047F8B515460C460646D3
:10A210006A4604210C2000F077F800280AD0047068
:10A22000210A41708570290AC1703046009901F0F9
:10A23000CCFCF8BD0620F8BD002901D0914201D91F
:10A2400003207047F8B507461E4615460C461846CB
:10A250000BF099FE011D6A46102000F055F8002809
:10A260000ED00470210A41708570290AC170011D49
:10A2700030460BF003FE3846009901F0A6FCF8BD0D
:10A280000620F8BD002901D0914201D90320704772
:10A29000F8B507461E4615460C4618460BF073FEE9
:10A2A000011D6A46082000F02FF800280ED0047027
:10A2B000210A41708570290AC170011D30460BF0DA
:10A2C000DDFD3846009901F080FCF8BD0620F8BDA0
:10A2D000F8B515460C4606466A460221122000F0E3
:10A2E00013F800280BD00470210A41702946009809
:10A2F0000EF076FD3046009901F067FCF8BD284667
:10A300000EF034FE0620F8BD70B516460C46054624
:10A3100007F039FE3060002809D0641C0646A1B25F
:10A320000EF0F5FD002803D030680570401C70BDAC
:10A3300030460EF01BFE002070BD70B50546491C6E
:10A34000144689B210460EF0E2FD002803D02068C2
:10A350000570401C70BD20460EF008FE002070BD48
:10A36000134610B50A46042107F04CFE10BD00004C
:10A3700010B508F051F9002807D004210181C180EF
:10A380000249098841810249816110BD24270020CA
:10A39000F1A30100704700000249F7200880002067
:10A3A000704700002427002030B583B0044607F032
:10A3B00091FD204601AA6B46042107F023FE0028E8
:10A3C00005D0002408F0C2F8204603B030BD009D3F
:10A3D000284608F06FF9002807D0AC89002C04D07B
:10A3E0006889A042EED20446ECE71724EAE70000B1
:10A3F000F0B583B0044608F033F907462D4887428C
:10A4000002D1072003B0F0BD206901AB0122002179
:10A4100010340EF005FD002802D0042003B0F0BD7A
:10A4200068460179244B0E460020C200D5182A78D0
:10A430008A420ED1002D11D0012120680EF01AFBA6
:10A440006A6821463846904705002FD0082D18D05D
:10A4500029E08A4202D8401C1B28E6D370060DD49E
:10A460002068018A0EF006FB062000900023324689
:10A470003846216801F0DEFA00202060082003B091
:10A48000F0BD6846067970060DD42068018A0EF08A
:10A49000F1FA06200090002332463846216801F088
:10A4A000C9FA00202060284603B0F0BD002003B0A8
:10A4B000F0BD0000FFFF0000ACD60200172900D25B
:10A4C000172181817047FFB5A5B01E4617460029A8
:10A4D00010D03C7AE00708D020460421084008212B
:10A4E00025460D4010210C4014E002201870102069
:10A4F00029B0F0BD397A880704D4032018701020E1
:10A5000029B0F0BD08462022104040220D461540DB
:10A51000CC09E40128431C902043F1D0259C07F08E
:10A52000D9FC204606F018FC846D08F00FF81C9842
:10A53000002801D0E00709D0002D35D0A00733D482
:10A5400005203070FF20063029B0F0BD07F0C2FCB6
:10A55000259806F0F1FB002811D01DA906F0C0FADD
:10A5600000200090019002900390049005900690C6
:10A570001EA90790072203316846EFF78AFF07F00C
:10A58000E5FF08A968460BF05BF8002805D110A884
:10A59000007AC00701D00F2000E005203070C0B263
:10A5A000FF30013029B0F0BD787A2106C90E88420B
:10A5B00005D90C203070FF200D3029B0F0BD0020EF
:10A5C00029B0F0BD70B515460E46002801D00468CC
:10A5D0000BE00A48046808E0002E0DD031466068A0
:10A5E0000BF02EFC002807D02468002C02D06089D4
:10A5F000A842F1D9002070BD204670BD3027002050
:10A6000008B50BA00090114B0C22102110480EF041
:10A6100063FF002801D00B2008BD0E4900204960CF
:10A6200008600D49496008600C49088008BD0000B9
:10A63000626C655F6174745F7376725F707265706F
:10A640005F656E7472795F706F6F6C00905B002055
:10A65000505C0020302700203827002028270020C9
:10A6600070B505680446002D0DD028682060002DC7
:10A6700006D0A8680EF07AFC294603480EF0BFFE0B
:10A680002568002DF1D170BD505C00200148008884
:10A690007047000028270020FFB58BB00C46074606
:10A6A000169D07F070FC060011D00D9809900896D1
:10A6B0000020694608721D4887420AD002AB224634
:10A6C00001213846FFF7FFFE002811D101E00624E2
:10A6D00026E0216908A8019100906189E4680122BF
:10A6E0003846099BA047002809D06946087209200E
:10A6F000002D02D069460A7A2A70040010D1348AEB
:10A700000E98844203D904240E20287008E02246C3
:10A7100000213046149B0EF083FB15980480002422
:10A7200030460EF023FC20460FB0F0BDFFFF0000C6
:10A73000F0B517461F4A85B014680A9D0022002C08
:10A7400017D066898E4211D1002C12D00646684679
:10A7500003931949027230468E4211D002AB224651
:10A760000121FFF7B0FE002819D109E02468002C70
:10A77000E7D1002D01D001202870052005B0F0BDE3
:10A78000216903A8019100906189E4683B46012298
:10A790003046A047002809D0694608720920002DDC
:10A7A00002D06946097A29700028E7D1002005B057
:10A7B000F0BD000030270020FFFF0000FFB581B092
:10A7C00005461C4611480A9F0B9E0EF000FE00280D
:10A7D00019D00021016045608160029901720399DE
:10A7E0000B4A41721188491C118041810949C76097
:10A7F00006614A68002C1060486001D040892080C2
:10A80000002005B0F0BD062005B0F0BD745B00204F
:10A810002827002030270020F3B500208FB00646FF
:10A820000390684686820C460846012107F0C1FB6A
:10A83000062804D00025049000287DD101E01125D0
:10A84000F9E7206801680F78039026600398018A71
:10A850000EF010F900211920039AFFF76EFD002871
:10A8600016D007F037FB0F9806F076FA446C466472
:10A8700007F06CFE002F79D00F980D9005A8079077
:10A880006846868220002DD007250122520209E069
:10A890001125062004909DE0002903D08B8887882D
:10A8A000BB4206D0C18800290DD08188079801805D
:10A8B0007DE0CB888968098A5918C388994202D0FB
:10A8C0000798078073E08368C1881B8AC918914282
:10A8D00004DD818807980D25018068E00146006845
:10A8E0000028D9D1002C61D008A80990A78800269B
:10A8F000251E17D0A888B84214D1002E37D0304674
:10A90000A9680EF06DFA0020A86024680694002D56
:10A9100005D00EF02BFB294634480EF070FD069D45
:10A92000002DE7D10998324907800C9668460D68DA
:10A93000008C002D07D000E04CE06989814203D0F3
:10A940002D68002DF7D1002500200D9E69460E9040
:10A95000087628480CAF86420BD006AB2A46002169
:10A960003046FFF7B0FD002811D102E023E0AE68C9
:10A97000C9E72869009701906989ED68022230468D
:10A980000E9BA847002802D0694608760920694630
:10A9900006460D7E0C980EF0E9FA002E04D06846AB
:10A9A000018C0798018002E0002C9DD10025002D2C
:10A9B00001D00920049021000CD024680F00264605
:10A9C00006D0B8680EF0D2FA394608480EF017FDE6
:10A9D0003100F2D16846808A009501901823039ACD
:10A9E00004990F9801F041F811B0F0BD505C0020BF
:10A9F00030270020FFFF0000F3B58FB00F46002482
:10AA000008460421059407F0D4FA0146062804D02C
:10AA100000200390002946D101E01120F9E73868B1
:10AA200001684A780B781502CA78897816021D43A6
:10AA30000E43B54233D8002D31D00F990024079131
:10AA400000903C600098018A0EF014F80121052066
:10AA5000009AFFF772FC0B90002825D00798FFF7AB
:10AA6000A3FC009907910C900B98099504700020A5
:10AA70000446069030480768002F44D07889B042D9
:10AA80002BD8099988423BD37868007810280B9816
:10AA900000780ED0002816D002281ED116E0012022
:10AAA0000A210595039038E0112006210390009CAF
:10AAB00032E0002802D001280FD102E00B990120DA
:10AAC0000870042103E00B990220087012210798F6
:10AAD000008A42180C98824201DD002413E0079896
:10AAE0000EF015FA0490002822D0798910F03DFC70
:10AAF00004997868891C0BF0C1F90698401C0690EF
:10AB00003F68002FBAD10698204301D0210011D010
:10AB10000A20009C052103900595059A039801924F
:10AB20000090042322460F9800F09FFF11B0F0BD63
:10AB30000624E8E7009CF0E730270020F3B50C4638
:10AB40009FB0002569460D7220460621069507F044
:10AB500030FA062805D0002269460A72010052D157
:10AB600001E01122F8E720680068417802780902C4
:10AB700011430591C17882780F021743B049427999
:10AB8000007909881202024388B21104084305992A
:10AB90000122B94232D8002930D0039002A80E46D3
:10ABA0001F9D009007F0EFF90D9000282CD0024671
:10ABB00000210720FFF7C1FB00282ED02846FFF711
:10ABC000F3FB0997149503990491216812910D994B
:10ABD00015911190002500981A95109099480468D5
:10ABE000002C7DD06089B04248D3002D1AD0694630
:10ABF000097C676804A8102941D117E068460272F1
:10AC000005980A21069006E120680D90002020603A
:10AC10001120694608720621F8E011206946087281
:10AC2000062108E1099988425AD84FE0397810295D
:10AC300022D10BF01FFA0521C902401A04D00128C5
:10AC400002D003281BD10AE038460BF013FA052185
:10AC5000C902884213D0491C884210D00CE0384603
:10AC60000BF008FA0521C902884208D0491C884225
:10AC700005D0891C884202D060891A908CE0159F0B
:10AC80001A9808903A8A1198121D824228DC2946A7
:10AC900007A810F06AFB022207A938460DF043FF0F
:10ACA00000287CD107A8089910F05FFB022207A9B1
:10ACB00038460DF038FF002872D101E006279AE0EF
:10ACC00000251A9561890998814209D804A960680C
:10ACD0000BF0B6F800285FD1149F009016A800E092
:10ACE00088E00B9010981C9007F04DF91B900028FD
:10ACF00016D000981E901B9808971D901C980A90DB
:10AD0000002069460873504908982746884209D0B0
:10AD100003AB22460121FFF7D6FB002811D101E049
:10AD2000062724E039691DA8009001917989FF6800
:10AD300001221E9B0898B84700280FD06946087367
:10AD400009200A99002903D069460A7B0A990A70EA
:10AD5000070003D01B980EF009F94CE01B98078AF6
:10AD6000102F07D91C980E21017004271B980EF094
:10AD7000FDF840E03A4600210B9B0EF051F81B987D
:10AD80000EF0F4F83B4616AA062112980DF068FF63
:10AD9000002801D165891A952468002C01E025E07E
:10ADA00015E000D01EE7002D24D0159E1198318AA1
:10ADB0001A9C091D81421DDC294609A810F0D5FA0C
:10ADC000022209A930460DF0AEFE002803D01098EB
:10ADD0001121017072E7214609A810F0C6FA02227B
:10ADE00009A930460DF09FFE002803D010991120CC
:10ADF000087063E700271598008A012801D901200F
:10AE000000E00020384312D0390016D00D9D0029F3
:10AE100001D0059806906846007A069A0192009043
:10AE200006232A461F9800F020FE21B0F0BD10989E
:10AE30000A21017005210D9DEBE70D9DEBE7000058
:10AE400084D7020030270020FFFF0000F3B5002761
:10AE500083B00D4608463E460221009707F0A9F848
:10AE60000628044629D0002C27D12868006841789C
:10AE700002780802104300902AD007F084F80700F7
:10AE800028D0024600211E20FFF757FA002826D0BE
:10AE90000398019007F01EF8019805F05DFF07F098
:10AEA00055FB022128680DF0E5FD01232A68009971
:10AEB000039801F035FD00202860009801901D23C3
:10AEC0003A4621460096039800F0CFFD05B0F0BD4C
:10AED0000A24F2E72F682E6011260624EDE70624E7
:10AEE0001126EAE7F3B589B00E460027084602218D
:10AEF000039707F05EF8062803D00024050030D140
:10AF000001E01124FAE730680024006841780278F3
:10AF10000802104303900998009006F0DBFF08AA8E
:10AF200000210098FFF71CFA0190002803D007F0D9
:10AF30000DFB019D15E008984089049007F006FB81
:10AF400037683460398A38460DF094FD3A4602215C
:10AF50000320FFF7F2F900280FD004990170090AC5
:10AF600041700020019002233A4629460094099836
:10AF700000F07BFD040003D00DE011240625F0E76E
:10AF800006F0A8FF05AA06A90998FFF7E9F9040049
:10AF900004D007F0DBFA20460BB0F0BD039905980A
:10AFA000FFF78CFA05980122817B11438173FEF72C
:10AFB0009EFE054607F0CAFA2A460421099801F0C8
:10AFC0008BFCE8E770B506460C460846022106F001
:10AFD000F0FF062801D0002801D0062070BD2068AF
:10AFE0000068417800780D02054313D006F072FF27
:10AFF000304605F0B1FE07F0A9FA022120680DF0F5
:10B0000039FD002329463046226801F089FC0020E2
:10B01000206070BD0A2070BDF3B585B000200D46DC
:10B0200069460390087206460421284606F0C1FFCF
:10B03000062805D000216A46117204007ED101E085
:10B040001121F8E7286807687878397806025448AB
:10B050000E430268002A0FD05089B04209D1002A5D
:10B060000AD002AB00210598FFF72DFA040065D144
:10B0700007E01268002AEFD1052401206946087212
:10B0800081E006F027FF79783A78090211430191AF
:10B09000F978BA780F02296805981743039105F0EB
:10B0A0005BFE00903F480EF092F9040023D0002090
:10B0B00020606060A06006F066FFA06000281ED0DF
:10B0C0000198A080E78003980422008A0399001F5A
:10B0D00083B2A0680DF08BFD039000281AD0A06801
:10B0E0000DF044FF21462F480EF089F909206946EA
:10B0F0000872039C31E009206946087208E00DF0EF
:10B1000035FF214627480EF07AF91120694608726A
:10B11000062422E000980021406C019A8446002811
:10B1200024D08388934208D8934202D1C388BB427B
:10B1300003D8014600680028F3D100E023E000298D
:10B1400014D0086820600C6012F02CF816494118E1
:10B150000098816407F0B2F9002407F0F7F9286835
:10B16000039000202860002C0DD104E06046206090
:10B1700000984464E8E7012103980DF0BAFF0398B2
:10B180001721006801706846007A00901623019626
:10B190002146039A059800F068FC07B0F0BD000056
:10B1A00030270020505C002030750000F3B50024EB
:10B1B00083B0684604720D4608462746264602219B
:10B1C00006F0F7FE062805D000216A46117201003C
:10B1D0001DD101E01121F8E72C6820684178007842
:10B1E0000E0206432F60218A20460DF043FC2246C2
:10B1F00000210B20FFF7A1F8002813D002A800902F
:10B200002346002231460398FFF792FA014668462A
:10B21000007A00900A2322460196039800F025FC4C
:10B2200005B0F0BD1120694608720621EFE7F3B5BD
:10B23000002483B0684604720D4608462746264619
:10B24000042106F0B6FE062805D000216A461172D8
:10B25000010022D101E01121F8E72C682068417833
:10B2600002780E021643C1788278080210430190DA
:10B270002F60218A20460DF0FDFB224600210D2083
:10B28000FFF75BF8002813D002A800902346314650
:10B29000019A0398FFF74CFA01466846007A00903D
:10B2A0000C2322460196039800F0DFFB05B0F0BDA9
:10B2B0001120694608720621EFE70000F3B5A1B03E
:10B2C00000266846868408A8067008680D46018A2C
:10B2D000062903D0142901D00A213CE1284606F0B2
:10B2E00068FE062805D0002108AA1170010076D159
:10B2F00001E01121F8E7296808684278037817020D
:10B30000C2788078140204431F430120A7420AD860
:10B31000002F08D00B8A042216A81B1F0AF0ECFD90
:10B32000002806D0042008A9087069468F840A21E5
:10B3300011E116A80AF09EFE0521C902884202D03A
:10B34000491C88424CD116A90B9108A90F9121984C
:10B3500009A9129100210E940C46029108A90C70C3
:10B3600069468F84FFF720F811902E682C60318A8F
:10B3700030460DF07FFB324601211120FEF7DDFF44
:10B380001590002832D0002000901598047079485C
:10B390000568002D77D06889B84275D30E99884228
:10B3A00073D8009800284BD068680AF063FE052126
:10B3B000C902884202D0491C88421CD1119A0099C6
:10B3C0000C9103A913916946097B3046102914D0CA
:10B3D0001421038A5B18934211DD04241FE0BAE0B4
:10B3E000102108A8017068468784B4E0112008A9DC
:10B3F00008700624AEE0688968E00621E9E70DF0F0
:10B4000086FD040016D00C990FF0AFFFA01C029926
:10B410000FF0ABFF211D13980AF030FD002400202F
:10B4200000900290002C0BD0129869890180062CA4
:10B4300002D08DE00624F2E70F991120087089E010
:10B4400068680B990AF0FCFC002840D103A80F9B08
:10B4500013900CAA1CA80293019200902946102375
:10B4600000224548FFF718F9040006D16846028E0D
:10B470001CA913980AF066FD0446002C06D0129809
:10B480006989018064E02DE021E024E015980078CE
:10B49000002804D006280ED014284AD110E06846AF
:10B4A000007B102803D01599142008700CE0159922
:10B4B0000620087008E06846007B102839D103E0B8
:10B4C0006846007B102834D06889009002902D686F
:10B4D000002D00D05FE700980024002829D0002D1F
:10B4E00002D003E0002424E02348029000990B914D
:10B4F00003A90D916946097B119A029D30461029D6
:10B5000006D01421038A5B18934203DD042410E063
:10B510000621F7E70DF0FBFC070012D00B990FF0A6
:10B5200024FF2946B81C0FF020FF391D0D980AF0A2
:10B53000A5FC308A022809D80F980A21017005213C
:10B5400009E006240F9911200870F2E7002C0FD0B3
:10B55000042C0DD021466846828C08A80078019200
:10B56000009010233246219800F07FFA23B0F0BDFE
:10B570000021F0E730270020FFFF0000F3B587B07F
:10B5800000246846048104730798059002A804907B
:10B590000D4603AF0598FEF707FF069006F0F3FC93
:10B5A000060007D0324621460F20FEF7C6FE0028CF
:10B5B00009D037E02E6811202C6021466A461073AE
:10B5C0000624118136E011206946087300200881A5
:10B5D00006242FE02846022106F0EBFC062809D0BD
:10B5E0000021002F00D03970040005D004980021FC
:10B5F00001801FE01121F4E7286800680BF02AFDA4
:10B600000190022128680DF035FA00973346002298
:10B6100001990598FFF78CF8040003D0049901986C
:10B62000088007E02868008A022803D3308A069938
:10B630008842CFD368460389007B0193009032464D
:10B6400021460E23079800F010FA09B0F0BD000063
:10B65000F3B5A7B00C46002669460E820E7320682B
:10B66000078A062F03D0142F01D00A2015E12046A7
:10B67000394606F09EFC062805D000216A46117363
:10B6800000287DD101E01121F8E72168086842789F
:10B69000037815021D43C278837810021843009086
:10B6A00085420CD8002D0AD03B1F04221CA80AF0AA
:10B6B00023FC002809D0042069460873EDE001212D
:10B6C0006846017305820A20E7E027980C9003A8DA
:10B6D0000D90009E04A80B95002769460F900F73EC
:10B6E0000B9808820E9705972068029027600298B1
:10B6F0001CAD018A0DF0BEF901210920029AFEF766
:10B700001CFE159000280BD00C98FEF74DFE00246F
:10B710000790001F149080B21690002C06D008E00D
:10B720001120694608730F820620C3E06748046849
:10B7300000E02468002C36D06189B14233D8002D56
:10B7400005D0294660680AF07BFB0028F1D1002C67
:10B7500029D061890B988142DFD30020069021A86F
:10B760000A900D980C9F179006F00DFC1190002880
:10B770001BD006981B90119808971994189000E018
:10B780008BE0179809900020694608765048089F7A
:10B7900087420FD006AB01213846199AFEF793FE77
:10B7A000002818D106E005206CE006250DF0DEFB30
:10B7B00028461DE0199918A8096900901998019167
:10B7C0004189C76801221B9B0898B847002813D0FD
:10B7D0006946087609200999002903D069460A7E3E
:10B7E00009990A70070007D011980DF0BFFB384681
:10B7F0000F9962890A8045E01198078A132F08D9AA
:10B8000017980E210170042511980DF0AFFB284602
:10B81000EEE73A4600210A9B0DF002FB0020009063
:10B8200011980DF0A3FB149900988F4200DD169F2C
:10B83000059900291CD0BAB2914223D10299079BE5
:10B840000A8AB9B2891C52189A421BDC89B2029842
:10B850000DF05DFB00280ED061890170090A41706E
:10B86000BAB221A9801CEEF714FE01200E9054E715
:10B87000B9B20591E2E70D99112008700F9861891E
:10B88000018006200E99002914D00D99002008701F
:10B890000599159A891C1170029E69460A8A097BCE
:10B8A00000910192014608233246279800F0DDF806
:10B8B00029B0F0BD0D990978002902D10D990A220D
:10B8C0000A700028E8D10520E6E7000030270020B4
:10B8D000FFFF0000F3B50C4683B0002569460D72EA
:10B8E0002E462046022106F064FB062805D00021E2
:10B8F0006A461172010022D101E01121F8E72068A7
:10B900000068417800780E02064306F03CFB1127E0
:10B91000054600281ED0024600211320FEF70DFD2B
:10B9200000281AD0022120680DF0A4F802A8009087
:10B93000234600223146039800F0ECF801466846A1
:10B94000007A009012232A460196039800F08DF8A1
:10B9500005B0F0BD0020256820606846077206210A
:10B96000EDE770B505460C46084682B0022106F0A8
:10B9700020FB062817D000216A461171002810D13B
:10B98000206801684A78097816020E4302210DF0FA
:10B9900071F801A80090234600223146284600F0A5
:10B9A000B9F802B070BD1121E6E70000F8B5124CFD
:10B9B000606810F0D3FD0026104D666028880028CE
:10B9C00018D0142148430FF0DDFC6060031E0AD03C
:10B9D0000BA00090142229880F480DF07DFD00284F
:10B9E00008D00B2500E00625606810F0B7FD28465A
:10B9F0006660F8BD0020F8BD28270020BC27002085
:10BA0000626C655F6174745F7376725F656E747289
:10BA1000795F706F6F6C0000745B00200268002A11
:10BA200004D04068401A00D5002070470048704795
:10BA3000FFFFFF7FFFB5154681B00F460A461C4643
:10BA4000042101200A9EFEF778FC00280AD0057028
:10BA50004470220A8270C6703946019800F0B5F829
:10BA600005B0F0BD062005B0F0BDFFB589B0139F4D
:10BA7000129E14460D0001D0002E29D006F02AFA9D
:10BA800001AA03A90998FEF76BFC002801D005461E
:10BA900001E0002D22D006F059FD002C34D0218A7F
:10BAA00020460CF0E7FF099802940790042101203A
:10BAB0000C9C029AFEF741FC002808D004704770E5
:10BAC0003A0A8270C6700299079800F07EF8002446
:10BAD00020460DF04BFA28460DB0F0BD20680078E6
:10BAE000FEF758FC2146019800F056F822460199CD
:10BAF000039807F0C7F900240546002800D00E2659
:10BB000006F024FD002DE3D006F03DFA0400CAD172
:10BB1000DEE70000F0B516461D4A85B014680A9DA0
:10BB20000022002C18D067898F4212D1002C13D02C
:10BB3000074603966846174902721E4638468F42EA
:10BB400011D002AB22460021FEF7BDFC002818D11F
:10BB500009E02468002CE6D1002D01D001202870D6
:10BB6000052005B0F0BD2069009601906189E46868
:10BB700002223846039BA047002802D0694608727B
:10BB80000920002DEDD06946097A297005B0F0BD75
:10BB900030270020FFFF000070B50D46044606F078
:10BBA00089FD00280FD0A08900280CD0618981422E
:10BBB00000D20846298A081A002803DD4142284697
:10BBC0000CF058FF70BD1720F4E730B50546086843
:10BBD00083B00C460078FEF7DDFB06F07BF96B4680
:10BBE00001AA0421284606F028FA050003D02046C1
:10BBF0000DF0BCF909E021460098FFF7CDFF224681
